:020000040800F2
:1000000000500020817A01081D7B0108A10601082B
:100010001D7B01081D7B01081D7B010800000000FD
:100020000000000000000000000000001D7B01082F
:100030001D7B0108000000001D7B010843A400088F
:100040001D7B01081D7B01081D7B01081D7B01082C
:100050001D7B01081D7B01086FA7000879A7000818
:1000600077A7000875A7000873A700087D6500083A
:100070006D6500085D6500084D6500083D65000878
:1000800029650008156500081D7B01081D7B010816
:100090001D7B01081D7B01081D7B010871A700085D
:1000A0001D7B0108291001081D7B0108191001089A
:1000B00009100108F90F0108E90F0108236C000875
:1000C000296C0008196C00081F6C00081D7B0108D2
:1000D0001D7B010881A4000875A400081D7B010890
:1000E0006DA700081D7B01081D7B010800000000B2
:1000F0000000000000000000000000000000000000
:0C01000000000000000000005FF808F1A3
:100110002DE9F04F0B4B0C4D0C4AC5F8B8340023B9
:1001200010680B49A1B08842C5F8BC3416D11360E1
:1001300062B6084B18680FF09FFF074B1B68984783
:10014000FEE700BF7194000800060020F04F002079
:10015000EFBEADDE00F0FF1F04F0FF1F0A930B930C
:100160000C934FF4E013BC4C0D93236843F480339D
:100170002360A36943F01003A361236803F40033F1
:100180000B930A9B01330A930B9B1BB90A9BB3F594
:10019000A06FF2D1236813F4003300F0FA85022334
:1001A0000C93AE4BAE4F1A6842F010021A601A68F8
:1001B00022F003021A601A6842F002021A606368B1
:1001C000636063686360636843F480636360A54B46
:1001D0001A68043B22F070425A60A34A3A6062688F
:1001E00022F47C1262605A6842F000425A60DA6877
:1001F00022F40042DA609B681E0449BF9B4B4FF417
:10020000E0133B604FF480130D930C9B012B00F027
:10021000D985022B05D10D9B6268134343F48033CB
:100220006360236843F08073236023689801FCD5E2
:10023000636823F003036360636843F00203636051
:10024000636803F00C03082BFAD16368DFF86C8253
:1002500003F00C03042B00F0BA85082B00F0BA85DC
:10026000814BC8F800306368DFF85492C3F303137E
:1002700019F80320D8F80030DFF848B2D340C8F8A6
:1002800000307B4B4FF6FF72CBF80C30A3690DF1B9
:10029000800A43F00103A361636A636A754E43F009
:1002A00080736362A369304643F01C03A36100239B
:1002B00015932AF82C2D51460FF066FE51466E48D4
:1002C0000FF062FE51466D480FF05EFE02214FF4C2
:1002D00000728DF846101021ADF844208DF84710BB
:1002E0003046326111A90FF04FFE654950464A6809
:1002F00042F000724A6014F06FFE159B614A30466E
:10030000B3FBF2F34FF47A72C5F8C034D8F800307A
:100310004FF0010CB3FBF2F35B4A013B5360F02357
:100320008BF82330002393600723DFF89CE11360F0
:10033000564A09F10E01002331F8026F46FA03F81C
:1003400018F0010F18BF0CFA03F803F101031EBFE8
:100350001060A2F804800832102BEFD100F5806005
:100360007045E8D13B68404A934240F046850123FE
:1003700085F8C43409F093FD18B910F0FDFC10F0B5
:10038000DDF910F019FB0522414942481AF084FAC0
:1003900018B110F0F1FC10F0D1F995F8C5343E4ECB
:1003A00043F0010385F8C5343C4BDFF820819A788F
:1003B0003B4B08F1050A1A703A4B1B68336095F8FD
:1003C000CA3485F8C634002313F808004FEA830BBB
:1003D0005F1C002800F0188503930AF0D5F8039BF2
:1003E0004AF8230010B10523C771837112215AF80E
:1003F0000B000AF0EFF8032F3B46E5D10021084639
:100400000AF04AF9002101200AF046F900210220F1
:100410000AF042F9012102200AF03EF9A369002105
:1004200043F00103A36140221F481AF0F2F94FF094
:10043000FF331E4AC5F818356420C2F8033009F0AE
:10044000F6FFA02200211A481AF0E3F90024194D02
:10045000194F002360593BE0001002400020024089
:10046000200400200410014000127A00001BB70095
:100470000005FA0500080140000C01400010014091
:100480000000014040420F0010E000E0301C00205E
:10049000B4C70108012000208C210020FC1F00208F
:1004A00080210020C8200020D80A0020180B00203E
:1004B000AC3A0020A0C6010884A901082000002051
:1004C0006CA9010800ED00E000140140C70A0020FB
:1004D00057F83310DA00884240F09A8409EB02039F
:1004E000187F103414F044FAE02CB2D1B94ABA4C57
:1004F0000021A0469146B94F00250B5D01F10F0088
:10050000204407EB030A10F801CFBCF1000F05D01F
:100510009AF80CE0E64508BF82F858E090F803C06E
:10052000BCF1000F05D017F803E0E64508BF82F8DC
:1005300059E00135032DE6D1B2F8580040B108EB7F
:10054000010009EB83035065C3F8202502F51772FB
:100550001C313829D0D104259E4C00212022A048EE
:10056000366884F82C551AF054F94FF0000E4FF00D
:10057000FF0A7146994F2B4697F80B9097F80AC0DF
:100580009748984D06F040084A571E2A827140F05D
:100590004684B8F1000F00F04C84BCF1000F00F06D
:1005A00048840131042900F10800EDD1BEF1000FAB
:1005B00001D084F82C3516F0010300F08784002563
:1005C000FF2294F82D85884B2946404683F84050F9
:1005D0001D605D609D60DD6383F8412083F84220EB
:1005E00083F8435083F8445083F8455010F0E2FC00
:1005F000064690B303687D496A18507C18B152686A
:10060000934200F01E841835C02DF5D10025C4F8A2
:100610003C6584F83055404609F0B6FF10B102231E
:10062000C571837100252A2109F0D4FF704A002189
:10063000304609F001FE6F4B6F4AC4F840356F4BEE
:10064000111F3046C4F84435C4F8485509F048FE37
:100650002A467179306811F021F9B4F81E8694F8B1
:100660001A66A4F820863046B8F1000F40F07F8467
:1006700009F08AFF94F81B26C4F82406003218BF3C
:10068000012284F8282658B1242294F81C3682715D
:10069000002B80F807800CBF1221162109F09AFF69
:1006A000002009F0CDFF4FF000080020C4F8487684
:1006B00005F012FF012005F00FFF5149514801F1EB
:1006C000200C51F8056C6EB311F9092CA31893F89E
:1006D0004C7693F84EE693F8509600EB02158B1E7D
:1006E00013F801AFBA4593F802A008BF2F71F24585
:1006F00093F804A008BF85F805E0CA4508BF85F84F
:1007000006908B42ECD1120183181D7955B15D79A9
:1007100045B19D7935B186504A7983F80C80DA71FC
:100720008A791A7210318C45CBD1364D14F0D0F93C
:1007300014F0CEF9287E14F01BF901232A7E02F072
:100740001F015209022A03FA01F300F03D84032A33
:1007500000F04084287D09F017FF064618B11223E7
:1007600083710223C371687D09F00EFF18B1132352
:1007700083710223C371A87D09F006FF18B1142309
:1007800083710223C3711B21304609F023FF687D6A
:1007900009F0FAFE072109F01DFFA87D09F0F4FE1B
:1007A0001B2109F017FF2A69174B9A4240F0188461
:1007B00003F56043D96841F48051D960D96821F4C8
:1007C0008051D9602B7F002B00F02784002318462E
:1007D0001CE000BF00060020A4A90108D8270020C3
:1007E0003C370020DCA90108643A00204C28002096
:1007F00040420F00755C0108440B0020B15D010808
:10080000E9A90108E415002000300140118801F435
:10081000415141F4457101430B431380938B23F401
:1008200000631B041B0C93830723138213889BB262
:1008300043F04003138094F8C434032B11D11F20DC
:100840000AF00FFA0023C84A02EBC30191F9021023
:10085000022901F01F860133042BF5D102200AF092
:1008600000FA08F01DFE012005F090FE2C2009F092
:100870008BFE9F238DF844300023C4F854063220A9
:100880008DF845308DF846308DF8473009F0CFFDB2
:10089000D4F8540609F0C0FE042315AA11A9B348E0
:1008A00009F08CFFD4F8540609F0BBFE9DF85630D1
:1008B0009DF855201B0243EA02439DF8572013433D
:1008C000AB4A93421FD0322009F0B1FDD4F8540650
:1008D00009F0A2FEF521A54809F09EFFFF21A348DB
:1008E00009F09AFF8DF85400D4F8540609F099FEE7
:1008F0009DF85430702B06D194F8C434022B02D1E9
:10090000032384F8C4349B4B5E799F7906F1FF3C46
:10091000DCF1000207F1FF3842EB0C02D8F10003D2
:1009200043EB080384F85C36934B84F858261D6823
:10093000079315F4004F40F0748315F0007507D04D
:100940008E4BDD7AA5F1080EDEF1000545EB0E05B4
:10095000142200218A4884F85A5619F05AFF012EB1
:1009600004BF94F8593684F860361DB194F85B36AC
:1009700084F86F3694F85E361BB194F85F3684F8CD
:100980006A36012F08BF94F85D367D4D08BF84F8A4
:10099000653600232E464FF0070B1F469946DFF8B9
:1009A000008208F1940A3078E8B109F0EDFD18B141
:1009B00080F806B080F80790002109F00BFE0023B4
:1009C00031781AF813005A00884240F02C8308EB63
:1009D000020393F8953073700723337101237A1C57
:1009E000B770F370D7B20BF1010B5FFA8BFBBBF161
:1009F0000B0F06F10506D6D1002B00F0DA80614E10
:100A00004920736843F44043736013F0B1FF5E4ABA
:100A10005E4900234FF01C0E104688460EFB032C47
:100A2000DCF804C08C4540F00483DBB21C2101FBE0
:100A30000303726919694FF000090A4372610622C3
:100A400083F819901A76514814F04DFA15A814F04D
:100A50001FFA4F4B022F159334BF4B4680231A9336
:100A60004FF480731B934FF480631C9320231D93DA
:100A70004FF40053474E15A9444818971E931696F5
:100A8000CDF85C90CDF86490CDF87C9014F00DFA20
:100A9000012F94BF00220122D8F800303E4943F0D4
:100AA0000103C8F800304B684FF0070E23F47023A1
:100AB00023F4807343EA02234B608A68374B134068
:100AC00043F4602343F002038B60CA6A7B1E22F466
:100AD0007002DBB242EA0353CB621F270123EA789C
:100AE0004AB395F80180581CB8F1090FC0B295F8C7
:100AF00004C040F2A482A8F10A02D1F80C9002EBE3
:100B000042020EFA02FA29EA0A090CFA02F242EA51
:100B10000902CA60062B00F29F8203F1FF3C4A6B78
:100B20000CEB8C0C07FA0CF322EA030308FA0CF224
:100B30001A434A6303460535AE42D0D1164B9A6834
:100B400042F480729A609A6842F001029A609A6850
:100B500042F008029A609A681607FCD49A6842F03C
:100B600004029A600C4B1DE016370020003800404C
:100B700015202000862B00208C21002054220020EC
:100B8000600C0020001002402400002008000240F9
:100B90004C240140740C002000240140FDF7F1FFBB
:100BA0006CA901089A685507FCD49A6842F4A0021F
:100BB0009A60D4F87C06002841F07784D4F8803617
:100BC000002B41F07284D4F88436002B41F06D8400
:100BD0000CF0D4F930B90120022109F09BFD01206D
:100BE00015F08CFD012194F8C534084643F002034A
:100BF00084F8C53409F050FD0021084609F04CFD89
:100C00000021022009F048FD4FF00A0B924C012010
:100C100009F0ACFC002009F0A9FC192009F007FC40
:100C20002368D80302D4012009F00AFD192009F035
:100C3000FEFB002009F004FDBBF1010BE7D1594692
:100C4000584609F029FD5946012009F025FD0FF00D
:100C500021FE824B18680DF0C5FC814B1A88814B30
:100C60001A80814B5B6B0BB10CF070F97F4A804BA3
:100C7000127898461A70079A7E4F15687E4C15F4C4
:100C80008055DFF83C927D4E00F00382A08816F07C
:100C9000A9FA7B4B3860C9F80030708A16F0A2FAC6
:100CA000784BDFF820921860608816F09BFA764B3C
:100CB0001860208816F096FA744B1860B9F81A007C
:100CC000C0F5FA6016F092FA714BB9F818901860F6
:100CD000E388704AA9EB030099446F4B80B21FFA76
:100CE00089F91080A3F80090A0F57A7016F07EFACA
:100CF0006A4B1860C9F5FA6016F078FA684B18600C
:100D0000B38A03930DB1A3880393B378042B05D161
:100D10004FF4805008F0E2FC00230393002598F87C
:100D20000020604CA2F11703022B257000F2CA814B
:100D30004FF0000ADFF89081514655F8080005EBA6
:100D4000080916F03BFC002800F0AD81079B1B68EA
:100D5000D90400F1D88100233968534A42F823109E
:100D60000133082BFAD12378C02200214F48069383
:100D700019F04FFD3779B378003718BF0127042BDE
:100D800000F2E681DFE813F0D603E401D8030402A1
:100D9000D003226842F0010222600A93236803F024
:100DA00002030B930A9B01330A930B9B1BB90A9B0B
:100DB000B3F5A06FF2D123689F0702D50123FFF797
:100DC000EFB9FEE7636843F46013FFF729BA3B68A5
:100DD000FFF747BA63686268C3F38343D10303F143
:100DE000020303D4324A5343FFF73BBA626812F45A
:100DF000003F3A6818BF5208F5E72E4A93427FF445
:100E0000B9AA0223FFF7B4BA4AF82300FFF7F3BAEE
:100E10000133042B7FF45CAB0020FFF762BB1F2A79
:100E20007FF4BFABB8F1000F03D0B9F1000F7FF42E
:100E3000B8AB013B80F806A0DBB24FF0010EFFF724
:100E4000B0BB1B8D1C4A9BB212680133B2FBF3F39B
:100E50001A4A1370FFF7DABB541E00209C200020B2
:100E6000A6200020701500202420002088210020CA
:100E70005C11002094290020343C0020B837002069
:100E800000007A44F81F00209811002078110020FB
:100E9000A011002072110020941100209011002058
:100EA0009C110020D4370020242800204C2800204A
:100EB00000093D00001BB70020000020280400208E
:100EC000D037002054220020481D0020B2047FF5B6
:100ED000C4AB1E4694F818169F4AA04D117005F138
:100EE000D00916F8092000211046039210F062F88C
:100EF0008046A8B300234FF0010B039A5FFA86FAED
:100F000005F80E3C05F80D3C45F8040C05F80FAC4F
:100F100005F810BC104609F037FB0AEB0B03DBB2F7
:100F200010B180F806B0C3714FF0000B2A2109F010
:100F300051FB8B4A0021404609F07EF9894B2A1D5E
:100F40002B60894B294640466B60C5F808B009F014
:100F5000C7F95A4698F80510D8F8000010F09EFC22
:100F60000136082E05F11C05BBD1FFF776BB09F051
:100F70000BFB4021C4F840060546304610F01AF835
:100F80000646CDB1C0B12423AB7101231A21EB7108
:100F9000284609F01FFB0021A4F8448601917349FB
:100FA0006F4A91FBF8F192FBF8F389B200919BB282
:100FB00031466F4814F0B4FF0023D4F82C26138078
:100FC00084F83D36FFF76FBB6A4AD1680B43D360A4
:100FD000FFF7C0BB674A11690B431361FFF7BABB48
:100FE000654B9A420BD103F5EC33196941F480410A
:100FF0001961196921F480411961FFF7E3BB5F4B67
:101000009A427FF4DFAB03F5EA33196941F40041FA
:101010001961196921F40041EEE701230220FFF76D
:10102000F5BB012594E401330A2B7FF4CAAC0023FD
:10103000D1E40133072B7FF4F1AC0023F6E40A6915
:1010400008EB480A0EFA0AF922EA09090CFA0AF230
:1010500042EA09020A615DE50C2B0DD8DA1FD1F8CE
:1010600030C002EB820207FA02F32CEA030308FA0B
:1010700002F21A430A635DE50D3BCA6A03EB830380
:1010800007FA03FC22EA0C0208FA03F31343CB62CB
:1010900050E5B08A16F0A6F83860308A16F0A2F84B
:1010A000C9F80000F9E5364B05EB030E99E80F008F
:1010B0008EE80F00237810350133802D23707FF4E4
:1010C0003BAE43E62F4B13F8321003EBC203082963
:1010D000217088BF0821D3F804C088BF2170BCF1FB
:1010E000000F3FF433AE0025DFF8948023789D4253
:1010F000BFF62CAE2B0103EB080E63440FCB01357A
:101100008EE80F00F2E72378012B7FF624AE4FF034
:101110007C591D4D05EB031303F110081035A8454C
:101120003FF419AE494655F80C0C16F0B3F8494691
:1011300045F80C0C55F8100C16F0ACF8494645F87B
:10114000100C55F8080C16F0A5F845F8080CE5E762
:101150000E4CA0461FE000BFFC270020400B0020E3
:1011600040420F00055E01084D5C010820A1070008
:101170002C0C00200010024000380040003C0040D1
:10118000A411002054B00108A81100206F120339E7
:10119000AD4CDFF84483AD4AAD4B21461A60AD4AF1
:1011A000AD4B4046002F18BF1346AC4A00251360D4
:1011B00015F068FF01464FF07A5016F01FF9A84964
:1011C0000590204616F066F8A64CDFF810A30790AD
:1011D000069BAB4240F30F8205EB0A035E790021C8
:1011E00030460FF0E7FE0490002840F0A7819E4AA9
:1011F000974B1A60974A994B1A609C489C4990F803
:10120000C5349C4D43F0040380F8C5349A4B9B4C85
:101210001B788246DE0031444A78994922602A6868
:101220000395114009B101222260002140F2DC50F7
:10123000944A22F8110001310829FAD12268002AC3
:1012400040F0F08103F0EF02082A8F4A40F00A8252
:101250001178182B41F01001117001D10DF07EF9B9
:1012600023688A4D002B40F00682AB89002B40F0AA
:101270003B82874B15AE587A15F0B8FF854916F0BA
:1012800009F8854915F0FEFE08F0A9FC834B1860AB
:10129000834B988A15F0AAFF0146824816F0AEF8F3
:1012A000CAF8880612F0BAFB01231593102316938F
:1012B000039B1B685A0201D47B4A1592DF0058BF7A
:1012C000159A7A485CBF42F010021592784A049051
:1012D00011688D0742BF159A42F0C60215924C075D
:1012E00042BF159A42F008021592159A42F0006129
:1012F0001591017801F0EF04082C01D00E2904D1DA
:1013000042F0006242F480521592159AD80354BFFD
:1013100042F4005242F420421592159ADF044CBF69
:1013200042F0644242F0444215929D0642BF159A33
:1013300042F4807215925C0742BF159A42F4003263
:101340001592159A42F400201590580505D5594B71
:101350001B7913B142F4C01215920125182902BF5E
:10136000159B43F060731593594630465FFA8BF432
:1013700008F0D8FD78B1204614F073FF58B94FEA51
:101380005B1256F8223004F01F0405FA04F423EA35
:10139000040446F822400BF1010BBBF1250FE3D109
:1013A000DFF83C8196E803004FF4197288E80300E7
:1013B000002108F1080019F02CFA09F071FE002252
:1013C0003D48DFF820E18346F4463C4B3C491A8017
:1013D0009A703C4D3C4B3D4C19603D4F2B8BDFF8D8
:1013E00008916760A0608AF8F82819B208F51C789F
:1013F000D9F800002EF8121000F5967048F8220077
:101400000132122AF4D1039A1068C20458BFB5F908
:101410002410ACF806102F49DFF8C8C001F1500EB7
:101420000A78002A69D18A7891F80380424564D20B
:10143000002A00F06981013A02EB820202EB82028B
:1014400002F5617252E000BFACC5A737615E0108CA
:10145000182E0020E15D01088D5E01081C2E002081
:101460006F12833A4C280020E35D0108000600203B
:1014700054B001088C2100205C11002024120020AF
:10148000200010005421002049150020B41A00202B
:10149000542E002035FA8E3CDB0FC93F742E0020FD
:1014A00024200020A889803A010000108821002013
:1014B0008421002024220020A1DD0008982B002098
:1014C000A086010054220020FC1700201C180020D8
:1014D000A5DD0008601E0020ACC5A736B837002087
:1014E0008C0C0020542B00209822002091F80180C1
:1014F00092B208F104082CF8182004318E458FD1DF
:10150000020740F19C81287A0A2800F29281DFE8E4
:1015100010F01F011F016104A004C404E404E404EA
:101520002805900165051F0100240023A04601271E
:10153000039330E6794CF8E7794C0AE6304609F037
:1015400023F86B1C6061DBB210B10322C37182719E
:101550001A2109F03FF8002F51D0BAF8000015F019
:1015600045FE16F099F86F4B4FF6FF791E68B6FBF3
:10157000F0F34B441B0CB6FBF3F60FB1B6FBF0F9DE
:101580009AF80230042B3ED1484615F02BFE6349F1
:1015900015F080FEA0600990304615F023FE41460C
:1015A00015F078FE099B08905F49184615F072FE09
:1015B000089A0146104615F063FD9AF80330E06082
:1015C0000193039B3246009304991FFA89F3204646
:1015D00014F0A6FC002318225449AB4218D1002372
:1015E00083F00103237401231D44082D637404F167
:1015F00018047FF4EDAD01224D4B1A70FDE50598FE
:1016000016F0B2FDADE7304615F0ECFD0799BFE7E7
:1016100002FB031046686068864201D00133DCE7B4
:101620000123DDE7434A444912F8335032445668F7
:101630000D70002E3FF406AE0020404FA842BFF6CA
:1016400001AEC0EBC0017218D2F800C001EB070E6A
:1016500041F807C091880130AEF8041092798EF8F5
:101660000620EBE70E2B3FF4F3AD1178192B21F098
:1016700010011170F1E500244FF00409304E05F11E
:10168000030818F8017F002F3FF4EFAD384608F04B
:101690007BFF013403467061E4B210B180F806901C
:1016A000C4710021384604930FF084FC0746049B64
:1016B0001A21184608F08EFF002F3FF4D6AD6B8834
:1016C000204A304692FBF3F3002201922A889BB213
:1016D000009239461B4A14F023FC0123082C737432
:1016E00006F11806CDD1C0E50024174F174EA88982
:1016F00015F078FD3A6801463019243408F080FB73
:10170000B4F5907FF3D1B4E508F1010808EB88083F
:1017100008EB880808F56172E8E600BF6F12833AAB
:10172000282930382000002000007A444C2800206E
:101730002812002070AF010855190020561900200A
:101740004C3B002040420F00682100204C1200203A
:10175000B84B40201C6009F081FC8046002868D00E
:101760000023B54A0693137005920EF0F3FD297A13
:1017700081460129059A0DD0069BC0F0E8820A290E
:1017800016D1AE4B1B6813F480631CBF80F00103BD
:10179000DBB213700322AA4B1A700722A94B1A70EE
:1017A0000122A94B1A700C23237042F6F8236380A0
:1017B000A64B6360A64BA36098F90200DFF878821D
:1017C000B9F1000F40F0D08298F80030002B0CBF28
:1017D0000123032398F80020002A40F0C782AA7A48
:1017E000002A0CBF0022082201920093994A4FF46C
:1017F000E133402109F07EFA974B1860B9F1000FF0
:1018000001D0964B18606B7D2178013BDBB2944A86
:10181000994213709CBF0023137030B198F80030C8
:101820001BB101228F4B83F84429003018BF0120DF
:1018300028B9082007F052FF6760C4F808B0039B7E
:101840001A6850040BD51223237044F6206363807A
:10185000854B86496360864BA360864B196042F2D4
:1018600001031A4209D044F620639104638040F1D9
:10187000E18308232370804B636095F8283021783A
:1018800004338B42A8BF0B464FF000087B4CD703B4
:101890008AF8453984F8008040F18A8112F038FDD9
:1018A00001232370764B40F22A3293F8F19041469F
:1018B000744818F0AEFFB9F1000F00F06C8141469A
:1018C00048460FF077FB704F036804463B6083681F
:1018D000002B00F06081484608F056FECAF848091F
:1018E00018B1282380F8078083711B2108F072FE4D
:1018F000664A00239046396802F1180E5EF83300FC
:101900004FEAC30C814240F09C836244107F13F085
:101910002FF838685E4A03884FF0000923F001036E
:101920001B041B0C03805B4BDFF878E11B68ADF8F0
:101930003E90934281BF03F1B772574902F5585266
:10194000B2FBF1F292BF002202F1FF3292B2511CBF
:10195000B3FBF1F35149ADF83A90B3FBF1F3032136
:101960009BB2B3FBF1F14FEA410CAEF800C0DFF8D7
:1019700038E18DF84090AEF8001020A921F8482DEC
:10198000ADF83C3013F05DF86023ADF84690ADF84B
:101990004890ADF84A90ADF84C90ADF85090ADF845
:1019A0004E90ADF85290ADF84430E3794FF0000915
:1019B000580757BF0122042303F00203ADF8462065
:1019C0004EBFADF848304FF48072ADF84C304FF058
:1019D000000358BFADF85020ADF84A3011AA617924
:1019E00038680FF0F3F96179386812F0FDFF3B6851
:1019F0002B48B3F84420DFF8B4A06FEA42426FEA04
:101A0000524292B2A3F844201A8892B242F0800265
:101A10001A80E279617912F0040F14BF04220122C6
:101A20008A40198C92B289B221EA02011984198C78
:101A30003EE000BFC4180020C91800208C210020FF
:101A4000C3180020C8180020DB16002011D9000898
:101A500069E0000889E1000828190020842200209C
:101A6000C2180020000600201DDE0008400D030003
:101A700005DE0008FC170020F5DD0008332B0020F0
:101A8000AC29002098300020C83300206CA9010840
:101A9000FF6BDC0220000020006CDC0200350C0033
:101AA000001002409630002094300020C433002003
:101AB00089B20A431A841A8892B242F001021A804B
:101AC0001C22217BAA4B02FB013142690B691A439C
:101AD0004261282281F819900A76426913434361D2
:101AE000A44BC1F814908B604B7B15A88DF8543033
:101AF00001238DF856908DF855308DF8573012F03F
:101B000055FFA068CAF8000013F0EDF9DAF80000FC
:101B1000036823F001031B041B0C036013F0E3F9BB
:101B200015A813F0B5F93B68627934331344159363
:101B300040F22A33189380231A938F4B15A91693DA
:101B4000102317934FF400731B934FF40053DAF8EC
:101B500000001E93CDF86490CDF87090CDF87C9085
:101B6000CDF8749013F0A1F9637938680C2B88BF15
:101B70004B4681899CBF08EB4308B8F8A83089B26E
:101B8000DAF800200B438381136843F002031360EB
:101B900001227A4B1A700023FF211C4678481A183C
:101BA0001C520433802B9170D170F8D112F020FCBC
:101BB000744B1A68984612F4806F4BD0042009F0D9
:101BC0004DFA714B0421186009F03EFA6F4B704CCE
:101BD0001870082009F042FA6E4B0821186009F0CD
:101BE00033FA6D4B2C221870002104F64C1018F0BB
:101BF00010FE7C2384F84C398E2384F84D39E02381
:101C000084F84F397D23202084F8773909F026FAAB
:101C1000624B2021186009F017FA614B18701020F0
:101C200009F01CFA5F4B1021186009F00DFA5E4BA9
:101C300018704FF4805009F011FA5C4B4FF480514A
:101C4000186009F001FA0022594B1870594B1A70AC
:101C50000EF098FB584C2288002A40F05F824C4FCF
:101C600007F67C13C7F87839022387F87C3997F890
:101C7000893997F88809013B5BB2012BDEBF4F4AD7
:101C80001B01D258C7F88029002800F0478208F0CD
:101C90007BFCC7F8840918B11A2383710023C37130
:101CA000132108F097FCD7F87839986808F0B9FC48
:101CB00000BFD7F878390221586808F05EFD4FF070
:101CC00000099F2332208DF844308DF845908DF81F
:101CD00046908DF8479008F0AAFB8DF8559000BF0C
:101CE000D7F87839986808F097FCD7F87809324621
:101CF00011A90423406808F061FDD7F87839986885
:101D000008F08FFC00BF9DF856309DF855201B024F
:101D100043EA02439DF857201343294A934200F0B7
:101D2000468300F39481274A934200F0998101325F
:101D3000934200F0E681A2F51A42033A934200F082
:101D4000318300232380A3816360A360E6E1022145
:101D50001D4A117003211D4A11701D4A137007237B
:101D6000237045F2F05322E5032333E508223BE5D7
:101D7000240000203D5F000898300020C23300207E
:101D8000A02A00208C210020802200208822002010
:101D900000060020502200208922002090220020EE
:101DA0008B2200209C220020A1220020A4220020BF
:101DB000A2220020A322002010040020E41500200D
:101DC0001620C20017BA2000C3180020C81800202F
:101DD000DB1600200A221B0193FBF2F30022A1492B
:101DE000A3F5B06341F822300132122AFAD142F64B
:101DF000F82363809C4B402063609C4B2270A3605F
:101E000009F02CF9804600283FF413AD0EF0A2FA39
:101E10006B7AA97A00280CBF01220322002B0CBF89
:101E20000623072300290CBF0021082198F902E0AE
:101E300080460B438DE80C008D4B8E4A4021704646
:101E400008F058FFB8F1000F3FF4EFAC8A4B186070
:101E5000EBE41023237042F6F8236380874B402085
:101E60006360874BA36009F0F9F8804600283FF4CF
:101E7000E0AC0EF06FFAAA7A00280CBF012303230E
:101E8000002A0CBF0022082298F902E00192009378
:101E900080464FF4E1337B4AD0E70823237042F6B3
:101EA000F8236380784B40206360784BA36009F08F
:101EB000D5F8804600283FF4BCAC0EF04BFA002267
:101EC00000280CBF0123032398F902E0019200933C
:101ED00080464FF4E1336E4AB0E700234FF00C0E1A
:101EE0006C4A6D4913706D4A062884F800E00B7047
:101EF00013702BD01B226A4B4FF4E1391A70052264
:101F0000684B83F800E0684B1A7042F6F823638050
:101F1000664B40206360664BA36009F09FF88046E3
:101F200000283FF486AC0EF015FAAA7A00280CBF00
:101F300001230323002A0CBF0022082298F902E0A3
:101F40000192009380464B465A4A77E72122544B30
:101F5000DFF89C911A70534B83F800E0524B1870D5
:101F6000D3E74FF00009544B402083F800900E2334
:101F7000237044F620636380504B6360504BA36032
:101F800009F06CF800283FF454ACB0F800804D4BD9
:101F900008F4825883F80090AB7AB8F5825F90F924
:101FA000020014BF01220322B3B9B8F5825F14BF47
:101FB0004B4608238DE80C0040214FF4E133424AA0
:101FC00008F098FEB8F5825F7FF42FAC00223F4BFB
:101FD00018603F4B1A7028E40823EBE70A221B0124
:101FE00093FBF2F300223B49A3F5B06341F82230A2
:101FF0000132102AFAD142F6F8236380364B402092
:102000006360364B2270A36009F028F800283FF483
:1020100010ACAB7A90F90200002B0CBF0023082310
:10202000019303232E4A009340212E4B08F062FEB9
:10203000FFF7FBBBD3077FF520AC0C2323702A4BA3
:102040001AE40133042B7FF459AC00205FE4274AE3
:10205000934200F0AE814DDC023A93427FF471AEC0
:102060008023A0E10C17002039D9000855D90008B9
:10207000A0860100D5E100088422002075D8000860
:1020800089D80008C5DF0008EDD7000805D800088A
:102090007DDF0008911800204015002090180020D6
:1020A000341600205816002092180020EBCC0008AF
:1020B00001CD0008A5DE0008EB1800202DDE000889
:1020C00061E30008E91800208DE2000810220020DA
:1020D0001C22002070170020D5DA000805DB00085C
:1020E00029E20008A0680600E5DD00081920C2000A
:1020F00090D00300BA4A9342B2D0013293427FF4A7
:1021000020AE4FF480732380A381638822881B0252
:1021100063605343A360012387F88A39A468B4B18C
:102120004FF00009E40A0DF1540AA1450ADA09EB5F
:1021300004077F1010223146F80210F06DFD0F28C1
:1021400000F33A8107F018FFA64BE4021C6000235D
:10215000A54AA64C1360A64A1380A64A1380A64A35
:102160001380A64A1360A64B1A689A461F2A40F0AD
:102170002D814FF48063A34A23801188A24800294F
:1021800040F07C8101809278A04B02B101221A704C
:10219000B4F900309E4A1B021360049B9D481B78D3
:1021A0009D4C052B02BF4FF4C8729C4B1A800AF05D
:1021B00031FEC8229A4B00211A809A4AA4F88C1941
:1021C0001378A4F88E1943F0080313700423964A79
:1021D00084F88B391370954A954B117064221970ED
:1021E0005A705960934B19805980934B5A7999468C
:1021F000012A0BD1282204F5196018F00AFB4CF2D1
:1022000050328E4904F6941007F0FAFD00218C4BF1
:1022100084F8B81919605960996099F80630012B53
:1022200009D11022874818F0F4FA4CF2503286494E
:10223000864807F0E5FD864B864A1B684FF0010B88
:10224000C8F80030844B80201B68844F9B1A18BF4D
:102250000123834A834E137014F050FA0021402268
:10226000814884F8F0B918F0D4FA00237F4A384640
:10227000C4F8F439136008F05FFC3368D90709D556
:10228000DAF800305946642BB8BF642358467B64A3
:1022900008F08AFC33689A0709D50121022008F06A
:1022A00083FC734B5B6B642BB8BF6423BB673168E3
:1022B0000320C1F3400108F077FC0121052008F05C
:1022C00073FC6C4B99F805B01A8C6B4B072093FB91
:1022D000F2F3642BB8BF64231BF10001C7F814317B
:1022E00018BF012108F060FC99F806A008201AF137
:1022F000000118BF012108F057FC99F80A30002BA3
:1023000040F05E8199F80B30002B40F05981D8F8ED
:102310000010C1F38041BBF1000F03D1BAF1000FEF
:1023200000D15146092008F03FFC0121042008F0AB
:102330003BFC94F84419062008F036FC01210A20E1
:1023400008F032FC31680B20C1F3800108F02CFC4E
:1023500033680C2013F0140F14BF0121002108F082
:1023600023FCD8F800100D20C1F3802108F01CFCDC
:10237000D8F800104B0507D52B7A083B012B9CBFE2
:102380004FF4FA63C7F8B432C1F300410E2008F0ED
:102390000BFC94F8C53463F07F0384F8C53421B096
:1023A000BDE8F08F202323804FF48073ACE64023F8
:1023B000F9E74FF40073F6E700235AF823200132BF
:1023C0006FD10133042BF8D13C46AEE63F2A16BF4D
:1023D0004FF4FA434FF40073B3FBF2F3CBE600BFC4
:1023E0001740EF00E03300209C3700209437002096
:1023F000A0370020A2370020A43700209837002003
:1024000004370020D033002096370020A637002064
:102410000822002034350020000600200823002078
:102420000623002049150020812B002032220020A5
:10243000841000201E220020862B0020CDCCCC3D15
:102440001C210020BC0F0020CDCCCC3ECC0F0020A6
:10245000C8200020E35D0108182E0020FC000020A9
:102460002812002084210020DC1B0020D81B002023
:10247000242000201637002040420F00B4F900301D
:10248000994204DD1F2B02DD012303807BE693FBD1
:10249000F1F3FAE732F83330002B7EF4E7A9FEF7C8
:1024A000DDB907F1010927468EE70022454B00B24E
:1024B0001A7014F09BFE444914F0ECFE0746B4F980
:1024C000800614F093FE404914F0E4FE0646B4F989
:1024D000840614F08BFE3C4914F0DCFE3B490546B3
:1024E000384614F0CFFD07F07AFB8146384607F0F6
:1024F00076FB36490746304614F0C4FD07F06FFB03
:102500008046304607F06BFB30490646284614F0FB
:10251000B9FD07F064FB8346284607F060FB494697
:102520008246584614F0B6FE49460390504614F0D1
:10253000B1FE59460490384614F0ACFE5146059061
:10254000384614F0A7FE41460690584614F0A2FE05
:102550001F4D5146286008F1004014F09BFE05997C
:102560006860AE60304614F095FE049914F08AFD60
:102570000699E860304614F08DFE0146039814F089
:102580007FFD4146286107F1004014F083FE039966
:102590006861304614F07EFE0146069814F070FD26
:1025A0000499A861304614F075FE059914F06AFD8F
:1025B0004946E861404614F06DFE2862FEF708BB0C
:1025C0000121A8E60E00002035FA8E3CDB0FC93F42
:1025D0004C1500202DE9F04FB34A97B013780192C3
:1025E000002B00F0B280B14B186800286BD006F0C9
:1025F000ABFFAF4FAF4D386807F093FF002862D0B4
:10260000386807F08BFF0928AB4C01D03F2851D127
:102610004FF0000AD046A94ED4F8009006F58C7B06
:10262000B9F1000F05D04A463168284618F034F950
:1026300018B9B246B8F1000F2FD008365E45EFD377
:10264000B8F1000F11D0D8F80060DAF800E0236884
:10265000F05C1EF80310814207D15A1CF9B97D2B9A
:102660001DD820202260E854A95423680BB1D0451E
:1026700009D0934813F03BFED04513D9914813F08D
:1026800036FE4FF0000923689945B4D215F80900C9
:1026900009F068F909F10109F5E7B046CDE7E8541A
:1026A0002260D4E758F8080B13F021FE092009F046
:1026B00059F9E1E72368002B41F0B082042805D1E5
:1026C0007C480FF0AEFB17B0BDE8F08F0C2841F04E
:1026D000C8827D4813F00BFE7A4813F008FE8AE7A3
:1026E00001220B4601F0ACBA591E685C2028F7D0D5
:1026F00002B123600022714EEA5406F58C783168ED
:1027000028460FF0CFFD30B908364645F7D36F485D
:1027100013F0EDFD03E04645F9D2736898470023B6
:1027200001F092BA7F2B3FF666AFA0F12002D2B241
:102730005E2A3FF660AF13B920283FF45CAF5A1C05
:102740002260E85409F00EF955E79846604F614D54
:102750003A7802F00102009255F80A3C002B41F051
:10276000FE8108F10108B8F1030F05F1CC05F3D1A2
:10277000A9E7012B05D14D280CBF0223002301F04E
:1027800004BA022B57D100233C2805F8023C4DD057
:102790003E284AD015F802ECBEF1060F41F0E08168
:1027A00015F8014C002C41F0B9814FF001094A4B5A
:1027B00005AE0FCB86E80F0015F8053C15F803AC05
:1027C0002B440A93BAF1440F0FFA8AF30995ADF836
:1027D0002C30ADF82E408DF83090ADF81C3001F063
:1027E0008D8100F20E81BAF1050F00F0518200F2E6
:1027F000C680BAF1020F00F0908100F2A880CA45AD
:1028000000F080813146504604F012FA0446002858
:1028100040F07681BAF1740F00F0C682BAF1770FFA
:1028200000F052836FF00109CCE2012305F8013C6E
:10283000032301F0AAB9032B0BD10023C0289FBFAB
:1028400005F8063C05F8050C05F8040C042301F016
:102850009CB9042B09D115F8043C05F8030C5E4023
:1028600005F8046C052301F090B9052B92D115F8F9
:10287000061C15F8053C15F8042C8B420CD94B1C92
:1028800005F8063CCC23424005F8042C134A03FB10
:1028900008230B4498727DE7824202D1062301F09F
:1028A00074B9002301F071B9902900204428002058
:1028B000482800200C2900208C29002058C5010838
:1028C000B9C70108BEC70108C3C70108CEC70108C0
:1028D0002C2B00209E0C002030AA0108940C002014
:1028E000009B002B41F03C81232824D10123019936
:1028F00055F80A2C0B708C4B8C491A608C4B8D4808
:102900001A609A609DF8002059605A7340221A7329
:10291000894A04331360894B894ADB78003318BF36
:102920000123137013F012FD864813F0E0FC4FF4FE
:10293000805013F0E3FE844B93F82230B3427FF4CF
:1029400029AF824B824A1A60824BDC6022E7BAF1DF
:10295000030F00F01B81BAF1040F7FF453AF002482
:1029600004227D49304606F0FBFF7C4B3046197847
:1029700007F014F8059B5A1C05921C70CAE0BAF1C6
:10298000240F00F0C3811FD8BAF1200F7FF43AAFB3
:10299000DFF8E0A1724B9AF80120D91C1A709AF85E
:1029A000002005915A709AF80220BAF808109A701F
:1029B000304606F0F3FF059B9AF80520591C059157
:1029C0001A709AF8062083E0BAF1280F00F0D0813F
:1029D000BAF1380F7FF416AF0522614B4FF00109B1
:1029E0005A700A2200249A705E4A83F80090117887
:1029F000DC701971517892785971D91D05919A71CD
:102A0000CCE0BAF1810F00F0858130D8BAF1540FD3
:102A100000F0C38108D8BAF1520F7FF4F3AE504BE7
:102A20005A1C05921C70B9E0BAF16E0F00F03D819E
:102A3000BAF1800F7FF4E6AE00210A264A4B4B4CD8
:102A40001B780B3BDBB299425ADA22880598FF2AA1
:102A5000A8BFFF2200F1010ECDF814E00670059822
:102A6000013100F1010ECDF814E00270EBE7BAF18C
:102A7000A00F00F03B8130D8BAF1820F7FF4C2AED4
:102A80003B4B30461A78364BDFF8F8A0591C1A70C9
:102A9000384B0591198906F081FF374B059A1B8841
:102AA000511CFF2BA8BFFF2305911370DAF8081003
:102AB000304681F3100189B206F070FFDAF8001099
:102AC000304601F30F0189B206F068FF2B4B1A78EC
:102AD000059B591C05911A7060E0BAF1B80F00F01F
:102AE0001781BAF1FE0F7FF48DAE0024DFF89890C5
:102AF00039F814103046013406F050FF042CF7D199
:102B0000002407E0164BDA1C059224221C7083F87F
:102B100001A09A704FF0010940E0042218493046A4
:102B200006F01EFF3AE000BF482800206BA5000811
:102B300028100020EEC7010844280020FC1F0020B8
:102B4000F00F0020BEC7010816370020F04F00200C
:102B5000EFBEADDE00ED00E001200020C40A002041
:102B6000603C00206C200020D4370020900F002013
:102B700032220020862B00201E220020812B0020E4
:102B8000F4C701081C210020F42000200222BD4BC4
:102B90005A70DA1C83F800A005929C70ADF81E9064
:102BA000B9F1000F66D0059B55F80A0C0693B54B9A
:102BB000059303681B6A03B19847059B069EF61AA6
:102BC00000230E9324238DF834304D238DF83530B7
:102BD000BDF91E30FF2E3246A8BFFF22013300F0A0
:102BE00090879DF82030002B14BF3C233E23FE2EFF
:102BF000CCBF4FF007094FF005098DF83630BDF80E
:102C00001C308DF837208DF838304A46C8BF331253
:102C10000DA955F80A0CC4BF8DF83A308DF839600B
:102C200007F085FC0DAB994400230DF137024A45AE
:102C300040F06A87002E8DF813300EDD324605997C
:102C400055F80A0C07F073FC059B9DF813201E44F1
:102C5000B34240F05E878DF8132055F80A0C01222C
:102C60000DF1130107F063FC55F80A0C03685B6A69
:102C700003B19847002305F8023C002C3FF471ADE6
:102C800055F80A0C07F0E2FF55F80A0CA04768E572
:102C90000B227D49304606F063FE08227B49304610
:102CA00006F05EFE07227A4939E77A4B754A1B889F
:102CB000DFF808A2FF2BA8BFFF23511C0591DAF80B
:102CC0000810137081F3100189B2304606F066FED9
:102CD000714B3046198806F061FEDAF8001001F3F6
:102CE0000F0189B2304606F059FE57E76B4B30466C
:102CF000196806F03FFE6A4B3046196806F03AFE46
:102D0000684B1968304606F035FE47E7664BF8E732
:102D1000664BF6E74FF00A0A4FF6FF7B644B654AB5
:102D20001B780B3B5FFA83F94C45BFF6E9AE11689F
:102D300093685945A8BF59460598029321EAE17165
:102D4000431C059389B280F800A03046039206F038
:102D500025FE029B30460AFB03F15945A8BF5946A0
:102D600021EAE17189B206F019FE0134039ADBE72A
:102D70000A22444BDFF848A19A70BAF800101A1DD5
:102D800083F8009083F801E083F8039030460592C1
:102D900006F004FEBAF80210A4E73A4A134603F814
:102DA000024B05935470F9E6099B0A9A9A420FBFA9
:102DB00021465A1C099219783F4A304613F064FAAA
:102DC0004FF0010919F1020F40F04783BAF1470FA4
:102DD000099B0A9A40F0868009A8A2EB030A06F034
:102DE00099FDBAF1050F814678D909A806F0A8FD2A
:102DF000099B0A9A83469A4202D009A806F0ABFDC5
:102E0000059A069BDFF8BCA09B1A103BDAF8082055
:102E10005B45CDF808B0A2EB0902B8BF1FFA83FBEF
:102E200093454946304688BF1FFA82FB06F0A2FD53
:102E30003CB95946304606F0B1FD059A511C059142
:102E40001470DAF8083009EB0B029A42059E88BF2D
:102E5000A3EB090B07F090F85A46314648460FF0AD
:102E6000DBFE059B03440593002C3FF449AE002292
:102E7000029B83427FF744AE059B0130591C0591AC
:102E80001A70F5E7603C0020F9C7010805C8010881
:102E90000EC801081E2200207C2B0020E8F7FF1F2F
:102EA000ECF7FF1FF0F7FF1FC8200020541E002082
:102EB000D4370020BC0F0020416201081C210020F3
:102EC0007020002010040020099B0A9A9A421DBF1E
:102ED0005A1C099219782146A14A6EE701244FF045
:102EE000800B8DE7BAF1290FA2EB030437D0BAF1BA
:102EF000390F20D0BAF1210F45D15A1C09921A4638
:102F0000984C12F8021B16A8099261705A78227028
:102F1000DA1C40F8342D9B78A37006F011FD099B54
:102F200020815A1C09921A4612F8021B61710992FB
:102F30005B78A37124E05A1C09921A780A2A40F09F
:102F400028869A1C09925978874A1170D91C0991D0
:102F500099785170191D0991DB78937010E05A1C13
:102F600016AC44F8342D1B7820460A2B40F0C18063
:102F700006F0E6FC7D4E3080204606F0E1FC7080D5
:102F80004FF0010969E2BAF15F0F00F0078400F227
:102F90005C81BAF1370F00F03B8570D8BAF12B0F86
:102FA00000F09D8420D8BAF1230F00F0B98206D832
:102FB000BAF10B0F00F08D854FF0FF394DE2BAF1F9
:102FC000250F00F07A84BAF1270FF5D109A806F091
:102FD000B7FC674C206009A806F0B2FC606009A845
:102FE00006F0AEFCA060CBE7BAF1310F00F03485FB
:102FF0001ED8BAF12D0F00F08284BAF12F0FDBD169
:103000005C4C04F1400609A806F09AFC099BA4F860
:1030100080005A1C09921A4612F8021B043484F8E4
:103020007E1009925B7884F87F30A642EBD1A7E747
:10303000BAF1330F00F0D984BAF1350FBCD15A1C64
:1030400009921A780E2AB7D8991C09915C78032C3A
:10305000B2D806215143484842185471DC1C0994E7
:103060009C784454191D0991D9785170197991703F
:103070005979D170D91D9B790991137180E7BAF103
:10308000480F00F016843AD8BAF13E0F00F00382E0
:1030900004D8BAF13C0F3FF473AF8DE7BAF1410F9A
:1030A00000F0AA84BAF1430F86D116AC5A1C44F83A
:1030B000342D1A78314B324E1A700023204633607B
:1030C00006F028FC33681843099B30605A1C0992AB
:1030D0001A782C4B20461A7206F032FC244E3060CF
:1030E000204606F02DFC7060204606F029FCB060FA
:1030F000204606F025FC204606F022FC40E7BAF107
:10310000510F00F0B38341D8BAF14C0F00F04D8459
:10311000BAF14E0F7FF450AF5A1C09921C78112C53
:103120003FF64AAF9A1C16A840F8342D5B78164E2D
:1031300006F8143006F004FC40F6CA039842A8BF13
:10314000184640F2EE239842B8BF18461923A0F261
:10315000EE2090FBF3F006EB4404607010E700BF34
:103160000D600108862B00206C20002070200020BC
:103170007C0C0020AC290020001F002088210020AA
:10318000C8200020542200202C190020BAF15B0F27
:1031900000F0AD82BAF15D0F7FF40EAF5A1C16AC91
:1031A00044F8342D1B78C14EDFF83493204689F85B
:1031B0000530D6F800A006F0C3FBAAF82000204690
:1031C000D6F800A006F0BCFB099A0A9BAAF81E00DC
:1031D0009B1A072B17DD204606F0B2FBA9F80A0060
:1031E000204606F0ADFBA9F80C002046D6F800A05A
:1031F00006F0A6FBAAF822002046D6F800A006F0AA
:103200009FFBAAF82400099A0A9B9B1A032B09DD4D
:10321000204606F095FBA9F80E00204606F090FB2C
:10322000A9F81000099B0A9AD21A002A05DD591C38
:10323000099132681B7882F826300DF02BFB11F0D3
:103240006FFC306810F0E6FA9AE6BAF1D40F00F09D
:10325000CB816FD8BAF1CA0F00F046813DD8BAF1E0
:10326000B70F00F0C28014D8BAF1610F7FF4A4AE9A
:103270005A1C09921A468E4912F8020B0992C8701C
:1032800059788C4A5171DA1C09929A788A4BDA7013
:1032900076E6BAF1B90F00F01B83BAF1C80F7FF4DC
:1032A0008BAEC4F34704122C3FF686AE00260DF118
:1032B0003409A642C0F2D4800023804A0DA99C4262
:1032C00040F0D58000217D4A122B40F0D6804FF08F
:1032D00001097B4B83F80090BFE0BAF1CE0F00F0FC
:1032E000BA8210D8BAF1CC0F00F03281BAF1CD0F0A
:1032F0007FF462AE3B78D9073FF542AE4FF4C87217
:10330000704B1A803CE6BAF1D00F00F09882BAF107
:10331000D20F7FF451AE5A1C0992187806065CD47D
:103320003B78DC073FF52CAE032828BF00200DF0CA
:10333000EFF925E6BAF1DC0F00F0C88126D8BAF122
:10334000D90F00F0A08114D8BAF1D60F7FF434AEB3
:1033500000245D4EDFF88C9133789C42BFF610AEAE
:1033600009A806F0EDFA13F03DFF49F824000134F6
:10337000F2E7BAF1DA0F00F09481BAF1DB0F7FF4D3
:103380001BAE4A4B4E22514918684AE0BAF1EF0F82
:1033900077D015D8BAF1DD0F00F08A83BAF1DE0FCD
:1033A0007FF40AAE09A806F0CBFA494C208209A89E
:1033B00006F0C6FA608209A806F0C2FAA082DFE52C
:1033C000BAF1F20F00F03B81BAF1FA0F7FF4F4ADDD
:1033D0003B78DB073FF5F0AD37E200F07F000328D4
:1033E00028BF002012F0FEFDCAE55A1C09921A46B9
:1033F00012F8029B0992DA1C587809929978B9F16F
:10340000000F11D101283FF6BBAD01293FF6B8AD41
:1034100081423FF4B5AD4E222E4B02FB013102FB3F
:10342000003014F0C5FDABE5B9F1010F7FF4A8AD94
:1034300001283FF6A5AD01293FF6A2AD81423FF438
:103440009FAD0C23244A584303FB01210B688418C9
:1034500083504B6863608B68A3600024FFF79EBBBA
:1034600009A806F06DFA29F81600013621E731F8AF
:10347000130022F81300013321E722F8131001335F
:1034800022E709A806F05CFA094CE08109A806F0D9
:1034900057FAA08174E55A1C09921A460F4912F88E
:1034A000020B887009925B784B7069E59C200020C4
:1034B000A6200020D22C0020B62000202E180020AC
:1034C0002C18002008230020D437002008C501084C
:1034D000B8370020922F002076200020C220002044
:1034E0006C34002024280020A04B1868034600F10B
:1034F0001E04099A0333511C0991114611F8026BFD
:1035000003F8036C0991517803F8021CD11C09914E
:10351000927803F8012CA342EBD110F0ABF82FE521
:103520005A1C0992197813293FF646AD9A1C099244
:103530000C2600225C78DFF85CE206FB02E090F8E3
:1035400008C0A44500F030830132252AF5D133E5C7
:10355000092C7FF731AD5A1C09921A46844E12F895
:10356000021B34682170099200225B78601DA370F1
:10357000022A14BF4FF0640E4FF0FF0E099B013278
:10358000591C099119787145A8BF7146032A00F8A2
:10359000011BEDD19A1C09925A7816A8642AA8BF7B
:1035A00064222272DA1C09929A78E2701A1D40F89D
:1035B000342DDB78237106F0C3F90A9B099A6081E8
:1035C000991A002904DD501C0990316812784A725A
:1035D000099A9B1A002B04DD511C0991336812785B
:1035E0005A7012F043FFCBE40D2C7FF4E5AC5A1C6B
:1035F00009921C78072C3FF6DFAC0C2609A806F0D0
:103600009FF96643DFF8909109EB0604A08009A8B2
:1036100006F096F9E08009A806F092F9099B20814E
:103620005A1C09921A4612F8021B09A8A1720992A3
:103630005B78E37206F06EF949F80600A0E45A1CC4
:1036400009921A780F2A3FF6B7AC991C09915C7859
:103650004848C2EBC20142184454D91C09919978D8
:103660005170191D0991D97891701979D1705979D2
:1036700011719979517103F10801DB790991937105
:103680000AF06CFF7CE409A806F05AF93A4C208055
:1036900009A806F055F9608009A806F051F9A08044
:1036A0006EE419465A1C099211F8020B334A09912B
:1036B00059781070517016A8D91C40F8341D9B78A9
:1036C000937006F03DF92C4BD88059E45A1C0992AE
:1036D0001A4612F8020B2A4909920870294A5978A9
:1036E0009170DA1C09929A78274B9A7048E45A1C18
:1036F00009921A46224C12F8021B244E0992A1701C
:103700005978234A0DF158091170DA1C09929A78F8
:1037100032711A1D49F8342DDB784846042BA8BFB6
:103720000423B37006F00CF9099A0A9B30809B1AA7
:10373000012B03DD484606F003F9F081099B0A9A44
:103740009A4206D05A1C09921B78003318BF0123F5
:10375000E3710DF09FF8099B0A9A9A423FF410AC6E
:103760005A1C09921B78F3700AE400BF9C200020C9
:103770003C3C0020C6190020343C0020A020002042
:103780006C340020A6200020B6200020B83700208E
:1037900074200020B4AD0108381A002009A806F0F2
:1037A000CFF809A806F0CCF809A806F0C9F809A8CE
:1037B00006F0D1F8099BB24C591C099119462268B0
:1037C00011F8020B82F82C000991597809A882F8A7
:1037D0003610D91C09919B7882F8373006F0BBF877
:1037E00009A806F0B8F809A806F0B5F809A82668EF
:1037F00006F0A6F8708709A8266806F0A1F8099BCC
:103800000A9A3087D21A012A08DD591C09912268C8
:103810001B7809A882F82E3006F09DF8099A0A9BB9
:103820009B1A032B09DD09A8266806F089F8708623
:1038300009A8266806F084F8B08620686DE63B7813
:10384000D8073FF59DAB0DF097FA0CF077FF0DF020
:10385000B3F8FFF795BB3B78DA073FF591AB894AA0
:10386000137843F004031370FFF78ABB8649097885
:1038700001293FF685AB591C09911946834C11F873
:10388000020BA070D81C0991121A5978012A0990CC
:103890009E7805DD09A806F053F82080FFF770BB7D
:1038A0007B4BB3F900304B4393FBF6F32380FFF7D8
:1038B00067BB0FF093F9FFF763BB0023754C09A8B2
:1038C000236006F027F8236818432060FFF758BBF1
:1038D0000023714C09A8236006F01CF8F5E7581C7A
:1038E00009901C786D49121A002A0C707FF748ABBA
:1038F0009A1C09925B78003318BF0123D4E55A1C47
:1039000016AC44F8342D1B78654E2046337206F011
:1039100017F8B083204606F013F83083204606F0EF
:103920000FF8099B70835A1C09921B78F3740A9B49
:103930009B1A032B07DD204606F002F8B0842046D0
:1039400005F0FEFFF084099B0A9AD21A032A0DDDC6
:103950005A1C09921A4612F8021B2046B1770992A6
:103960005B7886F8203005F0EBFF7084099B0A9A9B
:10397000D21A052A0CDD5A1C09921B782046F372D4
:1039800005F0C8FF099BF0605A1C09921B7833743C
:10399000099B0A9AD21A002A7FF7F2AA5A1C0992A6
:1039A0001B7886F82130FFF7EBBA5A1C09921A46A9
:1039B0003C4C12F8021B16AE46F8342D21715B7890
:1039C0003046637105F0BCFF099B20805A1C0992A8
:1039D0001B783046A37105F0B3FF099B60805A1C29
:1039E00009921B78E371FFF7CBBA5A1C09921A7837
:1039F0002B4B5A75FFF7C4BA00232949099A501C6A
:103A0000099012785A540133082BF7D1FFF7B8BA4E
:103A10000726B4FBF6F6C6EBC603E41A7FF4CCAA7D
:103A2000DFF888B0F6B2E3B2B3423FF4A9AA4FF090
:103A3000000A099B5A1C099293F900300BEBCA0942
:103A400099F902209A4200F0CA800AF1010ABAF1FB
:103A5000040FF3D1FFF7B0BA5A1C09921E781F2E3B
:103A60003FF6AAAA052C7FF4A7AA09A805F052FFE1
:103A70000D4B43F8260010F04BFCFFF781BA00BF56
:103A80009C20002049150020A6370020D0330020BC
:103A900094370020C8200020541E002088210020D8
:103AA00054220020982E0020AC2900201637002038
:103AB0005A1C09921A4612F8020B0992DA1C59781C
:103AC00009929A780FF064FD00287FF459AAFFF755
:103AD00073BA002111226A4816F09BFE102C4FF099
:103AE000000328BF10246649A342BFF449AA099ADB
:103AF000501C099012785A540133F5E7614CFFF7D6
:103B00004DB82123FFF773B812F8011B4B40FFF7A4
:103B10008EB813F8011B4A40FFF79AB8012C1BD14D
:103B2000102200210DA816F074FE15F8053C0D9525
:103B30002B440E9315F8033C6E2BADF83C300BD1A3
:103B40000DA805F008FF0DA805F0FAFE0DA805F078
:103B5000F7FE0DA805F0F4FE0024FFF78BB84A4CE1
:103B600055F80A0C06F0DDFC00283EF4FAAD55F8D5
:103B70000A0C06F0D3FC15F8023C0646002B7EF436
:103B8000F8AD24287EF4ACAE012305F8023CFEF724
:103B900001BE09A805F0DFFE09A805F0DCFE09A8B2
:103BA00005F0D9FEFFF7ECB9384A007802F8210099
:103BB000D81C0990987802EB81011A1D487009926F
:103BC000DA7800208A705A1D1B790992CB7012F0A6
:103BD000C3FB2F4B80F001001870FFF7D1B989F8B3
:103BE000023009A805F0ACFE099B2BF83A005A1CDC
:103BF00009921A4612F8021B0134099289F803103F
:103C00005A7889F80420DA1C09929A7889F80620F3
:103C10001A1D0992DB7889F8053004E70C283EF478
:103C200058AD0A2801D00D2820D112F079FB2321AC
:103C3000284616F023FE08B1401B206000222368AE
:103C4000002B7EF451AD02B1236080220021284672
:103C500016F0DFFD019B1B78002B7EF43DADFEF7D7
:103C600032BD7F287EF461ADFEF7C5BC7F287EF4AF
:103C700059AD0022013B2360EA540648FEF72DBDF2
:103C8000102000205F0601080400FA05601E0020D5
:103C900000000020EAC701082DE9F04FB24B9DB0AB
:103CA0001B780790012B07D1B049B14A0968C9694F
:103CB0001180B04909885180AF4D2A78002A00F060
:103CC000F084072B40F0FE8106F05EFB0890AB4FBE
:103CD0003B68069713F4806F05D0A948836813B139
:103CE00000F150019847A74BA7491B68B1F906405E
:103CF0005A890991944280F2E8814FF07E536B60BB
:103D0000A24B4FF0000893F90410A14A002914BFF8
:103D100001214FF0FF31168B93F801A093F800902A
:103D20009C4F05910A92099B33F918B0ABEB060042
:103D30000028B8BF4042B0F5FA7FA8BF4FF4FA7030
:103D4000B8F1020F00F0D4814845CCBFA0EB0900C8
:103D5000002013F04BFAB34547F82800C0F2D68193
:103D600008F10108B8F1030FDDD1069B1F6817F4B5
:103D7000805800F0D281B4F5FA6F2346A8BF4FF403
:103D8000FA63B3F57A7FB8BF4FF47A73A3F57A7309
:103D90002A7A22B16A7A5343642293FBF2F34FF0FA
:103DA000640E93FBFEF27C4802F1010C30F9121014
:103DB00030F91C006FF0630C0CFB0233401A5843BF
:103DC00090FBFEF0084400B213F010FADFF8C49143
:103DD0008246C9F80C00B8F1000F1DD01D2012F06A
:103DE000F5FAC8B16D4BDB78B3B96D49504613F0A5
:103DF00047F913F02BFC4FF47A7300B2000390FBE9
:103E0000F3F3C6F5FA6000B2584340F30F30304484
:103E100013F0ECF9C9F80C00624B1E8873063BD511
:103E2000614BB3F904000A2390FBF3F02B8AC01A0C
:103E300000B213F0DBF95D4913F02CFA5C4905463A
:103E400013F020F905F0CBFE8346284605F0C7FEA7
:103E5000504D81462B6859461846069313F01AFABE
:103E6000D5F804A005905146484613F013FA059A78
:103E70000146104613F004F959462860504613F0E5
:103E800009FA069B82461946484613F003FA014692
:103E9000504613F0F7F86860464B374D1B6813F037
:103EA000140F1AD016F4027F17D0434BDFF8E490BA
:103EB0001A7812F0100200F04581AB7C6869002B83
:103EC0000CBF01234FF0FF33584313F08FF9D9F89B
:103ED000041013F0D7F8C9F80400384BDFF8B0909D
:103EE0001A780693A2B1B9F81A30A34210DB344B0A
:103EF0001B78012B01D0192B02D1324A927B3AB99F
:103F00000E2B05D0082B1FBF0023224AEB639360C2
:103F100095F84240002C68D0B60766D02A4B2B4952
:103F20001E6A304613F05EFB002840F05E8130468A
:103F300014F01CFA696C13F0ADF914F09FF9B0F5A8
:103F4000617FA8BF4FF4617013F050F9204913F05E
:103F5000A1F905F044FE0646204613F047F9314624
:103F600013F098F936E000BF80210020F0220020F5
:103F7000F42000202C1C00207C1000208C2100202C
:103F8000803400203C3C0020542B0020A020002046
:103F90005422002034220020403C0020982B002096
:103FA00000007A447E2B00206C2E002035FA8E3CD7
:103FB000DB0FC93F842100204915002000000020AC
:103FC00088210020B41A00202C2E00208FC2753CBE
:103FD000D06D393A14F052F900B213F007F9884C59
:103FE0000146E06813F04EF8E06095F84860002E56
:103FF0005AD0844B0420D3F8EC4044F620639C4212
:10400000A8BF1C46B4F57A7FB8BF4FF47A74A4B247
:10401000A5F84A4012F0DAF908B9F80044D54FF48F
:104020007A73B4FBF3F4642393FBF4F4DFF8E8A1B0
:10403000142CA8BF1424DAF80030B8F1000F00F0F7
:10404000D6805F8E7F086E49EA6CD1F80C80531CD5
:10405000EB64404605EB420B059313F0F7FA059B22
:10406000ABF85000A342A4BF0023EB64EB6C05EB5C
:104070004303B3F9500013F0B9F80146404612F07B
:10408000FFFF13F0E3FA00B20028B8BF4042B84285
:1040900040F3B080DAF80030988E13F0A7F85A4950
:1040A00013F0F8F8069B586099F81E30002B00F0CA
:1040B000D781022B00F0B280032B00F0A581534B77
:1040C0005888B0E00023089301E6B4F5FA6F187A37
:1040D000BFBFA31A5843C2F5FA6290FBF2F0C0F1D9
:1040E000640013F083F84A4913F0D4F8686007E6D7
:1040F0005045D8BF0020059BC8BFA0EB0A0058431D
:1041000013F074F8B345B860BFF62FAE57F8281017
:1041100001F1004147F8281022E60A9B5A8B94428D
:104120000EDBB4F5FA6F2346A8BF4FF4FA634FF4E1
:104130007A719B1A4B43C2F5FA62B3FBF2F327E69E
:104140001346F4E7334BD978987871B3B5F9183042
:10415000E11A0029B8BF4942814210DDEA6101221B
:104160009C4285F82020C8BF404213F03FF801462A
:10417000D9F80C0012F086FFC9F80C00ADE695F8EE
:10418000201019B1A96A85F820206962686918446D
:10419000B0F5FA6FA8BF4FF4FA60B0F57A7FB8BFF8
:1041A0004FF47A7013F022F8E6E7B5F91820A31A55
:1041B00083EAE37EAEEBE37E86450BDD022193FBD3
:1041C000F1F3EB62012385F8303085F8203068691F
:1041D0001044DDE795F82030002BF8D0AB6A85F865
:1041E00030106B6285F82010F1E70020F4E6B3F997
:1041F000327028E74FF07E53069A536054E700BFB1
:1042000034220020FC0000206F12833A1C1800208A
:104210000AD7233CA02000209C200020B5F84A00AB
:1042200000F57A7080B299F81F400234E4B2002E93
:1042300000F0FF80002800F0FC808D4B00261B68FA
:104240008C4FB0FBF3F000B2A5F8780012F0CEFF6F
:1042500001464FF07E5013F0D1F88046DFF81C92F3
:1042600007F1100AA642C0F2D780834B1B78092BB6
:1042700011D1824B824E186814F000F8814B3080C7
:10428000D3F8EC004FF47A7390FBF3F012F0AEFF2A
:1042900013F0DCF97080B5F97830002B40F3E28040
:1042A00000273E46DFF81082DFF8D0A1A8F1100900
:1042B000A742C0F2C48095F848300024002B18BFF4
:1042C0000226714BDFF8F491D3F800806A4B1B781B
:1042D000099308F105030A93B44240F3F180099B66
:1042E0006A4C092B07D1664EB4F87830606BB38006
:1042F00013F0ACF9F080664B93F82160002E60D08B
:104300001E2012F063F800285BD0624B1B88590610
:1043100057D494F8B430B34214D084F8B460304623
:1043200012F064FF5C4912F0B5FF5C49064612F0DA
:10433000A9FE05F054FC5A4B9860304605F04FFC3E
:10434000C4F8B800069B6E6BD3F808903046494617
:1043500012F0A0FFD5F83C80D5F8B87082463946F7
:10436000404612F097FF0146504612F089FE4D4933
:10437000824613F037F908B9DFF828A14A495046B8
:1043800013F03AF908B9DFF820A149464046C5F8CC
:1043900034A012F07FFF39468046304612F07AFF93
:1043A0000146404612F06EFE3E49064613F01AF9E9
:1043B00000B93C4E3C49304613F01EF900B93A4E64
:1043C000EE63002384F84830384B1B78002B40F014
:1043D0005B81374EB278002A00F05681354C237845
:1043E000013B0D2B00F23E81DFE813F010012301A9
:1043F0002D0116023C013C013002440256027202B9
:104400008302A002AA02B30299F82000C0EB401375
:1044100000EB8300C00005E75AF8261059F8260083
:1044200012F02EFE414612F035FF47F82600013605
:1044300018E7B5F87830013BA5F878302BE758F845
:10444000270059F8271012F01DFE022F3E46B8BF74
:10445000022648F827004AF82700F6B2013727E776
:10446000A5F8783095F84830002BADD0002622E72B
:1044700068210020F8100020802100203422002034
:10448000F4200020FC0000203C3C00207C10002098
:10449000542200207E2B002035FA8E3CDB0FC93FD2
:1044A0000000002000C0F94400C0F9C49029002099
:1044B000D0330020A6370020081100200AD7233C63
:1044C000022C15BF98F8000098F8010098F802B087
:1044D00098F809B012F08AFE494612F0DBFE4FF060
:1044E0008041074613F092F860B14FF080413846A2
:1044F00012F0C6FDA34912F0CDFE0146384612F077
:10450000C1FD0746A30005939F4BA04953F8240023
:1045100012F0C0FE20F000439D4A0593059B42F82F
:1045200024000C32824642F82430BBF1000F20D028
:10453000584612F05BFE494612F0ACFE83465146E7
:10454000504612F0A7FE059912F0A4FE594612F04B
:10455000A1FE59460B904FF07E5012F091FD0B9A40
:104560000146104612F08EFD0146504612F092FEB2
:1045700082468849384612F08DFE514612F08AFE76
:104580000A9B074613F8010B0A9300B312F02EFEA4
:10459000494612F07FFE059912F07CFE7E49824664
:1045A00013F034F868BB0021504613F011F850BBEB
:1045B00051464FF07E5012F063FD01464FF07E50A1
:1045C00012F01CFF0146384612F064FE0746099BB4
:1045D0000C2B05D1384613F039F8704B23F8140032
:1045E0006F49384612F0FEFF00B96D4F6D493846ED
:1045F00013F002F800B96B4F6B4BA200D750013497
:104600006AE64946DAE74FF07E51D7E7674B1B78F9
:10461000DA0707D5802010F0CBFB08B106F052FB7B
:1046200013F04CFB1F2011F0D1FED8B10C232370E6
:1046300018E000225E4B1A605E4B1A605E4A1268F8
:104640005A600323F3E710F00DF85A4D5A4B1A68DD
:104650006B686433934205D240200FF0DBFF0028E3
:1046600000F0B68010F026F8002800F07981237859
:104670000C3B022B08D901232370504B93F8BC202C
:1046800012B1002283F8BC204D4B1B78072B05D1BB
:1046900005F07AFE089BC01A404B98800022474BD9
:1046A0001A70474F3B78072B40F0A68105F06CFE4F
:1046B0000890444C636820469847A246002849D099
:1046C0000026B4F8B45084F85560DFF80081002D5E
:1046D00040F0FC81626AB4F93C3094F856109B1AA1
:1046E0002363A26AB4F93E3004F130009B1A63637D
:1046F000E26AB4F940309B1AA36308F09BFB324B8B
:104700001B78002B40F07B811D4604F12C0656F8E7
:10471000040F12F06BFDDAF8201012F0BBFD05F566
:104720009C720146DAF834310AEB0200984705F52D
:10473000D4720146DAF8A4310AEB02009847DAF89D
:10474000B8300146D6F8F800984724356C2D48F863
:10475000040FDCD11A4C2278072A05D105F014FE8B
:10476000089BC01A0D4B1880144B93F8C5201D46AA
:104770000692002A00F07E82013A83F8C5201DB01F
:10478000BDE8F08FD7A36841342200206F12033BAD
:104790001811002000004843A4707D3FF420002041
:1047A00000C0F94400C0F9C4B01000202C2B002038
:1047B000CC33002008200020982200207C1000200C
:1047C0008021002080340020E015002004370020E4
:1047D000DFF8EC824027C246DFF8E8922B6818F831
:1047E000030068B10FF0E4FFD9F80030013F03F196
:1047F000FF33C9F800302B6803F101032B60EDD1C2
:104800002B681AF80330002B7FF42CAF2B604FF08D
:10481000FF336B6004230AE70FF024FF984A50210E
:10482000A2F10C0301932623029200934920A2F1E6
:104830000A03163A0BF0A8F800287FF413AF4FF0E4
:10484000FF32904B18605A600723F0E60FF00AFF22
:104850000523002100938C4B02910191A3F10802E2
:1048600053200BF091F800287FF4FCAE854B1860C4
:104870000823DCE60FF0F6FE0AF02AFD00283FF4DC
:10488000F1AE13F05BFB00283FF4ECAE7F4B1A68EF
:104890007F4B1A600A23CAE61A2011F097FDA0B1D7
:1048A0007C4B1B888BB97C4B14A91B680E2014937E
:1048B000079B159310F076FC744B1A68744B1A60C2
:1048C0000A232370079810F0B9FC10F047FCC9E6E2
:1048D000724B1B78002BF5D01A2011F077FD0028C1
:1048E000F0D16F4B93F8BC30002BEBD10923237030
:1048F000EBE76C4B1A68634B5B68C833934210D28A
:10490000B378032B0BD1684D286806F0C5F9002356
:104910002B60664B1B78022B01D106F0C1FB0123F3
:1049200085E613F00BFB0028EAD19BE6012A01D1B2
:104930000EF054F90D231320237006F029FC91E6A4
:10494000012A04D10EF066F800283FF48BAE0E2346
:10495000F1E71F2011F03AFD00287FF483AEDEE777
:10496000F378002B3FF490AE514B1D7815F0010504
:1049700008D1504BDFF850911F784F4BD3F800808F
:10498000BD4219DB474B464D1B68D5F8C0209A4203
:1049900023D92378012B7FF477AE414C94F8BC20C7
:1049A000002A7FF471AEB378032B0FD013F086F991
:1049B000012384F8BC3067E6414659F8250012F01F
:1049C000FDFD002801F093820135D9E7802010F029
:1049D000EFF900287FF458AEE8E72378012B3FF485
:1049E00053AE95F8BC30002B3FF44EAE0BF006F9F9
:1049F000002385F8BC3047E60023089359E62F4E84
:104A000004F12C0944460AF59C7897F800B059F84F
:104A1000040FBBF1170F02BF05EB0A039B8F338016
:104A200012F0E4FBDAF8201012F034FCBBF1080FAE
:104A3000014604D1059013F021FC05993080DAF885
:104A4000343140469847DAF8A431014608F1700045
:104A500098473B788346032B02D113F00FFC30803C
:104A6000DAF8B8305946D9F8F80098470235062DDB
:104A700044F8040F08F1240806F10206C5D169E6DE
:104A8000A6AA01080820002060AC01080822002026
:104A900098370020A03700209C370020902100206C
:104AA0007C10002098220020D833002064210020B0
:104AB0002C2B0020D437002094290020F420002043
:104AC00040AA0108CC33002024280020614BD8F8EC
:104AD00000205B78069609934FF47A73B3FBF2F3E8
:104AE000C3EB431203EB8203DB009BB205933B78DD
:104AF00004F124070A93584BB3F90690059B5B0811
:104B00000B93059B9D4201BF0023BB64C4F8883012
:104B10003B60524BF318B3F93C00BB6C0344BB64DD
:104B200012F064FBD4F8882002F10108B8F1010FFB
:104B3000C4F8888008D10023012DE067A067C4F87D
:104B400080305FD1002033E0D4F878A00D92514638
:104B50000C9012F095FA8346404612F047FB01464E
:104B6000584612F04BFC514612F08CFA0C9B014651
:104B70008246E067184612F083FA594612F08AFB23
:104B8000D4F8801012F07EFA012D8346C4F8840018
:104B9000C4F878A0C4F880000D9A33D1B8F1010FA1
:104BA000D0DD104612F022FB0146584612F026FCDA
:104BB00013F024FE0A9B8046032B05D113F05EFB05
:104BC00001230FFA80F90693099BA3B1184612F04E
:104BD0000DFB414612F0FCFC68B1069B13B11E4B65
:104BE000A3F806901E4808F015F900221D4B5A60E4
:104BF0009A60DA60AEE50B9ABB6C1344059A93FB9E
:104C0000F2F33B600236062E07F1040704F11404A8
:104C10007FF477AF069B13B10F4BA3F80690012DDD
:104C200011D10022104B1B689A621A63DA620F4B93
:104C300093F8C43023B10E4B1B8823F4006313B9DF
:104C4000012006F0A5FA054AB2F8B430013BA2F8FB
:104C5000B430CAE76C340020F420002080340020F7
:104C60003435002004370020F02200207C10002082
:104C7000BC2B0020AD4B5B79002B00F07585AC4B55
:104C80001B78013BDBB285F8C5302378072B40F059
:104C90006E8505F079FB0C90A64B4FF07E501B689B
:104CA00009936B680F93D5F8C83019460B9312F02F
:104CB000E7F9A14B196812F0EDFA4FF07E510D9013
:104CC00012F090FC10B94FF07E530D939B4B0025D2
:104CD00008939B4B9B4C0A9300230593059BDFF89D
:104CE000C0929E0059F82380059A974B294653F8A5
:104CF0002270384612F062FCF0B9059B09F1980960
:104D000059F823904046494612F0BAF9824620F0FD
:104D10000041384612F05CFC58B12946504612F06A
:104D200075FC002800F027854946384612F0AAF99C
:104D30008046864B46F80380854BB3F8009019F007
:104D4000030F3BD0059B022B38D0099B93F82EB064
:104D5000584612F04BFA7F4BF15812F09BFA8246FC
:104D6000CBF1000012F042FA07460146504612F01D
:104D70002FFC40B9584612F035FA5146074612F05A
:104D800031FC00B95746059A734B33F912000A9B60
:104D9000B3F90030C01A12F029FA704912F07AFA09
:104DA0000146384612F06CF919F0010F0E9000F030
:104DB000E8846B4B196812F06DFA8046694B4046E7
:104DC0003344D3F804A0514612F05AF994F8D8307D
:104DD0000746002B00F08580079AD4F8DC30D31A00
:104DE000614A126893427CDD099B93F84830022B9C
:104DF00002D1012005F024FC059B022B40F09E858A
:104E00005A49504612F002FC002840F0B785584934
:104E1000504612F0DDFB002840F0B085554B384677
:104E2000D3F8009009F1004B594612F0D1FB00284D
:104E300040F0A7854946384612F0D4FB00B94F46EA
:104E4000089B079A1D60D4F8DC30D31A4A4A1268CE
:104E5000934223DC4FF07E510B9812F0B9FB0028EF
:104E60003FD0464BDFF8FCB0D3F80090DBF80400ED
:104E7000494620F0004012F0ABFB90B3DBF808107D
:104E8000484621F0004112F0C1FB50B3DBF80C1092
:104E9000484621F0004112F0B9FB10B3384B1868B6
:104EA00010F0020019D0374B2B4837491A68B1F976
:104EB0000CE0B0F90030A3EB0E03002BB8BF5B424F
:104EC00093420EDAB0F90230B1F90E105B1A002BE2
:104ED000B8BF5B429A4204DD002084F8D80005F098
:104EE000AFFB2A4B0F98F15812F0D4F9394612F063
:104EF000D1F9059BDFF8AC90022B014646F809007A
:104F000006D1234A234B10681B689847C9F808004C
:104F1000089B1B680E93204B5968204B186812F0B1
:104F2000B9F90D9912F0B6F93EE000BF6C340020DB
:104F3000742000209C200020302D0020DC20002048
:104F4000B22000207C100020242D002048110020D9
:104F50007E2B0020181100206C2E0020CDCCCC3DE3
:104F60000C2D002004370020382D002000C0F8440C
:104F700000C0F8C4502D0020342D0020402D00200A
:104F8000842100203C2D0020A6200020E02C0020C1
:104F9000042E0020602D002000000020981A002020
:104FA000B0100020D0200020A34BF15812F072F96D
:104FB000394612F06FF90E9912F064F89F4B109079
:104FC000D3F800B00BF10049494612F001FB38B9A3
:104FD000109A59461046914612F004FB00B9D94682
:104FE000059B022B40F0D08494F8E030012B02D0D6
:104FF000192B40F0C9844FF00103914938461093B2
:1050000012F004FB109B00B90346DBB23BB10E9BD0
:1050100029F0004023F0004112F0DAFA10B1089BA9
:10502000C3F80090059B022B00F09380854A864BC5
:1050300051461B68B0589847844A854B01461B6807
:10504000B0589847099B814693F83730002B00F001
:10505000A684804B1B88002B40F0A1847E4BF15826
:105060007E4B186812F016F94FF07E51824612F00E
:10507000B9FA08B94FF07E5A794B5046196812F0C8
:1050800009F90146404612F005F9494611F0F8FFCA
:10509000744B8146F15811F0F3FF734B196812F00D
:1050A000ADF9704B804646F80390099B93F8483061
:1050B000002B44D06D4B1B78D80740D54FF07E5164
:1050C0000B9812F099FAF8B194F8D830E3B9684B1C
:1050D00028F00040196812F099FAA8B1654B27F042
:1050E0000040196812F092FA70B1634BF058634BAC
:1050F00020F00040196812F06BFA28B1012384F8FF
:10510000D830079BC4F8DC30079AD4F8DC30D31AC7
:105110005B4A1268934212DA564B27F00040196836
:1051200012F056FA40B9544BF058544B20F000405E
:10513000196812F06BFA10B1002384F8D830514B83
:105140000F98F15812F0A6F8414612F0A3F84E4B12
:10515000985194F8EC302BB94C4BF550089B1D60DE
:10516000494BF550059B01330593089B0433089385
:105170000A9B02330A93059B032B7FF4AFAD444E89
:105180003278072A05D105F0FFF80C9BC01A414B75
:1051900058803378012B40F0058405F0F5F83E493E
:1051A000D4F8F0303B4A0968C31A93805B1A079021
:1051B000D380C4F8F000394B394E1B6893F82C703B
:1051C000384B1B6813F4805F00F04C84274BB4F815
:1051D000F6801B784046D90758BF334BF6685CBF52
:1051E0001B8BA4F8F43012F001F8814601463046DA
:1051F00012F0F8F9002800F0DF832C4BD4F8FC10F3
:105200001868C4F80011C4F80411C4F8F80011F0CB
:1052100037FFFF23C4F8080184F80C31304612F040
:105220003BFA3146A4F8F400484611F029FFC4F8CF
:105230001001D4F814513BE0EC2C0020542D002038
:1052400000009642642D0020582D0020B42D00202F
:105250005C2D00207E2B002024110020082D002032
:10526000042D002060110020981A00202C2B002013
:10527000482D0020442D0020B01000204C2D00208F
:10528000382D0020F82C0020E8200020D02000201D
:1052900080210020F4200020682100209C20002094
:1052A000342200208C21002054220020D0370020FE
:1052B0002946D4F8100112F0A1F84FF07E510546AE
:1052C00012F090F908B94FF07E550021284612F0EF
:1052D00093F900B90025DFF8E492DFF8DCA2C4F806
:1052E0001051DAF80010D9F8000011F0CBFEAF4BE6
:1052F000196811F0C7FEAE49099011F0CBFFAD4B14
:1053000080461C6804F10046314612F061F900281D
:1053100040F0C6832146404612F064F900B9A04629
:10532000DAF80410D9F8040011F0ACFE9F4B59686C
:1053300011F0A8FE9E490A9011F0ACFF814601468B
:10534000304612F063F930B949462046264612F03D
:1053500049F900B94E46984B9968984B986811F0F6
:1053600091FE93490B9011F095FF954B8246D3F82F
:10537000009009F10044214612F02AF930B949465B
:105380005046544612F02EF900B94C468D4B5B78CE
:105390000BB904F100442FB38B4B5A7912B38B4AEB
:1053A0001778FFB1187811F01DFF8146384611F0CB
:1053B0001DFF0146484611F06DFF854B07461888D2
:1053C00011F010FF0146384612F018F881490746DF
:1053D00012F008F900B97F4F4FF07E51384612F0B5
:1053E0000BF908B94FF07E574FF0000A7A4BD346BD
:1053F0001B78DFF8249208930023089A9342C0F2A6
:1054000051835146584611F03BFE744C4FF07E518B
:10541000C4F8C800064612F0F9F8002800F08283AC
:1054200031464FF07E5011F0E9FF0025074614AEDB
:10543000089BAB4200F36D8310F0CEFF18B14FF024
:105440007C53C4F8103194F90C0111F0CFFED4F85C
:1054500010310C900D93D4F80831D4F8F8000E9365
:10546000D4F8043100250F935D4BDB78119312F0D3
:10547000EDF88146D4F8000112F0E8F8594B824665
:10548000D3F800B0584612F0E1F88046564B1E683B
:1054900006F010031293554B06F480561C78544BBB
:1054A00004F00104B3F90670524B5B8B1093089B18
:1054B0009D42C0F05B832CB94F4B504A0899A142E2
:1054C00000F39283454BD3F8A821002A00F0AF8463
:1054D00093F8E030192B00F2D38001229A40484B18
:1054E0001340002B00F0CC80464B424C1B8813F439
:1054F000807F00F09183444D286812F0A7F8ADF842
:105500005000686812F0A2F8ADF85200A86812F0D6
:105510009DF8ADF854004FF47A724FF461613B4846
:10552000B0F9023003F5E163534393FBF1F3A3F5C4
:10553000FA73ADF86830B0F9003003F5E1635A430F
:1055400092FBF1F22C4BA2F5FA7231491868ADF8D2
:105550006A2011F095FD12F079F8254A238B118805
:10556000ADF85600C91AADF858105188C91AADF8EF
:105570005A109188C91AADF85C10D188C91AADF8D3
:105580005E101189C91AADF860105189C91AADF8B9
:1055900062109189D289C91AD31AADF866300023F6
:1055A000ADF8641019461B4A38E000BFE82000201F
:1055B0006F12833A9C1A0020DC200020D0200020AB
:1055C000A01A002088210020862B002032220020F3
:1055D0001E220020713DAA3FD43700207C100020FD
:1055E000982B0020942900208C2100202C2B0020B7
:1055F000542B002054220020FC20002024280020CE
:10560000324130037E2B0020342200206C2E0020FB
:105610000080BB4454210020A411002022F8131064
:105620000133082BFAD14FF00C096427AF4BB04C73
:105630001B78B04DC3EBC3032344DFF8C482DFF80B
:10564000C4A20A930A9BA34240F0088300254FF0AE
:105650000C096427A84EDFF8A88209FB0583B6F978
:10566000024093F90A00444394FBF7F4E8B27480D3
:1056700008F09CFF01352044082D26F8020FECD1DC
:105680009E4C9F4D236813F0200F30D0002008F06F
:105690008DFF9C4E80463080012008F087FF074632
:1056A0007080082010F092FE08B3974B95F90A100D
:1056B00093F8CE31012B954B40F04283484295F947
:1056C0001620B3F90210B3F900304143534332209E
:1056D0006FF0310291FBF0F193FBF2F293FBF0F0EB
:1056E0000A44A8EB02023280084438447080DFF894
:1056F000089200234A46EE18B6F90410B2F90200E7
:10570000B6F90660884203DB86423146A8BF0146EF
:105710000C33602B22F8021FEDD17D4EB389002B94
:1057200040F01E83784F97F8E030013B182B00F2D1
:105730004783DFE813F0370345034503A903450317
:1057400045034503960345034503450345034503C8
:10575000B50345034503450345034503A903C603B4
:1057600045034503B50337030123FFF78CBA002334
:105770000C93FFF791BA3946484611F081FCFFF7C8
:10578000D7BAD4F8A890D4F8AC704946384611F08E
:1057900033FF00B94F465D4BB3F90000B3F9023057
:1057A0000028B8BF4042002BB8BF5B429842B8BF48
:1057B000184611F01BFD574911F06CFD564B8246FF
:1057C0001B78002B57D0554B2946D3F800B05846CC
:1057D00011F01CFF002800F08780514B2946D3F8B8
:1057E0000090484611F012FF00287DD007F10040DC
:1057F0004C4911F04FFD594611F000FE4FF07E511B
:1058000011F040FC51460746484611F039FC494624
:1058100011F0F4FD4FF07E51814611F0E3FE08B91E
:105820004FF07E592946484611F0E6FE00B9A946D8
:105830003946484611F02EFD81463B4B0E981968BB
:1058400011F028FD4FF07E510746484611F0CAFE80
:1058500008B94FF07E592946484611F0CDFE00B9EF
:10586000A9464946384611F015FD0146404611F05B
:1058700009FCFFF7A2BA2D4B2D49D3F800904846FA
:1058800011F0A6FE60B349464FF07E5011F0F8FBD0
:10589000284911F0FFFC51468346274811F0F0FBE0
:1058A0000146584611F0F6FC494611F0EBFB1B4B44
:1058B000196811F0EFFC81462946484611F092FE26
:1058C00090B94946174811F099FD07F10047014684
:1058D000384611F0DFFC4FF07E5111F0D3FBABE7FF
:1058E0000E4BD3F80090E7E7A946A6E7551900202C
:1058F000561900202A120020522100208C2100205D
:10590000381A0020542100207C1000206C2E00202A
:10591000B41A0020CDCCCC3D182D0020142D002031
:105920001C2D00200000C842102D0020202D00203A
:10593000AE47813F610BB63B00003443AD4B1B6863
:105940009B077FF57DAA0A9B059AB3F90000AA4B35
:1059500033F91230C01A11F049FCA84B0746A84988
:10596000186811F097FC0146384611F093FC514637
:10597000804611F085FB0746FFF762BA2F46FFF716
:105980005FBA5F46FFF75CBA4FF001034FF07E51FC
:10599000D4F8C800109311F02FFEFFF733BB29464F
:1059A000FFF770BB072B03D104F0EEFC079002E475
:1059B00000230793FFF7FFBBB4F8180111F016FCA2
:1059C00081460146304611F017FEF0B18D4BD4F8F8
:1059D0001C111868C4F8F810C4F80411C4F80001C8
:1059E00011F04EFB0123C4F8080184F80C31304655
:1059F00011F052FE4946A4F8F400304611F040FB85
:105A0000C4F81001D4F8205152E4B4F8F4304345FE
:105A100014D87D4BD4F8FC101868C4F80011C4F8F1
:105A2000F800C4F8041111F02BFBFF23C4F808019F
:105A300084F80C31C4F81051FFF7FBBB714BD4F85C
:105A40001C111868C4F8F810C4F80001C4F8041157
:105A500011F016FB0123C4F8080184F80C31C4F8D6
:105A60001051CFE7694B588B11F0C0FB0146F0682D
:105A700011F006FB644BC4F810011968614BC4F8BF
:105A8000F8101868C4F80411C4F8000111F0F8FA0D
:105A90000123D4F82451C4F8080184F80C3107E438
:105AA000B0463DE4D9F8041040460D9311F0F2FBE6
:105AB000D9F808100C90304611F0ECFB0C9A014616
:105AC000104611F0DFFAD9F80C100C90204611F0B6
:105AD000E1FB0C9A0146104611F0D4FA394611F058
:105AE000D9FB59460C9011F091FD0C9A0D9B70B9A1
:105AF0001146504611F076FD0C9A0D9B00B9924666
:105B000014A941F8232009F11009013375E49346E3
:105B1000F6E756F82500394611F0BCFB46F825009B
:105B2000013585E410F058FC38B94FF07C51284617
:105B300011F06CFD00283FF486AC4FF07C513046EC
:105B400011F0A8FB06460146284611F041FD50B968
:105B500031464FF07E5011F093FA2946064611F077
:105B600041FD00B92E46C4F810616CE4284A2B01AF
:105B700099580D9811F08EFB14AB53F82510139023
:105B80000C9811F087FB139B0146184611F07AFA26
:105B90000E9911F07FFB0F9911F074FA119BEBB184
:105BA00011F054FD404503DB5045A8BF504600E0CE
:105BB000404611F01BFB129A034652B14CB146B954
:105BC000139010F009FC139B18B9109A9742B8BFB4
:105BD0005B46104A42F82530013568E411F036FD85
:105BE0004845E1DA4846E4E752F8241043F8241027
:105BF000013463E4842100206C2E00200C2D002051
:105C0000CDCCCC3DF81F0020D037002054220020FE
:105C1000A4110020FC200020BA49099811F03AFB99
:105C200011F014FDB749ADF850000A9811F032FB9D
:105C300011F00CFDB349ADF852000B9811F02AFB9E
:105C400011F004FD00B2ADF85400002E3FF463AC37
:105C5000238B9F42BFF65FAC40425AE4A07928B143
:105C60001630C0B210F0B2FB002867D094F800E004
:105C700094F9051009FB0E83DA889B8894F801C01B
:105C8000D21A94F9043092B2534393FBF7F34FEADC
:105C9000520BA3EB0B030991E1781BB208934FEA77
:105CA0004C0681BB1CA90E4436F8201C2980012318
:105CB00009FB0EF158F8011003FA0CFC1CEA010F65
:105CC000B5F9006094F9021008BF184601FB06F10F
:105CD00091FBF7F1089B18BF4FF0FF30994209DBA9
:105CE000099B5A4392FBF7F2A2EB0B031BB28B42C8
:105CF000A8BF0B463AF81E2000FB03232AF81E30EB
:105D0000023507349EE41CAB1E44B5F9000036F999
:105D1000206CB04208DA0144884203DC8E423046EF
:105D2000A8BF08462880C2E7C1DD411AB14203DBA3
:105D30008842A8BF084606462E80B8E72880DFE7DD
:105D4000B3F90220B3F900004A43322192FBF1F289
:105D50004244328095F91620504390FBF1F0C4E4A0
:105D60000027DFF8C081B9F9020011F03FFA07EB14
:105D70004703014608EB030003F032FB12F07EFA02
:105D8000EA19B2F9043000B29842B2F9062003DBF6
:105D900082421346A8BF03460C37602F29F8023F02
:105DA000E1D1BFE4B37B002B54D0574BB3F90A00C9
:105DB00011F01CFA0146002010F09EF80123069312
:105DC00023689A0603D497F8E030052B16D14E4D80
:105DD000B5F9000011F00AFA0146069810F09CF897
:105DE000B5F9020011F002FA069B01460133D8B260
:105DF00010F092F8069B0233DBB206932368DB02B5
:105E000015D50024F67B414FE5B27319DBB2112B97
:105E10000DD8331937F9130011F0E8F9069B014644
:105E20001D44E8B2013410F077F80E2CECD1384C58
:105E300094F8AC21002A57D1364B1B78072B05D19B
:105E400004F0A2FA079BC01A334BD88001232370B9
:105E5000FEF795BC314B187810F00100A5D1002158
:105E6000AAE7294DB5F9060011F0C0F90146002056
:105E700010F042F8B5F9080011F0B8F90146012018
:105E800010F03AF802239AE71F4DB5F9080011F017
:105E9000ADF90146002010F02FF8B5F90A00EBE744
:105EA0000225DFF8648038F9150011F09FF9AB1E68
:105EB00001460135D8B210F02FF8082DF3D1062392
:105EC0007DE7114D059B35F9130011F08FF9059B06
:105ED0000146033BD8B210F01FF8059B0133072B96
:105EE0000593EFD104236AE70DF07CFDA4E70C4B8A
:105EF000074A1B6803F59C530833C2F8C030FEF70D
:105F000048BD00BF3333333F54210020542B0020C1
:105F10007C10002080210020F42000202C2B002069
:105F2000982200204C1200200346012283F84520CD
:105F300053F8043C103803B118477047022310B5DA
:105F40000168047B0A68A3401A420AD00024054A6B
:105F500040681470026822F001021204120C026000
:105F60004B6010BD342B002024234343F0B5A14CDB
:105F7000A14AE118E3585B689E8AB6B2F5B215F003
:105F8000010F4ED01D8825F400652D042D0C1D80B9
:105F90001D88ADB245F480651D80002515708D7E8D
:105FA000002D31D0557815B9C97DFF292CD101219B
:105FB0005170242101FB0041097E022901BF19888B
:105FC00089B241F400611980242101FB0041897DDF
:105FD00041F001011982242101FB0041097E92F95F
:105FE000005001318D420ED10021517092782AB1BA
:105FF0009A8822F440721204120C9A80242303FB24
:10600000004000234375F0BD242101FB00418D7D3C
:1060100005F0FE051D82C97DFF29DCD0FF2111702E
:10602000D9E7AF0744D5BFF35F8F0D7EEDB2012DE9
:1060300018D1897EB1B15178A1B1198821F480615C
:106040000904090C1980BFF35F8F198B19889570AB
:1060500089B241F400711980998889B241F4806154
:106060009980B8E7198BBFF35F8F242101FB0041B2
:106070000D7E022D0FD1897E69B1517859B11988F1
:1060800021F480610904090C1980998821F4806148
:106090000904090CE4E7242101FB00410D7E032DD6
:1060A000DAD1897E0029D7D051780029D4D0ECE705
:1060B0006F075CD5012595708D7E002D3FD05578FA
:1060C000002D3CD00D7E92F90060022D0F6A1D88D4
:1060D00021D925F480652D042D0C1D80B3F810E026
:1060E000F5B25FFA8EFE07F806E01E88B6B246F4F7
:1060F00000761E800E6AA91C1170198A0135C9B27A
:106100006DB27155998889B241F48061998019887E
:10611000C905FCD45FE7ADB245F400751D80B3F846
:1061200010E0F5B25FFA8EFE07F806E00F6A198AF2
:106130006E1C76B2C9B20335B9551570E7E75178D0
:1061400021B9242101FB0041497E41B1198889B25E
:1061500041F400711980117801311170D7E7198865
:1061600089B241F48071198001215170CFE715F097
:10617000400521D092F900C0B3F810E00F6A5FFA31
:106180008CF65FFA8EFE751C07F80CE06DB20F7E80
:10619000E91C8F42157005D1998821F480610904AA
:1061A000090C9980242101FB0041097E8D427FF476
:1061B00012AF023616700EE737067FF50CAF92F974
:1061C00000707E1C0AD0CE697D1CF65D6DB21E8209
:1061D000097E1570A9427FF4FEAE56E71570CD7D9D
:1061E0001D828D7E002D7FF450AF097E00297FF443
:1061F000F2AE4AE7B01400207313002003460222D7
:1062000010B41C7B1968A24040694A605A6810BCEF
:10621000136823F001031B041B0C136004F036B950
:1062200010B5084B07281B68C8BF14381844007EF7
:106230000C4604F0A9F920B12146BDE8104004F055
:10624000F5B910BD480C0020F7B5054690F8590087
:10625000002873D004F098F9044618B12023837104
:106260000023C3710621204604F0B4F9344B2B619E
:10627000002C63D0A388B3FA83F3C3F11F035A1C25
:106280004FD04FF00F0E2F4A103542F82350DAB29C
:1062900002F0030502F0FC0202F1804202F58032B6
:1062A00097682168AD000EFA05FE27EA0E0701F196
:1062B00040419760A1F584319768C1F38721A940D7
:1062C0003943012720489160C65C07FA03F3D9439C
:1062D0001E4A536115680D40156055680D405560A4
:1062E00015681D43156095680D409560D568294077
:1062F000D16091680B439360154B9A5DF02A10DDD5
:10630000F02230449A55037C01A88DF80430032311
:106310008DF8053000238DF807708DF806300EF0EB
:1063200045FBA3880122B3FA83F3C3F11F0312FADA
:1063300003F31FBF05490A6813430B6003B0F0BDA8
:10634000295F0008D80A002080AC01080004014041
:10635000180B0020C26C70B515880446ADB2A906B2
:1063600006D5036B23B9C36AA3B1908880B298475E
:106370002B0620D5636AA26A9A42E36C17D0511C9F
:10638000A069A162825C9A802369994213D3002399
:10639000A36270BDE169928840694E1CD2B2E66189
:1063A0004254E169E268914228BFE361E0E7DA68BC
:1063B00022F08002DA6070BD70B50446C56C866854
:1063C000AB8986B023F400531B041B0CAB8183798B
:1063D000617913F0020F14BF4FF40052002213F042
:1063E000040F14BF4FF48060002011F0010F14BFA0
:1063F000042300238907298A48BF43F0080389B290
:1064000021F4405111432982AA8922F4B05222F08A
:106410000C021204120C02431343AB81AA8A01A896
:1064200022F440721204120CAA820EF0D5FD294A01
:10643000039B0499954218BF19461922AB894A4318
:1064400013F4004F14BF7100B100B2FBF1F16426E8
:10645000B1FBF6F3AA891801120406FB13132ED51B
:10646000DA003232B2FBF6F202F0070242EA00032F
:106470009BB22B81A379DB070BD5E36C154A9342C2
:1064800025D0A2F57442934203D101200121FFF7E8
:10649000C7FEA379E26C13F0080F938A0BBF23F0B9
:1064A00008039BB21B0443F0080308BF1B0C938234
:1064B00093899BB243F40053938106B070BD1B01D6
:1064C0003233B3FBF6F303F00F030343D0E70020AE
:1064D000DCE700BF00380140072838B5D8BF0446C4
:1064E0000B4BC8BFA0F114041B6805462344187E5B
:1064F00004F04AF858B127220134C4718271122184
:1065000004F068F82846BDE83840002188E638BD28
:10651000480C00200348D0F8B0300BB1A830184721
:10652000704700BF240000200348D0F894300BB11E
:106530008C301847704700BF240000200248836F4A
:106540000BB1703018477047240000200248C36D1B
:106550000BB1543018477047240000200248036CE8
:106560000BB1383018477047240000200248436AB6
:106570000BB11C3018477047240000200248836884
:1065800003B11847704700BF240000202DE9F04FE9
:10659000B0F1FF3F87B0804600F0F580242000FB7B
:1065A00008F0824B1E581F189946002E00F0EB8011
:1065B0001430184410220021746814F02AF9BD68C0
:1065C00008F10103FF68DBB215B11522EB71AA7166
:1065D00017B11622FB71BA71B07B0EF0C9F9A3880E
:1065E000284623F440731B041B0CA38004F019F805
:1065F000384604F016F81621284603F0EBFF162162
:10660000384603F0E7FF4FF0080A4FF0640B25B15E
:106610002B68AA889B681A4203D1BBF1000F40F097
:10662000B580284603F0F8FF0A2003F0F5FE28465F
:1066300003F0F7FF0A2003F0EFFEBAF1010AE6D1FA
:10664000384603F0E9FF0A2003F0E6FE284603F08F
:10665000E3FF0A2003F0E0FE284603F0E2FF0A20F1
:1066600003F0DAFE384603F0DCFF28461F2103F072
:10667000B1FF1F21384603F0ADFF4D4B4D4F9C42FB
:1066800003F5DE331A6901A80BBF42F4001242F48D
:1066900080021A611A610BBF1A691A6922F400128A
:1066A00022F480021A61A388434A23F440731B0436
:1066B0001B0CA380242303FB089898F81030002BB0
:1066C00008BF1746238807EB47079BB243F0010337
:1066D0002380A5880EF080FC039B384825F03F05F9
:1066E000B3FBF0F02D042D0C0543ADB2A58021883D
:1066F0004FF4967221F001010904090CB3FBF7F382
:1067000021804FF47A7142439BB2002B92FBF1F24D
:1067100008BF0123013292B243F400432284A383D1
:10672000238800259BB243F001032380238801A81E
:1067300023F4816323F002031B041B0C43F48063E6
:1067400023804FF480432381238823F080031B049C
:106750001B0C23800124337C8DF805508DF8043008
:106760008DF806508DF807400EF020F9F37B9DF868
:1067700007208DF804308DF805508DF806505AB179
:1067800001A80EF013F907B0BDE8F08F0A2003F05E
:1067900043FE0BF1FF3B3AE75A09094903F01F0397
:1067A00004FA03F3203241F82230ECE7B014002061
:1067B0000054004000350C00801A060040420F00D3
:1067C00000E100E0F8B52425214F069C05FB00758B
:1067D0006E680EB34900C9B2A975EA75012100229D
:1067E0006A76A9762B7669752A75B3882C62990525
:1067F000EC611ED43388DA0516D44FF48054338804
:106800009B050CD5013CFAD1124A138801339BB287
:106810001380FFF7BBFE00E034462046F8BD338806
:106820009BB243F480733380B3889BB243F44073CC
:10683000B38024234FF4805403FB00777B7D13B196
:10684000013CFBD1E0E73C7D84F00104E5E700BFBB
:10685000B0140020281C00201FB5012202AB044602
:1068600000931C2106231046FFF7ACFF08B3042158
:106870009DF808309DF8092042EA032242F38D0278
:1068800092FBF1F29DF80A30E2829DF80B2042EA79
:10689000032242F38D0292FBF1F29DF80D30228328
:1068A0009DF80C2043EA022343F38D0393FBF1F39D
:1068B000638304B010BD1FB502AB044600930222EF
:1068C000062318210120FFF77DFFB8B19DF809309C
:1068D0009DF808201B0203EB9203E3829DF80B3026
:1068E0009DF80A201B0203EB920323839DF80D30D1
:1068F0009DF80C201B0203EB9203638304B010BDD0
:106900002DE9F043314B85B01B78054602AE002BD4
:106910003DD000242746A046A14601340096082316
:10692000322253210120E4B2FFF74CFF18B90020B6
:1069300005B0BDE8F0839DF809209DF80830202CB3
:1069400003EB02231BB29DF80B2099449DF80A30FB
:1069500003EB02231BB298449DF80D209DF80C30E8
:1069600003EB02231BB21F449DF80F3003F07F039B
:1069700001D0002BD1D199FBF4F998FBF4F897FBE7
:10698000F4F4A5F81690A5F818806C83D0E700966B
:106990000623322253210120FFF714FF0028C6D01E
:1069A0009DF809209DF8083003EB0223EB829DF847
:1069B0000B209DF80A3003EB02232B839DF80D205A
:1069C0009DF80C3003EB02236B83B1E7E215002046
:1069D0002423434373B5244E0546F218F3585C68EC
:1069E000A38A9BB20193019B13F4706F1CBF012318
:1069F0001375019B13F4E06F1DD0238BA38823F440
:106A000080631B041B0CA380019B9B0513D423886C
:106A1000980510D42388D9051AD52388DA05FCD423
:106A200023889BB243F40073238023889B05FCD406
:106A30002846FFF7ABFDA38A23F470631B041B0CED
:106A4000A382242303FB056500236B7502B070BD90
:106A500023889BB243F400732380A38823F44073FC
:106A60001B041B0CA380E6E7B014002073B5441C84
:106A70008DF807302AD0022828DC2423214E03FB7E
:106A800000635D6815B34900C9B29975DA750021D4
:106A900001220DF107045A7699761A765A751975FE
:106AA000DC611C62AB8899051DD42B88DA0515D4EE
:106AB0004FF480542B889B050BD5013CFAD1124A28
:106AC000138801339BB21380FFF760FD002002B0F2
:106AD00070BD2B889BB243F480732B80AB889BB234
:106AE00043F44073AB8024234FF4805403FB0066CF
:106AF000737D13B1013CFBD1E1E7307D80F00100F3
:106B0000E5E700BFB0140020281C002010B50023CA
:106B10002A221C2104460120FFF7A8FF02230E228F
:106B20001C210120FFF7A2FF03230F221C210120BB
:106B3000FFF79CFF12232B221C210120FFF796FF59
:106B4000152003F021FD18B1202383710023C371A8
:106B5000062103F03FFD02232C221C210120FFF718
:106B600085FF01232D221C211846FFF77FFF0023FC
:106B70002E221C210120FFF779FF05232A221C2148
:106B80000120FFF773FF4FF48073A38210BD10B58F
:106B9000082304460F2218210120FFF767FF0E2368
:106BA000102218210120FFF761FF4FF48053A382C8
:106BB00010BD184B10B51B780446DBB108232D22FD
:106BC00053210120FFF752FF0A23312253210120D4
:106BD000FFF74CFF0C232C2253210120FFF746FF27
:106BE0009023382253210120FFF740FF4FF4807398
:106BF000A38210BD08232D2253210120FFF736FF69
:106C00000A23312253210120FFF730FF0A232C22CF
:106C1000E8E700BFE21500200120FFF7A5B9012039
:106C2000D6E60020FFF7A0B90020D1E60000000062
:106C30002DE9F0435C2885B005460C4600F07E85C2
:106C400000F2D5803A2800F0908341D82C2800F03B
:106C5000378410D8222800F0E98304D80A2800F0ED
:106C60001D83002043E0262800F081832A28F8D1E4
:106C7000BA4B197888E3322800F07B840FD82E288D
:106C800000F07D843028ECD10025B54E56F8251053
:106C90002046013502F06EFE202DF7D144E1342864
:106CA00000F0E2833628DCD1AE4DAF4F05F120066F
:106CB000002395F90220D91991F90610914200F0AC
:106CC0007B850833202BF6D10835AE42F0D12BE17D
:106CD000462800F0B08436D83D2800F0538309D808
:106CE0003B28BED101200B685A1C0A60187005B001
:106CF000BDE8F083402800F03F844228B1D1974B93
:106D000020461A780B68994D591C21601A70984BCF
:106D1000196802F02FFE974B20461A7A2368591CF7
:106D200021601A70298802F039FEA988204602F0F5
:106D300035FE2989204602F031FE0021204602F06E
:106D40002DFE002105E34F2800F0AC8420D84B280D
:106D500000F0F5834D2884D10025874F874E3B787E
:106D60009D4280F2E180236816F81510581C06EB4E
:106D70004502206019705178204601EB810101EB3A
:106D8000810101F2EE2189B202F008FE0135E6E749
:106D9000502800F067845A287FF463AF784E0B6860
:106DA000F278002A00F0BF845A1C0A6008221A7088
:106DB0000B685A1C0A6001221A70724D23682A79E6
:106DC000591C21601A702368AA78591C21601A7016
:106DD0002988204602F0E2FDE989204602F0DEFD26
:106DE0002368F279591C21601A70EA7815E170283D
:106DF00000F0CF8200F21681672800F05E8200F278
:106E00009580602800F0C98452D85E287FF429AFAD
:106E100000260021204602F0C1FD0021204602F09C
:106E2000BDFD0021204602F0B9FD2368564D5A1CD5
:106E300022601E702B68204693F82C202368591C72
:106E400021601A702B6893F836202368591C216042
:106E50001A702B6893F837202368591C21601A7028
:106E600023685A1C22601E7023685A1C22601E7000
:106E700023685A1C22601E702B68598F02F08EFD09
:106E80002B682046198F02F089FD2B68204693F865
:106E90002E202368591C21601A7023685A1C226016
:106EA0001E702B68598E02F079FD2B68998E50E286
:106EB000652800F0378166287FF4D3AE334EB28A5E
:106EC000B2F5006F00F2E681B2F5806F00F2E48166
:106ED000B2F5007F2CBF0227012700257319996B9B
:106EE000204691FBF7F1043589B202F057FD0C2DD5
:106EF000F4D10125264E274F396A56F8250010F0A7
:106F00007DFA11F0BBF9013581B2204602F046FD51
:106F1000042DF1D10025204E36F8251020460135EC
:106F200002F03CFD032DF7D10120E0E66C2800F0D3
:106F3000018235D8682800F0E78169287FF491AE96
:106F400000250D4E154F33789D42EDDA37F81510B8
:106F5000204602F023FD0135F5E700BF882100201F
:106F6000AC290020163700203C3700207C0C002084
:106F7000C8200020542200201C1800202C190020BA
:106F80006C340020B83700209C20002024200020F2
:106F900004370020803400207C300020542B002057
:106FA0006D2800F0DA816F287FF45BAE574D2B68B7
:106FB0001A780B68591C21601A702B689A7823681C
:106FC000591C21601A7000232A681A4451792268DA
:106FD0000133501C032B20601170F5D12B68204623
:106FE0001A7A2368591C21601A702B68DA78236892
:106FF000591C21601A702B681A792368591C21606A
:107000001A702B68598902F0C9FC2B685A7A2368D8
:10701000591C21601A702B685A782368591C21600A
:107020001A7081E77E2800F06F832AD8782800F054
:107030004A810DD875287FF414AE354A12F8013F05
:10704000002B3FF471AF2168481C20600B70F5E7FE
:107050007C2800F03A837D287FF403AE2D4B226814
:107060001978501C2060117022685978501C2060DB
:1070700011709A782368591C21601A70264BD988A0
:1070800067E196284ED010D87F2800F090828328A0
:107090007FF4E7AD214D2046298A02F07FFC698A02
:1070A000204602F07BFCA98A53E1F02800F001821F
:1070B000F1287FF4D6AD1A4B03F1700122681878DD
:1070C000551C2560107022685878551C256010707A
:1070D00022689878551C256010702268D878551C55
:1070E0002560107022681879551C25601070226880
:1070F0005879551C25601070226898790733551C03
:10710000994225601070D9D10EE700BF3C3C0020A9
:1071100096AC0108A0200020343C0020B8370020A5
:10712000C619002000264FF6FF78AB4FDFF8F0922B
:107130000096019602960396F1574B1C0BD048FA25
:1071400006F3D80707D5B9F800303341DA0702D57E
:1071500002A802F0DBFE01360B2EEDD100260FF265
:107160007029D9E900893246404649460FF0D6FADF
:10717000002100F0010050EA010307D0F0B20FF047
:1071800025F918B1314602A802F0C0FE0136252EBD
:10719000E9D100273E46914BDFF888821B78DB0758
:1071A00042BF029B43F0010302933946404602F07E
:1071B000B9FE48B1394602A802F0B4FE18B1314612
:1071C000684602F0A3FE01360137252FEDD1844B2E
:1071D0002046B3F8501002F0E1FB824B204619889C
:1071E000814F89B202F0DAFB804B204619684A01D0
:1071F000C1F3400302F020021343C1F3800243EACB
:107200004203C1F3C00243EA8203C1F3401243EADE
:10721000C20301F01001194302F0C0FB04226946C9
:10722000204602F09DFB23683A78591C21601A70B1
:107230006F4B204619886429A8BF642102F0AEFB79
:10724000962D22D123685A1C226003221A702368CB
:107250007A78591C21601A700822193E96FBF2F2C6
:10726000236882F30402591C216020461A7001A988
:1072700002F076FB23685A1C226010221A705D4BC4
:107280001988204602F076FB4EE60021204602F0E7
:1072900085FBE1E7082720E604271EE656480FF0A5
:1072A00035FA002354498342BFF63EAE22685D5C46
:1072B000561C266001331570F5E710224F49204611
:1072C00002F04EFB30E64E4D05F16006A9882046DF
:1072D00002F064FBE988204602F060FB2989204621
:1072E00002F05CFB2368AA7A591C21601A7023689B
:1072F000EA7A591C21601A7055F80C1B204602F0DE
:1073000039FBAE42E2D10FE6002518263D4FDFF8EB
:10731000188106FB0573597C31B92046013502F00E
:107320003DFB082DF5D1FFE558F8250010F0B4F924
:1073300081B2F2E7344D2046298802F02FFB69889C
:10734000204602F02BFB0A23B5F9041091FBF3F160
:1073500089B2204602F022FBE6E52C4B2046196854
:1073600002F008FB2A4B1988F3E7002189E7294D31
:107370002046298802F012FBA988204602F00EFB65
:107380002989E6E7244B99782268501C2060117007
:1073900042E600212148036801EB41029D5C23681D
:1073A00001315E1C26601D7003680A2913445D7854
:1073B000236803F1010626601D70036813449A7860
:1073C000236803F1010525601A70E4D1ACE500BF24
:1073D00090E33FF408000000C7AC01082C2B00200C
:1073E000FC000020281C0020FC1F0020842100201D
:1073F0002C1C0020BC2B0020102000205421002039
:10740000381A00204C2800206C2E0020A4100020E8
:10741000681400207C0C0020C22000209C2000204A
:107420007E2B00208C0C0020FC200020AC4D05F1B0
:10743000500628780EF015FF2368027A591C216047
:107440001A7023686A78591C21601A702368AA7818
:10745000591C21601A702368EA780435591CAE4221
:1074600021601A70E5D15FE59E4B03F15A01226855
:107470005879551C2560107022681878551C2560B5
:10748000107022685878551C256010702268987812
:10749000551C256010702268D878551C2560107026
:1074A000226818790633551C994225601070DED188
:1074B0003AE58D4D2046E98902F070FAA98948E73E
:1074C0008A4D0B682A7A591C21601A70A98B2046B4
:1074D00002F064FA298B204602F060FA698B20469C
:1074E00002F05CFA2368EA7C591C21601A70A98CAE
:1074F000204602F053FAE98C204602F04FFA236846
:10750000AA7F591C21601A70236895F82020591C05
:1075100021601A70698C204602F040FA2368EA7AEA
:10752000591C21601A70E968204602F023FA23688A
:107530002A7C591C21601A7095F821206DE56C4D4C
:107540000B682A79591C21601A7023686A79591CC2
:1075500021601A702988204602F020FA2368AA794F
:10756000591C21601A706988204602F017FAEA79DE
:1075700053E55E4B5A7D50E508225C499FE65D4D20
:1075800005F14006B5F88010204602F007FA23689E
:1075900095F88220591C21601A70236895F8832081
:1075A0000435591CAE4221601A70EBD1BCE4514D38
:1075B000002306272846002107FB03F6226802F174
:1075C000010EC4F800E01370226802F1010EC4F845
:1075D00000E011708A192A4492F8C0E02268013153
:1075E00002F1010C0629C4F800C082F800E0E5D1E0
:1075F0000133062BDFD1002221684D1C25600B7062
:1076000021684D1C25600A70811891F8E4502168AA
:1076100001324E1C0B2A26600D70EDD123685A1CD6
:10762000226007221A7023685A1C226000221A70F6
:1076300090F8F020F1E40BF0EDF9002814BF0322DC
:10764000022223682C4D591C21601A70298820467B
:1076500002F090F9A968204602F08CF902F0E2FCF1
:1076600001460EE601250B68244E5A1C0A601D7067
:107670000B68B278591921601A700DF05DFD3388DE
:1076800058431F4BB3F9003090FBF3F023685A19AD
:10769000226018700DF050FD23685A19226018708E
:1076A000318856E600250B6820465A1C0A601D707A
:1076B0000B685A1C0A601D700B685A1C0A60294628
:1076C0001D7002F057F92946DBE50E4D204629884A
:1076D00002F064F96988204602F060F9A98838E66A
:1076E000601E0020001F0020A62000205422002041
:1076F000982E0020AC29002010040020D033002058
:1077000094370020343C00203A4B1A780B68591CFF
:1077100021601A70384B9A782368591C21601A70BE
:10772000364B9A7879E4B278591C21601A70344B40
:107730001A782368591C2160FFF73EBB2D4E0B6859
:107740007279304D591C21601A702B682046198CB3
:1077500002F024F92B682046D98B02F01FF97189B9
:10776000204602F01BF9B189204602F017F92B6878
:107770002046598C02F012F92B682046998C02F0B1
:107780000DF9F189204602F009F9318A204602F00C
:1077900005F92B6893F826203FE4174BDA780B683D
:1077A000591C21601A70184B5A792368591C2160A2
:1077B0001A70124BDA7830E423682046591C216095
:1077C0001A70298802F0EAF82368EA78591C2160C7
:1077D0001A7023682A79591C21601A702368AA79C3
:1077E000591C21601A7023686A79591C21601A702B
:1077F000FFF76ABA6C340020A6200020B6200020D3
:10780000742000209C200020D22C00202DE9F04F75
:10781000A74B00F59C4909F12009C3F80090A54B3E
:107820008BB01C788046002C65D1A34EA34DA44F8D
:1078300033789C420093C0F2C18042F201024FF4BF
:107840007A7AA04BB8FBFAFA1B68134001939E4B5F
:1078500006D09E4A12781A709D4A11789D4A11707E
:107860001E781EB19B4B1E7886F001060F23032065
:1078700085F82430924B00249A8CDB8C964D039330
:10788000964B029293F800B00AF59672BBFBF0F3A8
:1078900003EB4303ABEB0303DBB20493904BA5F183
:1078A000260705920690009A9442C0F2AF80834B5F
:1078B0008C4D93F824308C4C0F2B0CBF01220022EE
:1078C0008A4B1A7040F028811B200EF07FFD0028A3
:1078D00040F022812B68E268A3609B1AC82B05D96F
:1078E0000123042084F821300EF000FF7B4A137836
:1078F0000133137005E07E4A1268904201D9013CC1
:107900001C70704B1A68019312F4805F05D0002040
:107910000EF05CFD08B909F039FD694A537D9246C5
:10792000002B00F019816E4A013B32F913009AF8DE
:1079300017301BB1C0F53B60083000B2A0F57A707B
:10794000B0F57A7FA8BF4FF47A7020EAE0700FF0AC
:107950004DFC68490FF09EFC0FF09EFE664B1880B0
:10796000664B614C984503D9A3780BB90123A370EA
:10797000A378DFF89CB1002B00F0688194F82170A7
:107980009BF800501B200EF021FD012F05F001098E
:1079900008BF0025534EDFF87C81009018BF05F02A
:1079A000020594F82030052B00F24C81DFE813F03B
:1079B000140171017C019A01A501BB015048072CFB
:1079C000D4BFE15DE1B243689847032C1ADCC8B12B
:1079D0004C4B33F8242003EB8401831A4FF47A7064
:1079E00058434B889B1A90FBF3F040F6CA0300F50E
:1079F0007A709842A8BF184640F2EE239842B8BF6A
:107A0000184680B225F81400013411E7C6B137F9E1
:107A10001400029A80B290424FEA840E02D3039A75
:107A2000904220D9384A52F80E0082450AD233F8E3
:107A30001400019AE2B923F814000635013432E744
:107A40003046E6E7E0B2079306F02AFD032C079BD9
:107A5000EFDC012297F824C002FA04FE2CEA0E0E95
:107A600087F824E0E5E7059A274941F80E20E0E78A
:107A7000049A97F86EE025F81200BEF1000F06D1C7
:107A8000BBF1020FD7D94FF0010287F86E20B5F88D
:107A900000E068881D4A7044B5F804E0704400B204
:107AA00022F81400069A90FBF2F080B2C3E700BF00
:107AB0002818002054190020450F00207C130020B6
:107AC000542200208C2100202D2B0020F8170020AC
:107AD0001000002011000020A2130020F80E00204A
:107AE000542B002098220020982B00204A150020BB
:107AF00050190020AAF1823F7C2B0020404B4C0003
:107B00001C180020A41B0020FC0E0020EC130020F9
:107B10002C2B0020982E002001238D4A0420137066
:107B20008C4A8D4E13700EF0E9FD2B68A268E3605D
:107B30009B1A6268934284BF002384F8213000249A
:107B4000864B1D78AC42BFF6D1AEE0B206F0A8FC81
:107B500026F814000134F5E7019A126811047FF544
:107B6000FFAE7F4AD2F88810A8EB01010029FFF68A
:107B7000F7AE7C49C2F88890487C7B4931F8100008
:107B80009AF8161080B290FBF1F092F88C10013147
:107B900001F00F0182F88C10114481F88D00184615
:107BA0008D32815C01300B4410281BB2F9D193FB5C
:107BB000F0F31BB2002B0ADB642BA8BF64239AF8F6
:107BC000172032B918B20FF011FB6849C2E6002342
:107BD000F5E7C3F16403F5E7B9F1000F2AD00EF021
:107BE00009FC012806D164213268B8F8023001FB93
:107BF00003232361009B5BB198F8063043B10CF07E
:107C00000DFB032384F820304FF47A73E361C8E658
:107C1000012F17D0336822699A4207D20CF0FEFA7E
:107C2000032384F8203040F6B833EFE7012384F8CB
:107C30002030B6E6009B4FF480603BB30EF048FD69
:107C40000023236115B1284603F0A2FA0EF0D2FBFF
:107C500006460EF0C1FB464D002800F08F809BF8D1
:107C60000030DA0740F18A80BAF822000FF0BEFA3D
:107C7000404B0146D8680FF0BFFC002800F0198186
:107C80000122374B83F89D2001238AE00EF010FD7E
:107C9000D6E7012F01D10523C9E798F80730012B5A
:107CA000BCD00CF0BBFA7CE6012F04BF052384F89E
:107CB0002030B9F1000F09D00325BAF91820264B5E
:107CC0001A805A809A80B8F80020DA803368626996
:107CD0009A4202D3B9F1000F35D147F23053E36134
:107CE0000323A4E702200EF009FD09F04FFB3268E0
:107CF000E3691344A361042399E7012F0ED133688C
:107D0000A2699A429ED21C4B187818B90EF05EFBFD
:107D1000002897D102200EF0E9FCBCE73268E36945
:107D20001344A3618EE764213268B8F802304FF43F
:107D3000806001FB03232361002384F82030E3707B
:107D40000EF0B6FC2DE6012F3FF42BAE7AE700BF14
:107D50001000002011000020542B0020450F0020AF
:107D60007C130020600C0020740C002014AE234112
:107D700068110020342200200000002000226E4BF9
:107D800083F89D20002E7FF47FAF00226B4B1A609A
:107D90005A609A606A4B1B6893F82D30002B7FF471
:107DA00073AF2B709BF80030DB0724D5019B1B6859
:107DB000DF0620D5634A1278D5061CD4D8041AD41D
:107DC0000EF00AFBB8B9604B5B4D1B78002B00F03E
:107DD0008B805E4B9B78002E75D1002B00F0868047
:107DE0005B4B1A685B4B1B689B1A002B7EDA09F011
:107DF000CDFA85F89E6000221346BAF81A50BAF8F8
:107E00001C70554931F912009B08A842C4BF63F0A9
:107E10007F03DBB20132B842B8BF43F04003042A0B
:107E2000F0D1454D95F89F209A4266D14B4AB5F95D
:107E3000A0001268D1694A4A91FBF2F202F5FF42B2
:107E40007F32904206DC4FF47A7291FBF2F10144EA
:107E5000A5F8A0103C4A85F89F301778002F40F015
:107E60006E8138460EF0B2FA00284CD085F8A37027
:107E700009F086FB9BF80030DB077FD495F8A20061
:107E800000287BD1B5F9A030322B77DD012295F89F
:107E90009F3085F8A220572B40F08F81314804F0A5
:107EA000B9FF314B1B685F0768D50A222F4B1A8038
:107EB00064E0002E7FF4E8AE1F4B93F89D30002B5A
:107EC0007FF4E2AE61E73BB14FF47A71204A126869
:107ED00001FB03231F4A136095F89E30002B8AD0C4
:107EE00003F040F9002305E0002EF5D1102003F047
:107EF0004FF9012385F89E307DE70022A5F8A020E8
:107F000085F8A220A6E71A4B18609BF80030D90725
:107F1000B4D5184B1B788BB3E3787BBB95F8A330B3
:107F20000133DBB2032B85F8A33027D9074B5B78ED
:107F300013B309F02BFA9DE77C130020DC2000200E
:107F40009C2000204915002000000020C2200020B5
:107F50009822002010230020542B0020F022002023
:107F600018FCFFFF34350020842100200623002068
:107F7000142300202D2B0020002EDAD0019B1B683B
:107F8000580728D595F8A6309BB19BF80030D90743
:107F90000FD5B84BB3F90620BAF81A309A4208DD6B
:107FA00000200EF013FA20B9322385F8A600A5F8B8
:107FB000A83011200EF00AFA002800F0778195F819
:107FC000AA302BB995F8A43013B93223A5F8A830FC
:107FD000012385F8AA300023A74D08AE089305F1C8
:107FE00050077360294615F8010C0EF0C9F930B13D
:107FF00015F8021C242902D8304601F087FF043509
:10800000AF42EFD19D4B96E8030083E803009C4B01
:108010001E78002E00F05A8101200EF0D7F9994EFB
:10802000994D18B9E378002B00F0558333689B070E
:1080300040F151832C8814F0010440F05183012059
:108040000EF046FB02200EF0C1F9002800F04A8332
:10805000002C00F0478301200EF02AFB2B889F079D
:1080600002D402200EF034FB2988012011F0030114
:1080700018BF012102F010FB24200EF0A7F938B937
:108080009BF800305C0744BF23F004038BF80030FA
:10809000336813F00A0F17D006200EF097F9002866
:1080A00000F024832B88580602D440200EF010FBE9
:1080B00007200EF08BF938B10A22744BB3F9043063
:1080C00093FBF2F3724A13800C200EF07FF9002824
:1080D00000F010834FF480700EF0FAFA6D4B1B78AD
:1080E000082B01D00E2B02D140200EF0E1FA019BAB
:1080F0001B6859050FD5684B1B79002B40F0FF8298
:108100009BF80030DA0740F100833C200CF050FE71
:10811000002840F0FF820122604B1A7009F050F9EC
:1081200033685B0708D503200EF050F9002840F0B3
:10813000F78208200EF0BCFA0BB0BDE8F08F5F2B81
:1081400020D1B5F9A030B3F5FA7FFFF617AF95F857
:10815000A230002B7FF412AF012385F8A2309BF8E8
:10816000003013F0010602D009F010F906E70F20E5
:1081700003F00EF8B5F8A03085F8A260FA3BA5F838
:10818000A030FBE66F2B7FF475AEB5F9A030B3F5E8
:10819000FA7FFFF6F3AE95F8A230002B7FF4EEAE37
:1081A000012285F8A2209BF80020D20702D409F012
:1081B000E7F9E3E63A4A1360E0E6019909684E07F9
:1081C00016D55A2B14D195F8A43023B185F8A40004
:1081D00085F8A520D2E695F8A63083F0010385F84E
:1081E000A6301BB10B2002F0D3FFC7E60C20FAE744
:1081F0005D2B00F0AA825B2B00F0AD825E2B40F07D
:10820000AC820320A2E2A72B05D1264A137843F0C3
:1082100004031370B2E60022BB2B089218D102238C
:10822000ADF82230204BBDF820109A890A449A817B
:10823000BDF82210DA890A44DA8108F093FDB5F816
:10824000A030FA3BA5F8A030002385F8A23095E6CF
:10825000B72B02D14FF6FE73E2E7BE2B03D1022308
:10826000ADF82030DEE7BD2B7FF488AE4FF6FE730D
:10827000F6E700BF542B0020621E00203839002092
:1082800090290020842100207E2B00206C2E0020CD
:108290008C1000208821002024220020C4100020FF
:1082A0001423002049150020A620002095F8A430B2
:1082B000002B3FF490AE9BF8003013F0010302BF97
:1082C00085F8A430012385F8A53084E64FF00C0929
:1082D000BB4DBC4F05F15A08294615F8010C0EF0AC
:1082E0004FF8E8B12979AB7809FB0170B64A013B38
:1082F00003EB43031344D0F8B02095F803E0934216
:108300000ED0C0F8B030012303FA01F197F8DC3049
:1083100080F8ACE023EA0101C0F8B46087F8DC1013
:1083200006354545D8D1A94BDFF8B0821E68A84B69
:10833000A8F1AC051B680293A64B1B78039300239E
:108340000093D8F80430002B6BD01F78002F68D032
:10835000D8F8082002998A1A002A0DDB01F5FA7272
:10836000C8F808200122009902FA01F195F8DC20F2
:1083700022EA010285F8DC20039A002A51D098F8FD
:10838000002059780432D2B2002940F0518192493C
:1083900031F91210BAF8182002F1C80081422ADD22
:1083A00093F8029095F8DC20009B1A41D20738D44C
:1083B000B9F1000FCCBF0220012002F081FF7A1E2C
:1083C000162A41D8DFE812F035004D00570067004B
:1083D0007E008500A000BB00D700E300EF00400056
:1083E000670074008500A000BB009400AF00CB00C4
:1083F0000C0118012601C83A914203DA9978C1F1BB
:108400000009CFE70123009A03FA02F295F8DC3065
:1084100023EA020385F8DC30029B03F5FA73C8F8FF
:108420000830009B08F10C080133042B009388D11D
:10843000F2E5317801204944FA29A8BFFA2121EA5E
:10844000E17131700DF0FEFFD5F8E0000BF012F98C
:108450000123009A934095F8DC20134385F8DC3023
:10846000DFE7B178022049446429A8BF642121EAEA
:10847000E171B170E6E731798944B9F1640FA8BFC1
:108480004FF0640929EAE97986F804900DF0EEFFCF
:1084900049460320D6E7B1790D2049446429A8BF95
:1084A000642121EAE171B1710DF0CCFF0D2FCBD029
:1084B00071790E2049446429A8BF642121EAE17141
:1084C0007171BFE7F1790520494481F30801F17129
:1084D000B8E7D5F8E0200F20D1784944C829A8BFD3
:1084E000C82121EAE171D1700DF0ACFF0F2FABD0A4
:1084F000D5F8E020122011784944C829A8BFC82126
:1085000021EAE17111709DE7D5F8E0201020117982
:108510004944C829A8BFC82121EAE17111710DF0B1
:1085200091FF102F90D0D5F8E020132051784944C6
:10853000C829A8BFC82121EAE171517082E7D5F8A6
:10854000E020112051794944C829A8BFC82121EA57
:10855000E17151710DF076FF112F3FF475AFD5F831
:10856000E020142091784944C829A8BFC82121EAF5
:10857000E171917066E7D5F8E020092091794944CE
:10858000C829A8BFC82121EAE17191715AE7D5F83D
:10859000E0200A20D1794944C829A8BFC82121EA8E
:1085A000E171D1714EE7D5F8E0200B20117A4944F2
:1085B000C829A8BFC82121EAE171117242E700BFB2
:1085C000011F00207C130020D2AC01083C3C00209D
:1085D000982200202D2B0020542B0020281400204E
:1085E000717815204944B1F5967FA8BF4FF4967174
:1085F00021EAE171717025E7D5F8E020162092F8A4
:1086000037104944FE29A8BFFE2121EAE17182F812
:10861000371017E7D5F8E020172092F836104944B4
:108620006429A8BF642121EAE17182F8361009E7C4
:1086300001297FF40DAF504931F9121040F6330291
:108640009142A8BF11469A784FF49663B1F5617FC5
:10865000B8BF4FF4617193FBF2F3A1F561710C2F78
:1086600091FBF3F31ED0182F7FF4F2AED9B2C829D4
:108670000B46A8BFC823D5F8E020D8B292F817E07F
:1086800070453FF4E5AEA3EB0E034FF0080E93FBED
:10869000FEF30133DBB2D075384604930DF0D2FE01
:1086A000049B11E0354ADBB252789A423FF4D0AED7
:1086B000184604930DF096FC049B384619460DF0BD
:1086C000C1FE049B0133DBB2002B3FF4C1AE184660
:1086D00002F0F6FDBCE601200DF0EAFF0124B1E452
:1086E0000024AFE402200DF0E3FFBDE440200DF0D4
:1086F000DFFFDDE44FF480700DF0DAFFEEE41420CC
:108700000DF064FE00287FF400AD07F03BFE02F0A0
:10871000C7FC00E502F0D6FA3C200CF017FBF7E4AA
:108720002C8814F008047FF407AD08200DF0D0FF6A
:10873000134B1A68134B1A600F4BDA88124B1A80CE
:10874000124B1C60124B1C60F6E401200138C0B2D1
:1087500007F0DEFF12E40220F8E7562B01D108F003
:1087600001FB95F89F30972B7FF44DAD4FF4C87205
:10877000084BFFF79CBB00BF542B0020FC1F0020C0
:10878000A4100020A01000209410002098100020B9
:1087900090100020082300202DE9F04F85B081467D
:1087A00007F0F0FDCB4B1D78002D40F0AE83CA4F93
:1087B0003B685A0540F1A983C84BC94E1B68002B82
:1087C00000F05A81C74C32682368D31A7C2B40F2E0
:1087D00053814FF024082379DFF844A3013322604A
:1087E0002371AAF1340B404607F0A6FD5AF8040F96
:1087F0000EF0FCFC0090BBF814000EF0F7FC009AA1
:10880000014610460EF0FAFDB7490EF043FD0EF09A
:108810001DFF08F1010800B25FFA88F807F07CFD3F
:10882000B8F1270FDFD1302007F086FDB4F908003A
:1088300007F072FD07F07AFD23799B0734D141F2EE
:10884000883322689A421CD94FF06408DFF8D4A21A
:10885000102007F071FDDAF8000090FBF8F000B28C
:1088600007F05AFD212007F067FDDAF8003093FB8E
:10887000F8F008FB10300028B8BF404200B207F003
:108880004BFD142007F058FD984BB3F904000A2360
:1088900090FBF3F007F040FD1C2007F04DFD002099
:1088A00007F03AFD07F042FD2379580740F0BD80FC
:1088B000022007F041FD8E4BDFF86CA2986A64231A
:1088C000323090FBF3F000B207F026FD032007F0F2
:1088D00033FD884B1B7813F0010F00F080810DF001
:1088E00089FD854B85498046D8680EF0D3FC0EF093
:1088F000D3FE80B2B8F1000F04D13B6813F0100F23
:1089000018BF002000B207F007FD9AF80530002BD1
:1089100059D07B4B93F800B0BBF1000F53D04FF010
:108920006408784A06201188019308FB01B14FEAD8
:108930004B08B1FBF8F1B4F80C8000924FEA08182C
:108940001FFA88F848EA01281FFA88F8C1F30321C2
:1089500048EA010807F0F0FC0FFA88F007F0DCFCA9
:10896000A189009A013189B291FBFBF0B2F8008035
:10897000654A0BFB101B517AA4F80CB00129019B2E
:1089800040F03381392007F0D7FC0FFA88F007F068
:10899000C3FC282007F0D0FC0A23DFF89081D8F828
:1089A000000090FBF3F000B207F0B6FC042007F0E3
:1089B000C3FCBAF80830002B00F0408102F07EF8CA
:1089C00000B207F0A9FC03A9504807F07BFC132074
:1089D00007F0B2FCBDF90C0007F09EFC1B2007F06D
:1089E000ABFCBDF90E0007F097FC232007F0A4FCB8
:1089F0004E2007F091FC03A9444807F063FC1220C5
:108A000007F09AFCBDF90C0007F086FC1A2007F06D
:108A100093FCBDF90E0007F07FFC222007F08CFCD0
:108A2000452007F079FC07F081FC2379282B23D11E
:108A3000002317202371346807F07EFC4EF6602077
:108A40004FF03C08B4FBF0F3B3FBF8F008FB103038
:108A5000000200B207F060FC182007F06DFC4FF434
:108A60007A70B4FBF0F4B4FBF8F008FB104000B2ED
:108A700007F052FC07F05AFC254B1B78002B00F046
:108A80009780184C234A2369A9EB030393427CD9AE
:108A90000022214B9A701A711A4A1288D1B2120A16
:108AA0009977DA7719755A7531686269891A164AA1
:108AB000D07A4FF47A724243914239D3326862617C
:108AC000164A1278013A012A9FBF10229A70022298
:108AD0001A712DE0902900208C2100200C2200200A
:108AE000982200206014002000007A446C2E0020A0
:108AF000282100202C2B002034220020CDCC4C3EFD
:108B0000322200201E22002024220020809698007D
:108B10008A2200203F0D03004C0F0020812B0020F3
:108B200058200020A4100020862B00201C210020AB
:108B30000A20834AC4F810901168926891FBF0F102
:108B400092FBF0F2642083F82020121283F8212097
:108B50007C4A19771268091292FBF0F202F5FA7258
:108B600092B29A76120ADA76A268597702F1300147
:108B700083F8221002F5EA4192FBF0F2303109123B
:108B8000783283F8231083F8242094F818B0BBF1CE
:108B9000000F00F07583236A53B1237E002B7AD037
:108BA00040F6B732A36AA9EB0303934200F2A28016
:108BB00033680093644B1B78002B00F00681634CF4
:108BC0002368002B00F00181614B1B78013B012BD6
:108BD00000F2FB80DFF88C81DFF88491D8E0052378
:108BE000BAF80800B0FBF3F08CE66E2000FB08F04A
:108BF0004FF01508527B90FBF8F022B193F80080FB
:108C000080B290FBF8F01FFA80FB3A2007F094FB4B
:108C10006423BBFBF3F80FFA88F0009307F07CFBAA
:108C20003B2007F089FB009B03FB18B04FF00A08BC
:108C300080B2053090FBF8F000B2A8E6D8F8080042
:108C400080F31000BCE698F8003023B1C4F81C9003
:108C500088F800B09FE7E369A9EB0303B3F57A6FE7
:108C600099D30123DAF8000088F8003001F056FCAF
:108C70008046DAF8000001F051FC18F07F0F8AD12D
:108C80008E2888D1237E002B85D1324B23622D2361
:108C900084F824307FE7012284F82C302E4B227692
:108CA0001B689B781E3B93422C4B1ED918680221EF
:108CB000043007F0C5FA94F82420DFF8A0E0013A68
:108CC000D2B284F8242094F82C1094F82D30D2B924
:108CD0004A1C013384F82C2084F82D30DEF8000083
:108CE00001F022FCC4F8289062E70221186801F024
:108CF0000FFCE0E794F82430002BDCD123622376CC
:108D000007F0CAFAD7E7206A013310F801CB84F8DC
:108D10002D300CEB010284F82C2020626146DDE747
:108D2000206801F0FBFB83B27E2B32681CD100234C
:108D300089F82E3089F82F3088F8013028E000BFFC
:108D40001C210020A41000208C22002014220020CE
:108D5000942200204C0F0020502200204C220020A2
:108D6000601400200C00002098F8011081B999F8D7
:108D70002E20002A40F0D6801B2B40F0C9802068AE
:108D800001F0CFFB002840F0EF80012389F82F305D
:108D9000206801F0C6FB0028C2D1BC4C94F83D30DD
:108DA0000BB184F83D00DFF814B3DFF81483DFF86B
:108DB000149394F82F3043B13368009A9B1A012B17
:108DC00040F2E180002384F82F30B14B1B78002B58
:108DD00000F09680AF4B1B68002B00F09180AB4FEA
:108DE00036687B6CF31A632B40F28A800A24DFF822
:108DF000D882412007F0E3F9B8F9020090FBF4F0C3
:108E000080B207F0D3F9B8F9000090FBF4F080B21B
:108E100007F0CCF9B8F9040090FBF4F080B207F049
:108E2000C5F907F0ABF997F84830D80745D49A4B05
:108E30001B88D90513D4DA0600F1F0819C0600F1F5
:108E4000EF81580600F1EE81190700F1ED81DA0794
:108E500000F1EC8113F0020F0CBF012503258F4BAD
:108E60001C788F4B04F00104DB780BB144F0020452
:108E7000532007F0A4F98B4B188800EB800000EB1F
:108E80008000800080B207F091F9002007F08EF991
:108E9000FE20854B1B88584340F2FF3390FBF3F0D4
:108EA000C0B207F073F9002007F070F944EA8500BA
:108EB000C0B207F06BF907F061F997F848309BB939
:108EC0004F2007F07CF90BF07BFF0BF079FF0BF0E4
:108ED00077FF012007F05AF9744B187800F0010071
:108EE00007F054F907F04AF90A2197F848307E64F0
:108EF0000133DBB2B3FBF1F201FB123387F84830E8
:108F00006B4B1B78002B40F0B68105B0BDE8F08FAD
:108F10000D2B29D1012189F8303089F82E10A9F8BC
:108F20003A2035E77D2B03D1012389F83C302FE728
:108F300099F83CE0BEF1000F04D080F02000C3B2ED
:108F400089F83C10511CC9B24A44092989F82E10ED
:108F500082F830300AD1B9F83A20C2F1FF029342C8
:108F600002D1012389F83D300123E5E608293FF6C7
:108F70000FAFB9F83A00034403EB132303F0FF03E8
:108F8000A9F83A3004E794F83E303BF8130018B9DA
:108F900084F83E004FF4036094F83E30B0F5826FE1
:108FA00003F1010384F83E3000F0E1805BD8B0F5B6
:108FB000007F00F0B6800ED8B0F5807F00F0BC8056
:108FC000B0F5887F7FF4F5AED8F800305A077FF50A
:108FD000F0AEA1689DE0B0F5047F00F08580B0F5AB
:108FE000806F7FF4E6AE94F83F3042F210710133A7
:108FF000DBB2032B88BF012384F83F3094F83F3065
:1090000059432C4B1B88002B40F0AF800131234B80
:109010001B78DB07204B48BF04311B88D80748BFAB
:109020000A319A0748BF1431180648BF2831DA05BB
:1090300048BF2831580748BF64311A0748BFC831B4
:10904000980548BF01F5C8719A0648BF01F57A71C5
:10905000D80648BF01F5FA615A0648BF01F57A61A2
:109060004FF4806055E0B0F5E26F7BD02ED8B0F5BC
:10907000C06F69D0B0F5E06F7FF49BAE0E4A916B84
:1090800064234B43918A93FBF1F142E0601400208A
:10909000A0220020482200207E2B00202C2B002024
:1090A000982B00201E2200207C2B00204915002038
:1090B000A3220020BC2B0020242000201AAD010890
:1090C00084210020242200206C2E0020B0F5046FA3
:1090D00042D0B0F5116F00F09280B0F5E46F7FF4EC
:1090E00068AE724A116CCBE7714B5B79002B3FF491
:1090F00060AE704B197800293FF45BAE99F80D30E3
:109100006D4A63B1138893FBF1F30A214FF40470A5
:10911000594307F06BF8002384F82F3049E6138891
:10912000F3E7634B9B79002B3FF443AE634B196825
:109130000A2391FBF3F1ECE7D8F8003059077FF5EB
:1091400038AE5F4B1968E4E7594B9B79002B3FF42D
:1091500030AE5A4B9968DCE70A215A4BB3F9043018
:109160005943D6E7514AD16B8AE702314FE7D8F825
:10917000001011F0200A7FF41CAE3A68130605D5E2
:10918000514607F033F884F82FA012E699F80C3016
:10919000002B3FF40EAE94F84030032B2DD8DFE8BF
:1091A00003F002181F26484A1268107892F803E06C
:1091B0009179090401EB0E21014401EB03610133B4
:1091C000DBB2042B08BF00234FF4826084F84030E8
:1091D0009FE73D4A1268507892F804E0D179E8E7B9
:1091E000394A1268907892F805E0117AE1E7374A37
:1091F0001268507992F806E0F0E70021DDE72C4B89
:109200005B79002B3FF4D5AD2A4B197800293FF448
:10921000D0AD294B1A880A23534334E70D251EE6A7
:1092200009251CE604251AE6082518E6022516E697
:10923000306801F073F9264C804623783BB1013B3E
:109240002370306801F06DF90028F1D15DE6294600
:109250000322681E11F0C3FA0421681E87F84C80AF
:1092600006F00DFF0028ECD0681E06F023FF2378DF
:1092700018442070E5E7174F174E07F14A05E0E75D
:10928000DFF858A0DAF8000001F04BF9C0B201286D
:109290007FF681AC0228DFF848803FF4D4AC06F0BA
:1092A000EDFF012388F8003075E400BF2420002082
:1092B000862B0020322200201E2200201C210020AC
:1092C000A41000206C2E00209C2000203C3C00209C
:1092D000AC22002060140020A82200204C22002094
:1092E0000C00002070B50124B0FBF4F58D4202D2D1
:1092F0001CB91C7070BD4C43F6E7B0FBF4F6092EA8
:109300000BDD002A14BF37255725354404FB160012
:1093100003F8015BB4FBF1F4EAE73025F5E70368F5
:109320005A1C026019707047002B2DE9F041064667
:109330000F46144614BF4FF030084FF02008069B2C
:1093400013F8012B3AB92546002D0FDC24EAE4740A
:1093500004E0013CF4E7002CFBDC0024069D641BC8
:10936000281915F8011B31B9BDE8F0814146304696
:10937000B847013DE8E73046B847F1E770B5044625
:10938000A56808462B1D013544F82310E168A56047
:109390000DF078FE6668E060B54204BF0023A3606C
:1093A000A368043354F823100DF06AFE0546E0600C
:1093B0002068864207DB30460DF018FF014628463C
:1093C0000EF01CF870BD013020600DF00FFF01465B
:1093D00028460EF013F84FF07E510DF053FE70BD8D
:1093E000F8B50E460446016830460DF053FF61693A
:1093F0000DF048FE6168054630460DF04BFFA1694F
:109400000DF040FEE168074628460DF043FF014697
:1094100038460DF035FEA168606130460DF03AFF28
:109420002169064628460DF035FF014630460DF00D
:1094300027FEA0612846F8BD38B5044625680846D1
:1094400029460DF01DFE61680DF024FF29460DF040
:1094500019FE206038BD0846704700232A220360A9
:1094600042702B22C270012243604271C371704767
:10947000014B186801F058B828100020064B98429C
:1094800009BF064A4FF0FF30538B013301BF9BB237
:109490005383508B80B2704700380040E4150020A1
:1094A0002DE9F74F254CDFF89CB054F8033C0193AD
:1094B000002B3BD0242327464FF0000814F9075C0B
:1094C0001A4603FB05B60021304611F0A2F90BEB5A
:1094D000050292F8489092F84AA017F8010F484503
:1094E00003D1484601F050F8B060F878504503D1F8
:1094F000504601F049F8F06008F10108B8F1030F97
:10950000EBD1242303FB05F10BEB0102906868B15A
:10951000D06858B15D44E01F4BF8010095F84C103D
:10952000019B117495F84E1053605174044B143420
:109530009C42BAD103B0BDE8F08F00BF43AD010833
:109540006BAD0108B014002010B5427A044632B168
:10955000036800F10A01406898470023637210BD58
:109560002DE9F341056906460F46002D3BD1D0F8A1
:109570000080C8F3090373B300234FF40050D6F8FA
:10958000008001930BF076FD042821D12A4C4FF482
:109590000050236943F001032361BBB2A8F80030F7
:1095A0000BF068FD04283CD108F102030193019BF4
:1095B0003F0C1F804FF400500BF05CFD2369042822
:1095C00023F001034FEAC3434FEAD34323612FD073
:1095D0006FF0010507E04FF430200BF04BFD04283D
:1095E00005D04FF0FF35284602B0BDE8F081124C9F
:1095F0004FF43020236943F002032361C4F8148040
:10960000236943F0400323610BF034FD23690428F0
:1096100023F002034FEAC3434FEAD3432361ABD0A5
:10962000DFE7236923F00103DB04DB0C2361CFE7D1
:10963000336804333360D6E700200240F8B50446AF
:109640000D4600278E18B54201D12069F8BDE368A8
:10965000591CE16015F8012B234404291A72F2D138
:10966000A1682046FFF77CFFE7602061EBE770B55B
:109670000D46064644880021C4F30B0422462846C2
:1096800011F0C7F833690A4A934209D3094A934251
:1096900006D222462846BDE8704019460EF088BC26
:1096A00023B121462846BDE87040184770BD00BF71
:1096B00038EF0108E0EF0108064B07498B4202D35F
:1096C0000023184670471A88C2F30B029042F8D064
:1096D0001433F3E778EB010838EF0108024A136806
:1096E00023EA000010607047C82000202DE9F843ED
:1096F00002780346202A00F10100F9D0092AF7D0A8
:109700002D2A4BD10346444D1C460026DFF80C8120
:10971000234614F8012BA2F13007F9B2092943D9E5
:109720002E2A09D127463D4CA0463B4617F8010B8F
:109730003038C2B2092A44D91A7802F0DF02452A29
:1097400063D15A782D2A4CD10127023300240A20F4
:10975000013B13F8012F303AD1B2092947D9B4F5AA
:109760009A7F28BF4FF49A744FF07E50A046DFF8DE
:10977000B090B8F1070F3DD8DFF8A08004F00704DF
:10978000002C3DD1002F42D0014630460DF036FE70
:10979000014628460DF07EFDBDE8F8832B2A08BF60
:1097A00003464FF07E55AFE7414630460DF072FD5F
:1097B000064638460DF01AFD31460DF063FC0646AC
:1097C000A6E70DF013FD21460DF018FE01463046C8
:1097D0000DF058FC4146064620460DF05BFD044660
:1097E000A3E72B2A14BF013302330027AEE700FBA7
:1097F0000424AEE749460DF04DFDA8F10808B8E78E
:1098000041460DF047FD013CBAE74FF07E5001465E
:1098100030460DF03FFDBBE7000080BF0000204157
:1098200020BCBE4C002330B50C4687B00021054655
:109830000093019302930DF0E9FE294900283DD0E1
:1098400028460DF01FFC27490DF024FD0DF0FEFE0B
:10985000054680EAE07003A9A0EBE5700BF064FA1E
:10986000002DACBF20232D2303A88DF800300CF071
:109870004DFF012826D130238DF801308DF80230BC
:109880008DF8033003A9684610F0E9FF68460CF034
:109890003DFF0338C5B22A466946204611F035F827
:1098A000002311496355204610F0D9FF0DEB050147
:1098B000204610F0D4FF204607B030BD28460DF0FA
:1098C000DFFBC0E7022805D130238DF801308DF889
:1098D0000230D7E7032804BF30238DF80130D1E7E9
:1098E0006F12033A00007A4476C9010870B5064643
:1098F000B6FBF2F40846154614B12046FFF7F6FF12
:1099000005FB1464024B1B5D00F8013B70BD00BFFA
:10991000D7C80108026810B51146531C036011F83E
:10992000024BD31C01605178036093781B0443EA17
:109930000123111D0160D078234343EA006010BD6C
:1099400003685A1C02601A4612F8021B026058781B
:1099500041EA0020704703685A1C0260187870477B
:1099600038B50446154600680EF022FB22682A44EA
:10997000226038BD03685A1C0260197003685A1CC3
:1099800002600A0A1A7003685A1C02600A0C1A70F4
:109990000368090E5A1C02601970704703685A1C4C
:1099A000026019700368090A5A1C02601970704736
:1099B0002DE9F04F82468B4615461C46002789B09C
:1099C0000DF114082978002930D0252904D05046FB
:1099D0000135D8470137F5E76A784FF00009302A9A
:1099E00012BF00230123AA780293A2F1300314BF0F
:1099F000AE1CEE1C092B0CD8A2F13003D9B20929F8
:109A000018D9A2F16103052B1AD8A2F157030A2B2A
:109A100010DD6C2A74D13278751C642A00F0AB809A
:109A200022D8252A66D012D8002ACBD1384609B0D0
:109A3000BDE8F08F0A2202FB093916F8012BDBE79B
:109A4000A2F14103052BE4D8A2F13703DFE7582A3E
:109A500018D0632AB6D12E4621785046D847251D06
:109A600001372C463546ADE7732A37D006D86E2A23
:109A7000A8D12E46236804341F60F3E7752A65D009
:109A8000782A9FD143461021A2F15800424204F1A6
:109A900004064241206807E02D2340428DF814302F
:109AA0000DF1150300220A21FFF71CFC3446CDF806
:109AB0000080029B4A4659465046FFF735FC074452
:109AC00080E72D2340428DF814300DF1150300225C
:109AD0000A21FFF707FC3546039CE8E72E4623687A
:109AE0004A460093594600235046FFF71DFC251DAA
:109AF0000744B6E72E4625215046D8470137B1E73F
:109B0000642A31D00AD8252AF5D002D8002A8DD06F
:109B1000A8E7582A0CD0632A9ED0A3E7732ADED088
:109B200002D86E2AA6D09DE7752A14D0782A99D13A
:109B3000A2F158014A4204F104054A412068434613
:109B400010212C46FFF7CEFB3546B0E7261D4346D5
:109B500000220A219EE7231D0393002243460A2187
:109B60002068FFF7BFFBB6E72068231D002803939A
:109B7000A7DB4346ABE72068261D00288CDB434665
:109B800090E70FB437B50B4906AB0B4853F8042BDD
:109B9000096800680193FFF70BFF0446074D28682A
:109BA00000F0B9FC0028FAD0204603B0BDE83040F0
:109BB00004B07047B80A0020BC0A0020281000201A
:109BC00080EAE073A3EBE0738B4206DB002801DD43
:109BD000401A704702D0084470470020704770B5A3
:109BE00004460DF033FD203040284DD8274D284E37
:109BF000294620460DF00AFD002830D1254D244E7F
:109C0000294620460DF0E4FC00282ED122492046AA
:109C10000DF0FCFC00282ED021461C480DF030FA37
:109C20000446214620460DF035FB05461B490DF044
:109C300031FB1B490DF026FA29460DF02BFB194983
:109C40000DF01EFA2946064620460DF023FB01467C
:109C500030460DF01FFB21460DF014FA70BD204672
:109C600031460DF00DFA0446C2E7204631460DF0AC
:109C700009FA0446C4E70C4920460DF0A9FC002867
:109C8000CFD021460348C9E7002070BDDB0F494013
:109C9000DB0FC940DB0F49C0DB0FC93F92E741B979
:109CA0009730083C15A82A3EDB0FC9BF10B5142217
:109CB0000021044610F0ADFD0123636010BD2DE9C5
:109CC000F74F054610461F4688460DF08BFA4B4964
:109CD000044640460DF0DEFA014620460DF0DAFA61
:109CE00080460EF005FB044640460EF081FA3946E8
:109CF000834638460DF0C6F9014620460DF07EFB3E
:109D00009DF830600746012E4FF0000449D008D37B
:109D1000022E5DD02346A3462646A046A146A24673
:109D20001DE059464FF07E500DF0AAF94FF07C51DE
:109D300081460DF0AFFA4FF07E51824638460DF065
:109D4000A1F94FF04041064658460DF0A3FA3946B6
:109D500083464FF07E500DF093F9D04603463146CE
:109D6000504601930DF04AFB3146286048460DF0FD
:109D700045FB3146686040460DF040FB3146A86027
:109D800058460DF03BFB019BE860314618460DF04C
:109D900035FBAC6128616C612C62EC6103B0BDE8FD
:109DA000F08F4FF0404158460DF074FA4FF07E515D
:109DB000814638460DF066F9394606464FF07E502A
:109DC0000DF05EF94FF07E580346CB46C246C6E71B
:109DD0004FF07E5100F100480DF054F94FF0404132
:109DE000064658460DF056FA394683464FF07E50E7
:109DF0000DF046F9BA460346A146B0E727D4D2365D
:109E0000002307B50093034BFFF759FF03B05DF83C
:109E100004FB00BFF304353F70B50D460DF0E2F9C9
:109E2000044628460DF0DEF9014620460DF0E6FA1C
:109E30000EF01AFA01460DF025F94FF08044054660
:109E4000014620460EF05AFB4FF07C51064628464C
:109E50000DF020FA014620460EF050FB4FF07E51E7
:109E6000044630460DF00CF9014620460DF0C6FAC6
:109E700070BD10B541F221040A44914200D110BDD9
:109E800011F8013B80EA0320082310F4004F4FEA49
:109E9000400018BF6040013B80B2F6D1EDE7F8B555
:109EA000174D2B78A32B28D16B78BE2B25D10222FE
:109EB00029464FF6FF70FFF7DCFF124FAC1C2288DB
:109EC0004AB1A618BE4218D2052A16D92146FFF774
:109ED000D0FF3446F3E721460222FFF7CAFF0222F1
:109EE000A118FFF7C6FF0634074B641B1C8041F620
:109EF0000F53C31A58425841F8BD0020F8BD00BFA7
:109F000000F80108000002082A1C002001234A0969
:109F100001F01F0103FA01F150F822300B4340F821
:109F20002230704701234A0901F01F0103FA01F1B1
:109F300050F82230194214BF01200020704700223F
:109F40000120094B1978094B01299DBF5A7098705F
:109F5000074B9A7094BF1A70587001299EBF2C222B
:109F6000044B1A71704700BFC40A00201A0C00206D
:109F7000880F0020B620002030B50B4C0B4D227806
:109F80002B7885B09A420CD002A9684608F016FDDD
:109F90000123022202A9684608F074FD00232B70F9
:109FA000237005B030BD00BFE5330020E43300204E
:109FB000094A0A4913781844C0B210F0800F18BF3C
:109FC00080381070107813460A78904202BF002241
:109FD0000A701A70704700BFE5330020E433002098
:109FE00030B50E4D0E4C2A78237885B09A4212D0A7
:109FF00002A9684608F0E2FC0023022202A9684692
:10A0000008F040FDFFF7D4FF28782378C31A5842A0
:10A01000584105B030BD0120FBE700BFE53300200B
:10A02000E43300201FB502A8694608F0C7FC044BC2
:10A0300000981B681844019B184405B05DF804FBA8
:10A04000E033002010B5046B0346C168406944B199
:10A050001A6C8C1A013A08BF0A46005D1A64C0B235
:10A0600010BD1A6A805C01328A4228BF2246C0B203
:10A070001A6210BD436B13B190F850007047836AA9
:10A08000406A1B1A584258417047416A836A026904
:10A09000994238BF8918CB1A416B21B149680B44EA
:10A0A000511E8B4202D2501EC01A704700207047CA
:10A0B000036B4BB1026C5B689342A3EB02032EBFB0
:10A0C0001846C068C0187047C269036A9A422FBF19
:10A0D000D01AC0688018C01A70470A4B30B503F117
:10A0E000100493F900205D78072AC8BF143A81183C
:10A0F0000D739D780433855413F8012CA3420A761E
:10A10000EFD130BD64AD01082323037024234370D5
:10A1100000238370C37070472D2343702E23C370B8
:10A120002F23437170472DE9F04101270B4DDFF8D4
:10A1300030802C686A6914400CB9BDE8F081B4FA2B
:10A1400084F3C3F11F0358F8230007FA03F60368EA
:10A15000984724EA06046E61EEE700BF0004014060
:10A16000D80A00204171FCF727B98160FCF724B9B7
:10A170002DE9F047064689464FF000474FF00008AA
:10A18000038A8589ADB21D400DB9BDE8F087B5FAE7
:10A1900085F327FA03F2D2431B3B91B2318215407B
:10A1A000042BF1D8DFE803F02925211A0300D9F8A0
:10A1B000244084B1013CA4B2C9F82480D9F820A07D
:10A1C000BAF1000FE0D0DAF8003050462146984747
:10A1D000DAF804A0F4E7B48DA4B2EFE7D9F80000F0
:10A1E000B18E036889B29847CEE7D9F80400318F61
:10A1F000F7E7D9F80800B18FF3E7D9F80C00B6F803
:10A200004010EEE71FB50023ADF80A30ADF8063078
:10A210008DF80C30074B01391B68ADF80810B3FB03
:10A22000F2F204A9013A21F80C2D0AF00AFC05B05B
:10A230005DF804FB2000002073B504460068FFF7BA
:10A24000E1FF2268174913889BB243F00103138092
:10A25000002351F8334001EBC300A2421DD14579E0
:10A260000124002601A88DF804508DF805408DF8D2
:10A2700006608DF807400AF099FB1B2D0BD11923BE
:10A2800001A88DF804308DF805408DF806608DF832
:10A2900007400AF08BFB02B070BD0133042BD8D10C
:10A2A0000025DDE784A901080B4B800A98420FD0F6
:10A2B00004D8B0F5801F09D0FE207047074B9842A4
:10A2C00008D049339842F7D10020704701207047E9
:10A2D00002207047032070470100100002001000A8
:10A2E000F8B5046805462046FFF7DEFF032841D88D
:10A2F0006B794FEA930E39B975460227A689AF40AC
:10A30000B6B226EA0706A6810A2505FB00E51D4E22
:10A3100046F82510043546F82520324631B1990813
:10A320000223A5898B402B439BB2A381282343435F
:10A3300003F120011144EFF31286502585F31288B2
:10A340000425103313441F6817B10F6019680431D6
:10A35000013D03F10403F6D10D60F3B283F31188DC
:10A36000282303FB0020036A2BB1A3899BB243F08F
:10A370000103A381F8BDA38923F001031B041B0C77
:10A38000F7E700BFAC3A00201E4B30B55B681E4AB1
:10A39000C3F308039BB9EFF3128383B91B49106819
:10A3A0008C6800BF13689842F9D14FF47A72184B49
:10A3B000196802FB01F31B1BB3FBF1F31EE0EFF383
:10A3C0001281102383F31288104CA568236813F4BC
:10A3D000803F18BF01200F4B1CBF1860A568146890
:10A3E0001868CAB282F311884FF47A72084B20447D
:10A3F000196802FB01F35B1BB3FBF1F302FB0030B6
:10A4000030BD00BF00ED00E09822002010E000E029
:10A41000C00A00200815002038B50446FFF7B4FF35
:10A420000546FFF7B1FF401BA042FAD338BD10B577
:10A43000044604B910BD4FF47A70FFF7EDFF013CFC
:10A44000F7E7EFF31283102282F312880649DBB29A
:10A450000A6801320A600021044A1160044A126845
:10A4600083F31188704700BF982200200815002050
:10A4700010E000E0014B5868FBF76CBF200B002098
:10A48000014B1868FBF766BF200B002070B5EFF397
:10A490001282502383F31288436BD2B2196811F0F1
:10A4A000010F08D15E68DEB9446A816A8C4205D129
:10A4B000012380F8503082F3118870BD856998BF00
:10A4C00004690D448CBF611A611ADD608CBF59604C
:10A4D00059604FF000018CBF8462866280F8501092
:10A4E000196841F001011960E5E7436A8269D154B6
:10A4F000436A02690133934228BF00234362436BDE
:10A5000003B1C3E7C26CD36843F08003D3607047E4
:10A5100003689B69184703685B6918470368DB6831
:10A52000184703685B68184703681B681847036887
:10A530002DE9F041DB6904460E46174693B90D46F6
:10A540007B1B3344002B01DCBDE8F08123682046EF
:10A550009B6898470028F9D015F8011B2046FFF7A3
:10A56000E3FFEDE7BDE8F0411847E0E7054B53F89E
:10A57000202032B193881268D1680B4218BF1B04A7
:10A5800013617047CC0A002010B50409013C022C6D
:10A5900000F00F0215D80C4B33F8141041FA02F3F7
:10A5A00013F001000ED001209040013808400DF05A
:10A5B000E3F8064B1C44237C0344054800EBC3002E
:10A5C00010BD002010BD00BF7CA9010864AD0108CA
:10A5D000301C002037B50D460446C8B103680D4A4B
:10A5E00003F14043A3F5843302EB9323D87C0AF0B4
:10A5F000BFF9A38801A9ADF80430206805F0030372
:10A6000005F07C058DF806308DF8075005F0BCFC90
:10A6100003B030BD64AD010810B1036882885A618F
:10A62000704710B1036882881A61704738B10029F9
:10A6300014BF00211021838802688B40136170478A
:10A640000F4B01461B883BB90E4B18680E4B1B780D
:10A650000BB981F00101E9E70C4B5A6972B150B1B5
:10A660000B4A196810880B4A92FBF0F292B20A80EA
:10A6700001225A7470471A6810805874704700BFDE
:10A68000200C0020240C0020280C00202C0C002082
:10A69000440C002020A107000123084A83401278BF
:10A6A0001340074A52F8200019B1191C18BF0121A4
:10A6B000BCE7B3FA83F14909FAE700BFC60A0020F4
:10A6C000CC0A002038B50D46012104460846FFF7A4
:10A6D000E3FF00210846FFF7DFFF04B938BD012082
:10A6E000FFF744FF0020FFF741FF0120FFF7A8FF1D
:10A6F0002846FFF79CFE0120FFF738FF0020FFF7F8
:10A7000035FF0020FFF79CFF013C2846FFF78FFE36
:10A71000E4B2E2E738B50D460130C4B205B938BD40
:10A7200005203221FFF7CEFF4FF4FA70FFF77FFECE
:10A730001CB1FA212046FFF7C5FF4FF47A70FFF7EE
:10A7400076FE013DEAE708B50A21FFF7E3FF034A79
:10A75000034B1A60034A044BDA6008BDEFBEADDE5E
:10A76000F04F00200400FA0500ED00E0DBE4DAE43D
:10A77000D9E4D8E4D7E4D6E4D5E4038823F0400351
:10A780001B041B0C0380038823F038031B041B0CE1
:10A7900059B141F4807191FAA1F20029B2FA82F222
:10A7A00008BF4FF0FF32511EC900194389B2018022
:10A7B00003889BB243F0400303807047F8B5848957
:10A7C0004FF6FF764FF47A740BB90120F8BD91B1C2
:10A7D0000D7801310789BF070FD54FF47A74ADB2F8
:10A7E00085810589ED0712D58589ADB20AB115704D
:10A7F0000132013BE8E7FF25ECE7013CA4B2B4429B
:10A80000E8D1FEF73BFE003018BF0120F8BD013C47
:10A81000A4B2B442E5D1F4E708B540F2E9330289C5
:10A82000920708D540F2E93389B281810289D207C3
:10A8300009D5808905E0013B9BB2002BEFD1FEF7E3
:10A840001DFEC0B208BD013B9BB2002BEED1F6E766
:10A8500070B50446806815461E46FFF7DDFE606849
:10A8600041F08001FFF7D8FF33462A460021606897
:10A87000FFF7A4FFA068FFF7D4FE012070BD38B534
:10A88000044615468068FFF7C7FE6068FFF7C4FFFF
:10A8900029466068FFF7C0FFA068FFF7C2FE0120ED
:10A8A00038BD00BF024B1A889B78028083707047C6
:10A8B00080AD0108064A116849B1642350684343DA
:10A8C000B3FBF1F303490B8000231360536070471F
:10A8D0000C1500202C1C002070472DE9F843304B4C
:10A8E00006461B782BB92F4A136053609360BDE86E
:10A8F000F8832D4B9F6898602C4B9B79012B09D0D6
:10A9000001D3042B04D90022264B1A605A609A60A6
:10A91000BDE8F88340F6E4494FF47A74244BDFF83D
:10A92000A480DA79234B244D33F81200B8F90230B1
:10A9300080B209FB00F2C3EB12336343B8F9002085
:10A9400093FBF2F3EB600CF04DFC01461B48FEF765
:10A9500047FD0CF0A1FE80B209FB00F9B8F9020036
:10A96000B8F90030C0EB193904FB09F494FBF3F497
:10A97000D5F80C80F01BAC6008FB00F00CF036FC46
:10A980000F490CF087FC69680CF07CFB68600CF0E8
:10A990005DFE044B286083E810019860BDE8F883F1
:10A9A000322200201C2100200C150020862B0020C4
:10A9B000600C0020740C0020BC0F0020CC0F002085
:10A9C0002FE33E31702000202DE9F843224B234D28
:10A9D0005B79012B3BD1224B224E9A78224B33F8E4
:10A9E0001240A4B220460CF0FDFB01463046FEF7B3
:10A9F000F7FC1E4B9F7893F8009093F801800CF0C1
:10AA00004BFE44F6FB7209EB491983B209FB0323A1
:10AA100009FB0424C8EB0838B3FBF8F3B4FBF8F4E3
:10AA2000B3FBF7F3B4FBF7F49BB2A4B226F8043CF3
:10AA300026F8024C2B806C800D4B1B78022B04D126
:10AA40000C4B6A881A802A885A80BDE8F883002354
:10AA50002B806B80F0E700BF862B00201E22002099
:10AA6000600C0020940F0020740C00206C2000204B
:10AA700080210020F4200020F8B524220021044683
:10AA80000FF0C7FE002223460521042510460A4F79
:10AA9000D65D0132042A9E70D9701D71987159716A
:10AAA00003F10803F4D101232380522384F82230D8
:10AAB00064232384F8BD00BFDCA9010838B5194B15
:10AAC000187808B318490C89FCB120460CF08AFBB1
:10AAD000164B054698680CF089FB014628460CF099
:10AAE000CFFA13490CF0D6FB054620460CF07EFB4E
:10AAF000014628460CF082FC0CF0A8FD6428A8BF93
:10AB0000642020EAE070C0B238BD0A4B4D781B8843
:10AB10000A7800FB15346423521B63435043B3FB94
:10AB2000F0F0EBE732220020862B00201C210020D1
:10AB30000000C8421E220020194B2DE9F0411C687C
:10AB400007460E2C984607DC0023164A9C4206DC7A
:10AB50000025144EA54208DD0020BDE8F08152F822
:10AB600023108F42F8D00133F0E756F82530681CE7
:10AB70007BB98000621B011F9200314430440134D4
:10AB80000FF02DFE46F82570C8F800400120BDE802
:10AB9000F0811A7D3B7D9A42EBD30546DAE700BF90
:10ABA000D81B0020DC1B00201028F8B50FD00E2881
:10ABB0000CD83422124B02FB003009B1C3684BB9E8
:10ABC0000022104D10492C68A24206DBF8BD0F4B45
:10ABD0001868F2E7BDE8F840AEE751F8227093003C
:10ABE000B84203EB010609D1A21A043392001944BA
:10ABF0003046013C0FF0F3FD2C60F8BD0132E3E775
:10AC0000FC000020D81B0020DC1B0020F0220020CC
:10AC100008B50C4B197801290CD00AD302290DD0A4
:10AC2000FFF7B2FB084B00F5F42000F590701860B8
:10AC300008BD00210020FFF72FFDF1E70020FFF7FE
:10AC400095FCEDE70A2300200C23002010B50446F4
:10AC50002046FFF760FC00B110BD0A20FFF7E7FBBC
:10AC6000F6E70022F0B51446FF270949094E0B7894
:10AC7000951995F906E00832864501BF03F1FF33C7
:10AC8000AF71DBB20124202AF2D104B10B70F0BD08
:10AC90002C0B00203C370020002310B5084A52F846
:10ACA000331002EBC304884203D00133042BF6D1E6
:10ACB00010BD0021C162A18042F8331010BD00BF59
:10ACC0003C370020F8B505460024094EA359A719C2
:10ACD000AB4207D12846FFF7DFFFCC2200213846E0
:10ACE0000FF097FDCC34B4F5197FEFD1F8BD00BF5C
:10ACF000940C00202DE9F04F07464FF0000893B068
:10AD000003929DF870909DF874A02B4A05910293D0
:10AD100002EBC80393F90610B9424FD008F10108BD
:10AD2000B8F1040FF4D100207EE11F2FFBD1CDF844
:10AD300000A04B46029A0399012039E00135072D06
:10AD400068D100256DE00132072A40F0838000229F
:10AD500088E0049B53B1711CC9B220B14FF00B0EB7
:10AD6000C17180F806E01A21FFF734FC19F0010FD9
:10AD700000F0BE800136F6B215B10C21EE71A9715A
:10AD80004A212846B2E04FF6DF72E36C1A80DA6897
:10AD900042F02002DA6007E1E26CD36843F08003FE
:10ADA000D36030E14B462846029A0399CDF800A0C3
:10ADB00006F062FC2EE100BF3C3700209D88002D8C
:10ADC000B1D11E2FEED0B0DC012FACD8984BFEB223
:10ADD00053F82740002C00F01C81964BD4F854B057
:10ADE0002360029BDBF80420A36004F15A03636133
:10ADF00004F5AD73A3614FF48073E264E3602361F3
:10AE00009BF8160009F0B4FDDBF80C20CAB18A49A2
:10AE10001C208C4600FB051EDEF804309A428DD1C2
:10AE2000EDB21C2101FB05C5844B2969586901431A
:10AE300059610C212976711C69762263E26C043217
:10AE4000A264DBF80810002935D07B4800224FF0BF
:10AE50001C0E05460EFB020CDCF8043099427FF410
:10AE600072AFD2B21C2101FB0255744A29695069A4
:10AE7000084350610B202876701C687653699BF854
:10AE80001900194351616E4A8009AA606A7B8DF8E6
:10AE90001D008DF81C2000228DF81E2001226C61FF
:10AEA00007A88DF81F2009F081FDDBF808206263F8
:10AEB000E26C0432626494F85800FFF765FB0546C3
:10AEC00094F85900FFF760FB09F002031AF0080F2D
:10AED00004933FF43EAF0136F6B210B10B22C671B7
:10AEE00082711AF0100F14BF1A211E21FFF772FB96
:10AEF000DBF80C2012B1DBF808208AB99BF8182087
:10AF000007A88DF81C209BF81A309B098DF81D307E
:10AF100000238DF81E3001238DF81F3009F046FD07
:10AF20000123002684F85030039B2662E362029BD3
:10AF3000E661A662666284F80590A36084F806A0C4
:10AF40002046FBF739FA19F0010F2DD0236B002BA7
:10AF50003FF419AF07A809F09BFFA36C206B079380
:10AF60004FF48053109380230C93E36811960A9357
:10AF700020230F9363690B9608930D960E960996FE
:10AF800009F0B1FF07A9206B09F08FFF226BE16C7C
:10AF9000136843F0010313608B8A9BB243F04003B4
:10AFA0008B8253689BB22364049B002B2BD0636B72
:10AFB000002B3FF4F1AE07A809F06AFF636C00258F
:10AFC00007934FF48053109380230C932369606B95
:10AFD0000A931023119509930B950D950E950F95D6
:10AFE00009F081FF07A9606B09F05FFF636B1A68C6
:10AFF00042F002021A60E26C5D605D60938A9BB26F
:10B0000043F080039382E26C93899BB243F4005334
:10B010009381204640B10B4BBDF8141003EBC802DE
:10B020000771918043F8380013B0BDE8F08F00BF7E
:10B03000200B002084AD01082400002000100240F5
:10B04000FD6100083C37002038B1038813EA010095
:10B0500003D08B420CBF0120022070470023F0B5C3
:10B060001D460D490D4E0B73DAB2032A03D905B103
:10B070000A730020F0BD5F1C06EBC30436F83330C2
:10B0800001321842D2B24FF0010502D00A732046B5
:10B09000F0BD3B46E8E700BF0C1500201637002046
:10B0A0002DE9F74F0120FFF7D9FF0024214D224E53
:10B0B00068B3022C2BD84FF0CC0909FB04F855F8E3
:10B0C000087005EB080A17B10134E4B2F0E7032376
:10B0D000C27890F902000093184B019753F8223080
:10B0E00001213A46FFF706FE834640B14A463946FB
:10B0F000504601340FF08DFBE4B245F808B0002152
:10B10000327B0F4FD3B2032B04D901B1337303B099
:10B11000BDE8F08F02F1010E07EBC20037F83220D4
:10B120000133D207DBB24FF0010101D53373BFE722
:10B130007246E7E7940C00200C150020ECB70108DC
:10B1400016370020142809D80C235843044B185CE8
:10B1500028B10123013803FA00F07047002070473E
:10B1600064B6010810B500240020FFF769FA054B0A
:10B170001C70FFF74DFD044B1C70044B1C619C823E
:10B180009C6110BD0A230020352B00200C150020E7
:10B19000F0B440B1134B1B6813F4003306D0124BCC
:10B1A0001B78032B01D1F0BCDCE700230F4C0C26ED
:10B1B000224606FB03F10F5D0D19874204D00133CF
:10B1C000152BF6D1F0BC7047094B986918B16C7813
:10B1D00040788442F6D20A449A6100229A821A6127
:10B1E000F0E700BF541E0020812B002064B6010848
:10B1F0000C150020F8B506460D200BF0E7F810B14D
:10B200000A20FFF7C5FF294CA269002A4CD0236908
:10B21000B34249D8264BA18A1878576838BB012019
:10B2200018707B5C002B33D01378224A013B1268E4
:10B2300000FA03F3134201D1FFF702FA01221E4B79
:10B240001A70FFF7E5FCA38A43B9A3691B78053B95
:10B25000012B03D8FFF798F8184B1860A369A28A4E
:10B260005B689B5CFE2B0ED10023A382F8BD0025FA
:10B270001D707B5C63B12846FFF7E2F90E4B1D7031
:10B28000FFF7C6FCEAE7FF2B06D1BDE8F84069E707
:10B29000A369A28A5B689B5C42F2107101FB0363A5
:10B2A00001322361A282F8BDF8BD00BF0C15002059
:10B2B000352B0020541E00200A2300202C390020AA
:10B2C0004000402830B4A8BF4020002302251424A9
:10B2D000064A9D5402339918984201F8014CF8D857
:10B2E000FF21D1540E2030BC52E700BFB41F002014
:10B2F000037903F00C03042B05D0082B0FD0BBB946
:10B30000B0F80B0070470B4BB0F80B001B7803EB49
:10B310008302C3EBC20300EB430080B27047054BCE
:10B32000B0F80B005B7803EB430300EB8300F4E71A
:10B3300000207047FC1F002020B10078B0FA80F098
:10B34000400970470120704708B520210FF096FA98
:10B35000034618461BB102780133202AF9D008BDF4
:10B360002DE9F8430D4616468146002440F6340781
:10B370004FF019084846FFF7E7FF814690B10CF0FF
:10B38000EFFDB842A8BF3846B0F5617FB8BF4FF4B3
:10B390006170A0F5617090FBF8F04CB928703378BB
:10B3A000013333700134022CE4D14846BDE8F88300
:10B3B0006870F4E701480AF0C9BF00BFFCC8010883
:10B3C00010B50446B0F80900FEF776F901462046AC
:10B3D000FFF78EFF4B68184410BD38B505460C4684
:10B3E000FFF7EEFF2B7903F00303012B00D001D20E
:10B3F000047038BD048038BD0FB407B504A951F8F6
:10B40000040B01910AF090FF03B05DF804EB04B067
:10B41000704713460A4601460048EDE708C901088F
:10B42000F7B50646FFF788FF054658B1002401A985
:10B43000204609F079FC0134FFF7F2FF122CF6D117
:10B4400003B0F0BD30460CF08BFDC4B2112C5BD8BC
:10B45000701CFFF779FF2F4D0746B8B92E4B13F834
:10B4600014108A1E514251412B4B13F81420AA5C30
:10B47000002944D003EB4403597819234B43274850
:10B4800003F2EE232146FFF7B7FFD9E701782846FC
:10B490000FF0F4F950B1032C8CBF03220022204B93
:10B4A000401BC0B213441E5C032E02D1FFF782FF83
:10B4B000C6E73846FFF748FFF0B1022EF6D10CF090
:10B4C0004FFD40F6CA0280B29042A8BF104640F23B
:10B4D000EE229042B8BF10461922A0F2EE2090FB57
:10B4E000F2F00D4B03EB44035870B31E594259411F
:10B4F000094B03F81460B7E7022EF6D1D6E72146D0
:10B500000848FFF779FF9BE7112229460648FFF715
:10B5100080FF95E760B701082C19002021C90108B8
:10B52000ACAD010831C90108E0DD01080FB413B565
:10B53000084C04AB53F8042B074920680193FEF72D
:10B5400037FA2068FEF700F802B0BDE8104004B0FA
:10B55000704700BF44280020D16201082DE9F04F58
:10B5600085B00346FFF7E8FE064620B1FFF722FF4D
:10B5700005B0BDE8F08F03AA5E4918460CF04CFDFB
:10B5800035460446B0464FF0FF37DFF89491DFF8B8
:10B5900094A1DFF894B1B4B957483946FFF7C6FF14
:10B5A000564B78B203EBC40292F90620824200F0B7
:10B5B00086800134042CF5D1B8F1000F33D1504806
:10B5C0000AF0C4FED4E7012E0ED0022E11D01EB90F
:10B5D00020460CF0C5FC074603AA464900200CF0A3
:10B5E0001BFD01360446D6E720460CF0B9FC804628
:10B5F000F2E7494620460FF09DF920B9414920461F
:10B600000FF098F908B145F00105514620460FF0BA
:10B6100091F928B9594620460FF08CF90028DBD063
:10B6200045F00205D8E7002D08BF03250022EDB242
:10B630000192009543461146FFF75CFB044608B9AA
:10B640003148BDE741463148FFF770FF30480AF006
:10B650007DFE304B1D682846FFF7F8FA2046FFF7BD
:10B66000F5FA00210846FFF717F800210120FFF73F
:10B6700013F82846FEF755FF70B101210020FFF7AF
:10B680000BF82846FEF74AFF01462046FEF74CFF1E
:10B6900000210846FFF700F82046FEF742FF002889
:10B6A000E7D001210020FEF7F7FF2046FEF736FF26
:10B6B00001462846FEF738FF00210846D7E753F831
:10B6C0003440002C3FF478AF13480AF03FFE55B1E8
:10B6D00061798D4207D011482A46FFF727FFE9B26A
:10B6E0002046FEF715FFE36A002BAFD00023E3628C
:10B6F000ACE700BF21CC010844C901083C37002059
:10B700004DC9010810DB010863C9010878C90108A7
:10B71000B9C90108482800208DC901089BC9010842
:10B720003EC9010841C9010855D30108F8B503799C
:10B7300003F03003102B0AD0202B24D043BBBDE8EC
:10B74000F840B0F90720B0F90510124854E600247B
:10B750004579114E11480AF0CAFD06EBC5031F7961
:10B76000BC4203D3BDE8F8400AF0DABD14B10C487E
:10B770000AF0BDFD56F835300A4853F82410FFF79B
:10B78000D5FE0134ECE74179BDE8F840064833E6E0
:10B79000F8BD00BFDAC90108D8C10108F1C9010824
:10B7A0008ED9010858D9010801CA01082DE9F041D4
:10B7B0000379054603F0300020280E46144625D1B3
:10B7C0000024274FDFF8A4806B799C4201DBBDE8A1
:10B7D000F0812B7903F00303022B11D0032B12D03D
:10B7E000012B14BF315D31573846FFF79FFE6B794F
:10B7F000013B9C4202DA40460AF079FD0134E3E75E
:10B8000036F81410F0E736F91410EDE703F00303EF
:10B81000012B06D008D2097848B1102813D0BDE812
:10B82000F08191F90010F7E7B1F90010F4E70C4846
:10B83000FFF77CFE8CB1B5F90720B5F90510094872
:10B84000BDE8F04172E66A79074BBDE8F04153F874
:10B85000323053F821000AF04ABDBDE8F08100BF44
:10B86000EEC90108E7CB0108D8C101088ED901084B
:10B8700038B50D460446FFF7A3FD2A46014620468B
:10B88000BDE8384092E72DE9F74F324C81468846B3
:10B890000025274601F0100300932F4B1868FDF791
:10B8A00053FE94F804B00BF00C034B453FD10D232D
:10B8B00003FB0573B3F80900FDF7FEFE06462046BC
:10B8C000FFF716FD0BF00302012A82467168B0688B
:10B8D00035D039D210F80A0011F80A20831A5A42DA
:10B8E0005A41009B03B112BB18F0200F10D07AB957
:10B8F0000D2101FB0571194809680192FFF716FE39
:10B900007168019A51442046FFF750FF0AF008FD84
:10B910000D2202FB057212481168FFF707FEB1689D
:10B92000002251442046FFF741FF0AF0F9FC01359F
:10B93000BA2D04F10D04B0D103B0BDE8F08F10F9B9
:10B940000A0011F90A20C9E730F90A0031F90A2082
:10B95000C4E700BF64B801084428002012CA0108E7
:10B9600013CA0108074B1B68597A4A1CD2B2194402
:10B970005A728872197A914202D81846FDF7E4BDCE
:10B98000704700BF442800200CB407B510F0200019
:10B9900009D069B92320FFF7E5FF05A904980191B3
:10B9A0000AF0C2FC012003B05DF804EB02B070475E
:10B9B0000020F8E70CB4C30607B500D551B905A9B6
:10B9C000049801910AF0B0FC012003B05DF804EB8B
:10B9D00002B070470020F8E72DE9F04F814690460D
:10B9E0000C46154600261927DFF8B0A087B0B8F13D
:10B9F000000F51D023782A7893422B794AD160786E
:10BA00006978884246D1A078A978884242D1E07806
:10BA1000E97888423ED1217999423BD161796879B0
:10BA2000081A414241410593EB7848460493AB78AC
:10BA30008B467B4303F5617303936B7801927B43E1
:10BA400003F5617302936B79524600933346FFF717
:10BA50009BFF237952460593E37859460493A378D4
:10BA600048467B4303F561730393637806357B4354
:10BA700003F56173029323780634019314F8013CB3
:10BA8000009333460136FFF795FF0F2EAFD107B075
:10BA9000BDE8F08F0021C6E7C346DAE71DCA0108FA
:10BAA000F7B50746FFF748FC044630B10022364997
:10BAB0000120FFF791FF03B0F0BD38460CF050FABB
:10BAC0000E28054659DC06264643781C8DF80740AB
:10BAD000FFF73AFC2C4C074650B10CF041FA032812
:10BAE00006D8A31958719DF8073001338DF8073037
:10BAF0003846FFF729FC074658B10CF031FA0D28FB
:10BB000007D806236B43E0549DF8073001338DF8C6
:10BB10000730711C0DF1070221443846FFF720FC65
:10BB2000FFF712FC074660B10CF01AFA182808D883
:10BB3000062303FB0543D8709DF8073001338DF8C9
:10BB400007303846FFF700FC60B10CF009FA0D2809
:10BB500008D8062303FB05459DF8073028710133FB
:10BB60008DF807309DF80730062BA4D00023A219CA
:10BB7000A3519380FFF71EFC9DE70E222146034848
:10BB8000FFF747FC97E700BF001F00203BCA0108F2
:10BB90002DE9F04F814690460C461646344FDFF8AB
:10BBA000D8A087B002F1200B002394F9022031497C
:10BBB000591891F90610914254D00833202BF6D130
:10BBC00008365E4504F10804EED107B0BDE8F08FF9
:10BBD00096F9023071799A42328841D12088904298
:10BBE0003ED1E578F07885423AD1257930798542A1
:10BBF00036D1A579B079854232D16579681A454246
:10BC0000454157F8211048460491B17957F8211061
:10BC10000391317957F821100291F178009257F889
:10BC20002110524601912946FFF7AEFE627994F940
:10BC3000023057F8222029460492A279484657F844
:10BC400022200392227957F822200292E27857F8B4
:10BC500022200192228800925246FFF7ABFEAFE706
:10BC60000025CEE7B8F1000FB2D14546DEE700BFB0
:10BC7000ECB701083C37002041CA01082DE9F34127
:10BC80000346FFF759FB044630B100220120374933
:10BC900002B0BDE8F0417BE70090019018465E1CC1
:10BCA0000CF05EF9314B40B203EBC40595F902206C
:10BCB000824256D00134042CF6D100252C46304661
:10BCC000FFF742FB074628B10CF04AF90134ADF802
:10BCD0000000E4B20026DFF898803846FFF734FB16
:10BCE000074600B30CF03CF9002258F82210D3B2FA
:10BCF000884203D00132102AF7D1002358F82320BC
:10BD0000904210D1022E1AD0032E1DD05A1E012EA1
:10BD1000D2B20FD00B2A03D88DF803300134E4B22D
:10BD20000136042ED9D1052C14D802B0BDE8F0415B
:10BD3000FFF740BB042AF3D88DF80430EEE7052B5B
:10BD4000EED88DF80630E9E79A1E0D2AE8D88DF86E
:10BD50000530E3E76B4603CB2860696002B0BDE8BD
:10BD6000F0818DF802000124A9E700BF16370020FA
:10BD7000ECB701082DE9F04F814690460C46154678
:10BD800000261927DFF8A8A085B0B8F1000F4CD025
:10BD900028782378834246D162786B789A4242D1E0
:10BDA000A278AB789A423ED1E178EB78CB1A59422F
:10BDB00059418B460AF055FA98B1EB7852467B43CD
:10BDC00003F561730393AB7859467B4303F56173C5
:10BDD00002936B780193037A484600933346FFF74A
:10BDE000D3FD20780AF03DFA98B1E37852467B43C0
:10BDF00003F561730393A37859467B4303F561739D
:10BE0000029363780193037A484600933346FFF721
:10BE1000D1FD0136142E04F1040405F10405B4D15A
:10BE200005B0BDE8F08F0021C3E7C346D9E700BFE6
:10BE30005ECA0108F7B50746FFF77EFA044630B13F
:10BE400000222C490120FFF795FF03B0F0BD3846D2
:10BE50000CF086F8132805463ADC8600781C8DF82D
:10BE60000740FFF771FA074690B10CF079F84FF0F0
:10BE70000C0E214BC0B203F108010EFB04F201EBE2
:10BE8000020C9CF808C0844528D00134252CF4D13C
:10BE90003846FFF759FA174C074650B10CF060F8D6
:10BEA0000D2806D8A31958709DF8073001338DF876
:10BEB0000730B11C0DF1070221443846FFF750FA54
:10BEC0009DF80730042BC0D0002344F82530BCE790
:10BED000132221460948FFF79CFAB6E713441A7A61
:10BEE000044B03F825209DF8073001338DF8073007
:10BEF000CEE700BF601E0020ACAD01083BCA0108C0
:10BF00002DE9F04F824691460E46154600278FB028
:10BF1000337896F90280089373780993F3780A933B
:10BF200096F904300B9396F905300C93B3790D9381
:10BF3000B8F1000F04D10FB0BDE8F04F0AF0F0B92E
:10BF4000B9F1000F4CD02B78089C6A789C4295F987
:10BF50000210E87895F904E095F905C095F806B067
:10BF60003CD1099C944239D1884537D10A9C8442FE
:10BF700034D10B9C744531D10C9C64452ED10D9C61
:10BF80005C4514BF002401240390029101920093A8
:10BF9000CDF818B0CDF814C0CDF810E03B46114AEA
:10BFA00021465046FFF7F0FC0D9BCDF80880069324
:10BFB0000C9B0C4A05930B9B214604930A9B50460D
:10BFC0000393099B07360193089B073500933B4673
:10BFD0000137FFF7EFFC102F9AD1ACE70024D3E72D
:10BFE0004C46E1E7D1CB01082DE9F0478AB0054680
:10BFF0000AF08CFB024630B995490120FFF780FF1B
:10C000000AB0BDE8F0870522924928460EF044FCAC
:10C01000044660B9702201468D480EF0FAFB2046B6
:10C0200022468D4BC2500C306028FBD1E8E7042239
:10C030008A4928460EF030FC0446002841D12846A3
:10C04000FFF782F906460028DAD00AF05FFB0746C0
:10C05000DFF8308258F824501DB981480AF076F98B
:10C06000CEE73A46294630460EF016FC0134002849
:10C07000F0D1774B0246194603F170069A719A7017
:10C080005A7003F8072BB342F8D1764B13F834708B
:10C0900003EBC404B84205DB29467348FFF7ACF94B
:10C0A000724886E06368C0EBC0021344D3F800E036
:10C0B0008E1841F802E09A880130B2809B79B37102
:10C0C000E8E707226A4928460EF0E6FB0446002806
:10C0D00075D1202128460EF0D1FB06460AF016FB4A
:10C0E000054680BB6348FFF721FA2C46624D214686
:10C0F00028460134FFF71AFA0E2CF8D10AF010F98D
:10C100000024DFF88491544FDFF880810C2621460B
:10C110004846FFF70BFA002506FB0476DFF870A10E
:10C1200001233268AB40134214BF41465146534885
:10C130000135FFF7FBF90E2DF2D101340AF0F0F8CA
:10C14000082CE3D15CE7304601AA4D490BF064FFAF
:10C150004B4E02AD00283DD0022C15D1029A072A81
:10C160002AD803990D2927D80378722B17D06E2B64
:10C1700022D10C2353430122374802FA01F1C2585D
:10C1800022EA0102C25013E00BF0EAFE01AA45F8D0
:10C190002400314600200BF03FFF0134DAE70C2386
:10C1A000012053432C4C00FA01F1E0580843E050C1
:10C1B0002F48FFF719FF23E7FFF7FCF8F8E72846B9
:10C1C00001AA2F490BF028FF00242D4E02AD78B1B3
:10C1D000082C02D1FFF7EEF812E70BF0C1FE01AA1E
:10C1E00045F82400314600200BF016FF0134EEE73D
:10C1F000082CEFD1029B0F2BECD8DDF80CC0BCF162
:10C20000070FE7D8049F0D2FE4D8059E06F16402BE
:10C21000C82ADFD8069DFF2DDCD807986428D9D816
:10C2200008996429D6D88842D4DA099C032CD1D83D
:10C23000DFF81CE0C3EBC3020EEB02030EF802C0F2
:10C240005F709E70DD70187159719C7128E700BF96
:10C25000C6190020EECB0108381A0020F4CB0108E3
:10C26000F9CB010870AF010806CC0108EDC7010841
:10C2700010CC01085AD9010818CC01081DCC0108BE
:10C2800021CC01087CB50108EEC901084ECC01089B
:10C29000FFD501082DE9F04F8046894616460D4628
:10C2A00014464FF0000ADFF810B189B0002E6FD0AD
:10C2B0006A6863689A4269D1AF68A368FB1A5F42F3
:10C2C0005F4194F90B305A46049394F90A30394689
:10C2D0000393B4F9083040460293B4F90630019351
:10C2E000B4F9043000935346FFF74EFB95F90B3039
:10C2F0005A46049395F90A3039460393B5F9083044
:10C3000040460293B5F906300C340193B5F9043078
:10C310000C35009353460AF1010AFFF74BFBBAF1C3
:10C32000080FC3D100242546DFF890A096B300275C
:10C330000123325903FA07FB59F8043053403BEA12
:10C34000030314BF0123002312EA0B0F079306D047
:10C3500000972B46524607994046FFF715FB59F8C0
:10C3600004301BEA030F06D000972B46524607996C
:10C370004046FFF71FFB01370E2FD9D10135082D9D
:10C3800004F10C04D2D109B0BDE8F08F002798E782
:10C390003746ABE73746012359F80420BB40134228
:10C3A00006D000972B46524601214046FFF702FB7C
:10C3B00001370E2FEFD1E1E723CC01083BCC010878
:10C3C000F0B585B00546FEF7B7FF002838D1044622
:10C3D0002B78002B3BD1062C41D1BDF904309AB209
:10C3E000072A3CD840F2DC54BDF90610A1F2EE2237
:10C3F00092B2A24233D8BDF90820A2F2EE2080B258
:10C40000A0422CD8BDF90A00814228DC824226DBFA
:10C41000914224DCBDF90C5005F16404A4B2C82C8F
:10C420001DD8BDF90E40112C19DC0C27194E07FB45
:10C4300003639980DA8018819D72DC7205B0F0BDCB
:10C4400000220120134905B0BDE8F04022E72D2B62
:10C4500003D0A3F13002092A16D8052C04DD05B05B
:10C46000BDE8F040FEF7A6BF28460BF079FD04AB0F
:10C47000661C03EB440424F80C0C15F8013F303B18
:10C48000092BFAD93446A3E7202BE8D101352646FB
:10C49000F8E700BF381A00202DE9F04F054688461E
:10C4A00014460027DFF8E0A085B0062300267B4372
:10C4B0000393039B334408EB030292F8C0B0002CB3
:10C4C0005ED0234493F8C0305246ABEB0300D0F16A
:10C4D000000949EB0009019300963B46494628466E
:10C4E000FFF752FA8DE840083B4652464946284637
:10C4F0000136FFF75FFA062EDBD10137062FD4D1C4
:10C500000026DFF884B008F1E40A1AF8019B002C39
:10C5100038D0A31993F8E4305A46A9EB03014F42EF
:10C520004F4101930096062339462846FFF72CFA1F
:10C530008DE840020623144A394628460136FFF7A3
:10C5400039FA0B2EE1D198F8F0606CB194F8F03024
:10C550002846F21A019300235442544100930A4A98
:10C5600007232146FFF710FA002301960093064A9D
:10C57000072321462846FFF71DFA05B0BDE8F08FD6
:10C58000A146AFE72746D3E750CC01087FB5054663
:10C59000FEF7D2FE044630B1002218490120FFF711
:10C5A0007BFF04B070BD28466A4615490BF034FD88
:10C5B000134E01AD78B1032C02D1FEF7FBFEF0E77C
:10C5C0000BF0CEFC6A4645F82400314600200BF003
:10C5D00023FD0134EEE7032CEFD101AC70CC3246E1
:10C5E0002946E0B206F0D4FF0028E6D033462A46BA
:10C5F00021460448FEF700FFD3E700BFAC29002026
:10C6000021CC010850CC01082DE9FF478146904616
:10C610000E4615460027DFF864A0B8F1000F2AD0B7
:10C620002B8832889A4224D174886A88A21A54428C
:10C630005441EA7821460292AA7848460192009332
:10C6400052463B46FFF7A0F9F37852460293B3787F
:10C650002146019336F8043B484600933B46013798
:10C66000FFF7A8F9102F05F10405D6D104B0BDE8F5
:10C67000F0870024DDE74446E6E700BF64CC01080C
:10C680002DE9F0410646FEF757FE044628B1BDE805
:10C69000F041002222490120B6E730460BF060FC51
:10C6A0000F2805462EDC3046FEF74EFE0646DFF824
:10C6B0007C801C4F203530460BF052FC38F814308B
:10C6C000984226DC012C11D0022C13D027F825002B
:10C6D00030462C210EF0D2F8064678B101230136FF
:10C6E0000134B3B1032CE6D1BDE8F08107EB85033B
:10C6F0009870EDE707EB8503D870E9E7A21E534277
:10C700005341EDE72146BDE8F0410F220648FEF710
:10C7100080BE002347F82530BDE8F041FEF74ABE51
:10C720002C2A0020AC2900203BCA010848B001088F
:10C730002DE9F04F07468A46164600248FB0DFF8F1
:10C7400060800DF124095AF82430494602A802936A
:10C7500008F052FB16B356F82430029D0393EB1AEF
:10C760005D420DF1100B5D41594603A808F044FBF2
:10C77000CDF800B02346424629463846FFF704F973
:10C780002346CDF800904246294638460134FFF74B
:10C7900011F9202CD7D10FB0BDE8F08F3546EFE767
:10C7A00076CC01082DE9F04F87B00546FEF7C4FDB1
:10C7B000044638B1002255490120FFF7B9FF07B000
:10C7C000BDE8F08F28460BF0CBFB1F28074600F38F
:10C7D00097802846FEF7B8FDA0460646A246A14629
:10C7E0002546A346494B009443F827400193484B04
:10C7F000E1B2E05C00230DF10C0CB64616F8012BFB
:10C800001AB190420FD00A2B09D106AE334400264C
:10C81000904203F80C6C08D0FEF7CCFDCFE703F88C
:10C820000C200133E9E70246EFE701390EF101067A
:10C83000032932D8DFE801F04E1F025B4FF0010EF2
:10C84000DFF8DCC00DF10B0010F8011F49B3002325
:10C85000304AD25C8A4203D00133072BF8D15346C9
:10C86000002212F80CA08A453DD10EFA02F248EAE5
:10C8700002089A46E8E74FF0010C0DF10B0111F8A0
:10C88000012F72B10023244813F800E0964526D109
:10C890000CFA03F349EA0309F1E703A80BF060FB84
:10C8A00083460134052CA2D1009B05F00F0545EA13
:10C8B000834545EA895949EA0A2A4FEA0B134AEAAD
:10C8C0000838019ADBB248EA030342F8273007F040
:10C8D0001FFD74E703A80BF043FB0546E1E70133B6
:10C8E000062BD0D1CBE70132062ABAD1C1E703A883
:10C8F0000BF036FB03460F28C8BF00230093D0E798
:10C900001F2221460548FEF784FD58E7AC29002088
:10C910004EB0010886C7010880C701083BCA01085C
:10C920008DC701082DE9F34781460F469046022640
:10C930000024DFF860A0B8F1000F28D037F82420D9
:10C9400038F824309A4238F806201ED1BD5BA91A67
:10C950004D424D4101920093524623462946484696
:10C96000FFF712F8BB5B5246019337F82430294693
:10C970000093484623460134FFF71CF8042C06F1C7
:10C980000406D8D102B0BDE8F0870025E2E74546AD
:10C99000E8E700BF80CC0108F8B50546FEF7CCFCFF
:10C9A000064628B1BDE8F840002226490120B9E733
:10C9B000254928460DF035FF68B94FF47A714FF4D8
:10C9C000FA62204B19805A809980DA8019815A8145
:10C9D0009981DA81F8BD28460BF0C2FA0328044693
:10C9E00028D82846FEF7B0FC064658B10BF0B8FA36
:10C9F000012705463046FEF7A7FC30B9BDE8F840F0
:10CA0000FEF7D8BC05460746F4E70BF0A9FA002F5D
:10CA1000F4D040F2DC53A5F2EE229A42EED8A0F216
:10CA2000EE229A42EAD8074B23F8245003EB840302
:10CA30005880F8BD3146BDE8F84003220348FEF7B0
:10CA4000E8BC00BFA41B0020EECB0108E0DD01081C
:10CA50002DE9F04F0E461546002797B00890099231
:10CA6000D6F80080002140460AF0A8FD04460028C0
:10CA700069D173680493B3680593F3680693099BBF
:10CA8000002B3DD0D5F800B0EB6859464046D5F8AC
:10CA900004A0D5F8089007930AF090FD80B15146A4
:10CAA00004980AF08BFD58B1494605980AF086FDB6
:10CAB00030B1079906980AF081FD041C18BF0124C3
:10CAC00013A95846FCF7AEFE10A983465046FCF762
:10CAD000A9FE0DA982464846FCF7A4FE0AA9814694
:10CAE0000798FCF79FFECDF808900390CDF804A0BE
:10CAF000CDF800B03B46154A21460898FEF744FFA2
:10CB000013A94046FCF78EFE10A904460498FCF7D2
:10CB100089FE0DA980460598FCF784FE0AA9814686
:10CB20000698FCF77FFE3B4603908DE81003074A0A
:10CB3000002108980137FEF73DFF082F06F1100687
:10CB400005F110058CD117B0BDE8F08F91CC01082C
:10CB50002DE9F84F07460026534D3846FEF7ECFB0B
:10CB6000804628B10022BDE8F84F4F4901206FE709
:10CB700005224E4938460DF08FFE38B900224A4B47
:10CB8000C25010308028FBD1BDE8F88F04224849FC
:10CB900038460DF081FE04463846002C3FD1FEF7A2
:10CBA000D3FB814600287CD009F0B0FDDFF818A146
:10CBB0005FFA80FB5AF82480B8F1000F04D13D4899
:10CBC000BDE8F84F09F0C2BB5A46414648460DF051
:10CBD00063FE013407460028ECD1374B2E6003EB8F
:10CBE000C404D4F8E8E02E612E622E632E642E6514
:10CBF0002E662E67BEF1000F03D094F8E4C067459F
:10CC000005DB41462D48FEF7F7FB2D4FA5E73B011D
:10CC1000EC1873440FCB013784E80F00EFE70BF0FB
:10CC20009FF90728054635D83846FEF78DFB06469E
:10CC300028B3FCF75BFD01241B4A2B01D050304682
:10CC4000FEF782FB064630B1FCF750FD164B01346F
:10CC500003EB051358603046FEF776FB064630B10D
:10CC6000FCF744FD104B013403EB0513986030468C
:10CC7000FEF76AFB28B9BDE8F84FFEF79BBB0446F8
:10CC8000DDE7FCF733FD084B032C03EB0515E860EB
:10CC9000F1D167E74146BDE8F84F07220948FEF7A2
:10CCA000B8BBBDE8F88F00BF481D0020EECB0108DF
:10CCB000F4CB0108F9CB010870AF010806CC0108DC
:10CCC000EDC701083BCA01087CB5010810B5102268
:10CCD000002104460DF09DFD0A2323800023A3813B
:10CCE000E381E3802381638110BD03788B4286BF9B
:10CCF000024B33F811000020704700BF28150020B8
:10CD0000034B187E10B1002201201A76704700BF35
:10CD1000281500207FB5294E294A31681268294C10
:10CD200091422949294A2A4B096826DB1B78C4F815
:10CD3000191092F8202094F82110E37794F822300B
:10CD40006177A27784F82030532007F031FDD4F8C2
:10CD5000190008F0A4F9607F08F0A1F9A37F01A8E9
:10CD60000193E37F029394F82030039307F048FD8A
:10CD700000230120336004B070BD1B7892F820209E
:10CD8000019194F821108DF80A3004F1190594F8F6
:10CD900022308DF808108DF809202946082201A8B4
:10CDA0008DF80B300DF00CFD0028E4D001AB03CB67
:10CDB000C4F81900C4F81D10C6E700BF983700205A
:10CDC000082200202815002038390020982B002048
:10CDD0002D2B00202DE9F041884600240C4B93E8D0
:10CDE000E000054406440744444501DBBDE8F0810A
:10CDF00037F9142036F9143035F91400134402229F
:10CE000093FBF2F3C01A07F08AFD0134ECE700BF90
:10CE1000A8370020064B1A684FF47A73B3FBF2F37D
:10CE2000C3EB431203EB8203DB000380704700BFB8
:10CE30000437002002392DE9F843426804460368AC
:10CE4000806806290DD8DFE801F004086A6D727564
:10CE5000780022605B42636003E05B4252422360E1
:10CE60006260384B1B78002B57D120680AF0BEF95E
:10CE7000804660680AF0BAF90746A0680AF0B6F979
:10CE8000314D0646696A40460AF004FA296B81462C
:10CE900038460AF0FFF9014648460AF0F3F8E96B14
:10CEA000814630460AF0F6F9014648460AF0EAF8AB
:10CEB0000BF0E4F9A96A206040460AF0EBF9696BCF
:10CEC000814638460AF0E6F9014648460AF0DAF8A3
:10CED000296C814630460AF0DDF9014648460AF0E1
:10CEE000D1F80BF0CBF9E96A606040460AF0D2F95C
:10CEF000A96B804638460AF0CDF9014640460AF053
:10CF0000C1F8696C074630460AF0C4F90146384654
:10CF10000AF0B8F80BF0B2F9A060BDE8F88352420D
:10CF2000226098E75B4223604042A06099E722605C
:10CF30006360F9E752426260F6E7524222605B4268
:10CF4000F6E700BF0E00002028150020F8B50024E9
:10CF5000084D094F05F14C06B5F848000AF042F9B2
:10CF60007A6B014630192434FCF74AFF6C2CF3D15C
:10CF7000F8BD00BF28150020242000202DE9F04F27
:10CF8000C04B89B01978C04DCB1EDBB2142B66D8CC
:10CF9000012202FA03F3BD4A1A40002A5FD085F845
:10CFA000B81010220021BA480DF033FC00273D23B1
:10CFB000B84C232084F859300126E761FDF737FA91
:10CFC000682308AA637602F80B7D2676334675211E
:10CFD00004F1140005F00AFC04F11408002842D002
:10CFE000AD4B0DF11602E365AC4B39462366404666
:10CFF000334605F0FBFB9DF8163003F07E038DF8F9
:10D000001630002840F00A819DF8153003F07E03A9
:10D01000682B8DF8153040F02281022384F85730B8
:10D02000062306AA1946E66D9D48B0479DF81D30B7
:10D030009DF81B209B00520002F0020203F0040343
:10D0400013439DF8192002F00102134300F0F88009
:10D05000012B40F0E980002384F858303CE00023A5
:10D0600085F8B8309DE78F4BE069A36110B92C209B
:10D07000FDF78AFA95F8B930E06183B910B11C2246
:10D08000C37182711321FDF7A5FAE069FDF7C9FAB2
:10D090000221A069FDF771FB012385F8B930E06931
:10D0A000FDF7BAFAF521A069FDF7B6FB012306AA40
:10D0B0000021A069FDF782FBE069FDF7B2FA9DF857
:10D0C0001830712B00F09E8000F29480122B00F03B
:10D0D000A180702B00F0EC82734A9379914684F81A
:10D0E0006830002384F8563094F85730022B40F013
:10D0F000E3826E4A22606E4A62606E4A22620122B8
:10D1000084F856206C4E0D2B326842F001023260DA
:10D1100005D8012202FA03F313F43E5F02D1002383
:10D1200089F8073099F803B0BBF1000F03D0BBF1C9
:10D13000070F40F0028199F8073099F80200002BA0
:10D1400000F0E68005235D4F84F85330431E84F8D9
:10D1500054300AF04BF839460AF09CF80AF09CFA71
:10D16000DFF82CA12368CAF8000084F852B04948BF
:10D17000984799F800300BB184F856304FF0000909
:10D1800007F0CEFC4FF0010BDAF80070CA464C4CA9
:10D190004822002120460DF03CFB98E8070004F1EE
:10D1A000080383E80700474B04F1240E93E80700C7
:10D1B00033F8053C8EE80700A4F81F30424B1A797B
:10D1C00093F8038084F83020039384F81E90B8F11C
:10D1D0000C0F00F29282DFE818F0C1009002C1004B
:10D1E000F00000011701F0002B012B012B012B0196
:10D1F0002B012B01AC2B00F05D82AF2B0CD0732BDD
:10D200007FF46AAF062384F85730304BE365304B28
:10D21000236661E70823F6E70923F4E7682B7FF428
:10D22000F3AE84F8576057E7022B01D1012313E7CF
:10D2300003F00303032BF9D00320FDF784FA4BE737
:10D240000123E66D0DF117020C211548B0479DF83A
:10D25000173013F00F03EFD0042BE7D1FBE6702B50
:10D2600004BF042384F8573036E71A4A84F856304E
:10D270002260194A04236260184AA2600D4A2262A1
:10D2800040E700BF80210020281500202100110068
:10D290000437002080340020ED270108E127010831
:10D2A00094340020003800406C340020FB28010832
:10D2B000DB26010890C1793D842100200000FC415B
:10D2C00024200020DC340020A620002051A80008E3
:10D2D0007FA800086B290108972601086726010826
:10D2E000914A2260914A063BDBB26260904A032B6E
:10D2F000226296BF8F4A0723D35C012284F856200E
:10D30000002B00F0E781FDE68B4A22608B4AEAE7BA
:10D3100094F857300A2B06D00C2B09D10223884FE2
:10D3200084F8533012E70423864F84F853300DE716
:10D330000323854F84F8533008E794F857300120D1
:10D340000A2B13BF002384F85300804F84F8533016
:10D3500018BF7F4FFAE64FF0000836E708AB03F836
:10D3600008AD00930123002253211846F9F72AFA49
:10D3700018B39DF81830E52B1FD1764B85F8BAA06D
:10D380002360754B63600423A3773368734843F0CD
:10D39000020333604FF48073A382236898474FF4ED
:10D3A0007A736363B5F84830002B51D1039B9B78A7
:10D3B000002B00F0A681A377A3E1E37F022B0CD121
:10D3C000674B2360674B636094F82030002B0CBFE1
:10D3D0006F236E2323770123D6E708AB03F8089D5C
:10D3E000009301230D221C211846F9F7EBF958B1DF
:10D3F0009DF818302A2B01D01A2B05D15A4B2360E7
:10D400005A4B63600223BFE708AB03F8089D009303
:10D410000123002218211846F9F7D4F940B19DF8EC
:10D420001830FB2B04D1524B2360524B6360D2E780
:10D43000E37F042B40F05E814F4B2360494BF5E7BF
:10D440000BFA03F313F4587F00F057814B4BF4E7CA
:10D4500000264B4FB5F8480009F0C4FE626B014648
:10D46000B8192436FCF7CCFC6C2EF3D19EE7454965
:10D470000A70DA781B79013A0A714B71042E00F2B6
:10D480001481DFE816F017003301170017002F0092
:10D490005B783C4C013B5BB2012BCEBF002305EB1C
:10D4A0000313D3F8BC30227063608878FDF76CF802
:10D4B000A060E3E7334C0A20FCF7B9FF2678012E81
:10D4C0002FD163796BBB772363710DF117030122B1
:10D4D000A0212C4805F0E9FB8146002856D1002EFA
:10D4E00040F0BE80274E1420FCF7A1FF3478012CB9
:10D4F00040F0B9807379002B40F0B58076237371CA
:10D50000214B0122D0211F4805F0CFFB95F8EC30CC
:10D51000582B00F0AA80002C00F0E88000237371E3
:10D52000E4E00026D1E700BF01280108DB2601085E
:10D5300090C1793DDFB30108BF28010861270108C8
:10D5400000009C43E438DE420000FA42D1456344C7
:10D5500000007A44B36B0008016900082420002011
:10D560004D2601081F2701080D6B000859680008A7
:10D570008F6B0008B76800083D26010845260108A2
:10D580007415002028210020141600209DF8173063
:10D59000FF2BA4D0002701221E215B4805F070FB61
:10D5A0004FF42F60FCF738FFBA46DFF85CB1A7F103
:10D5B000600106AB0222C9B258468DF818A08DF85A
:10D5C00019A005F072FB9DF818209DF8193043EA68
:10D5D00002234E4ABB520237102FE8D100231946CE
:10D5E000B5F8EA2002F00F0702F47F42A5F8EA201E
:10D5F00021F001002844B0F8DC00002818BF4FF0EB
:10D60000000911F0010F1ABFC0B2434083EA102392
:10D61000082013F4004F18BF83F4C05301384FEAB9
:10D620004303F6D101311029E2D13A43A5F8EA20AB
:10D63000B9F1000F7FF453AFC3F303339F427FF47C
:10D640004EAF42F21073A381E381314B2361314B22
:10D650006361314BA361314BE361314B23621EE0C7
:10D66000002363713EE700244AE72E4B18228821ED
:10D67000254805F01AFB3122F421234805F000FB70
:10D680000023B381284B7361284B3361284BB3616E
:10D69000284BF36145F6D813F381274B3362274AB1
:10D6A000136843F00403136020E0012EF7D11DE05E
:10D6B0000523A8E50723A6E5012B3FF4D6AD042BEF
:10D6C0003FF40EAE092B05D801229A4012F4587F80
:10D6D0007FF41AAE4FF00008194B1A785E79012AD0
:10D6E00019463FF4C4AE022A3FF4D2AE404609B018
:10D6F000BDE8F08F092B7FF6A3AEB8F1010F3FF61E
:10D700002AAE4FF00108E7E7282100200416002088
:10D710009F2C01080D2D0108992C0108FD2C0108F2
:10D72000E1220108181600203B26010839260108CD
:10D73000A52C01081D2D0108812401088421002049
:10D74000D22C0020F0B5002541F221072B462449B8
:10D750000A78961EECB2B44219DB0244941E013AD8
:10D760000C440A446478527802EB042292B2934249
:10D770000CD100244FF4AF6791F82450194E0130BA
:10D78000E3B29D4217D80122174B1A70F0BD044432
:10D790000C44647883EA0423082413F4004F04F152
:10D7A000FF344FEA430318BF7B4014F0FF049BB2E1
:10D7B000F3D10135CEE700EB4303DAB28B18013227
:10D7C0000A4493F801E0537803EB0E239BB27B43AA
:10D7D0001B1303F5487326F814300134D0E700BF5B
:10D7E00034160020281500204015002007298FBF7F
:10D7F0000020034B03EB8101886A80B2704700BFB1
:10D80000341600202DE9F041174D95F8482012B943
:10D810000020BDE8F081002285F8482095F84920D5
:10D82000A82AF5D195F85C40002CF1D10F4F104E8D
:10D8300005F14908283508EB0403D8781B7903EB78
:10D84000002009F0CFFC394609F024FD314609F0EB
:10D8500017FC09F021FF45F814000234102CEAD11E
:10D860000120BDE8F08100BF341600200000203EFA
:10D870000080BB43034B03EB4101B1F85E00C008DD
:10D88000704700BF341600201F4BF0B593F87E2080
:10D8900019460AB90020F0BD002093F87F40B3F884
:10D8A000806003EB440595F8857095F8862083F831
:10D8B0007E0042EA07229642ECD193F88330012B96
:10D8C00002D0812B14D0F0BD1846102C88BF102335
:10D8D0004FF0000288BF81F87F300C4B91F87F40F9
:10D8E000A3F12705D1B28C4203F1020302D8F0BDA7
:10D8F0000320EAE713F8026C13F8011C41EA062141
:10D9000025F812100132EDE734160020B916002078
:10D9100003788B420CD9074B890093F8A7200B445E
:10D92000D3F8A80002B1400800F5777080B27047C4
:10D930000020704734160020054B03EB8101D1F81D
:10D94000D80000EB8000C00800F55C7080B2704722
:10D95000341600205E4B10B593F82001002800F02B
:10D96000B680002293F8234193F8240183F8202104
:10D9700093F8222104F0070142EA012200F03F015E
:10D98000490141EAD401C3F8D82093F82521C3F80E
:10D99000DC1093F82611920093F8274142EA901286
:10D9A00001F0010042EA8022C3F8E02093F8280148
:10D9B00004F00F02D20142EA510200F07F01C3F8E5
:10D9C000E420090193F8292141EA141193F82A412E
:10D9D0005200C3F8E81042EAD01204F0030193F8B1
:10D9E0002B0142EA4122C3F8EC2093F82C2100F0ED
:10D9F0001F018901D20041EA940142EA501293F8D2
:10DA00002E4193F82F01C3F8F42093F82D21C3F889
:10DA1000F01004F0070142EA012200F03F01490141
:10DA200041EAD401C3F8F82093F83021C3F8FC1080
:10DA300093F83111920093F8324142EA901201F0CA
:10DA4000010042EA8022C3F8002193F8330104F078
:10DA50000F02D20142EA510200F07F01090141EABE
:10DA60001411C3F80811C3F8042193F8342193F872
:10DA70003541520004F0030142EAD01242EA412249
:10DA8000C3F80C2193F8372193F83601D20042EA0B
:10DA9000501200F01F01C3F8142193F838218901B6
:10DAA00041EA9401D407C3F810114CBF40F214713D
:10DAB000AD21C3F8181191074CBF40F21471AD218C
:10DAC00012F0080F14BF03200120C3F81C1110BD71
:10DAD0003416002008B5084B03EB8101D1F83C0156
:10DAE00009F080FB054909F0D5FB054909F0CAFAA0
:10DAF00009F0D2FD80B208BD3416002001F11F3FAD
:10DB000000405C446E4B30B593F87C210AB900208C
:10DB100030BD002293F87F0183F87C21162840F065
:10DB2000C980082210F0800F4FEA400018BF80F033
:10DB3000D500013AC0B2F5D193F87E11614D02399A
:10DB40008A42C0F2A78093F896218242DFD1182240
:10DB500093F8814193F8820183F87E2193F8802124
:10DB600004F0070142EA012200F03F014901C3F835
:10DB70003C2141EAD40193F88321C3F8401193F882
:10DB80008411920093F8854142EA901201F001005D
:10DB900042EA8022C3F8442193F8860104F00F0280
:10DBA000D20142EA510200F07F01C3F84821090185
:10DBB00093F8872141EA141193F888415200C3F881
:10DBC0004C1142EAD01204F0030193F8890142EAB1
:10DBD0004122C3F8502193F88A2100F01F018901E6
:10DBE000D20041EA940142EA501293F88C4193F832
:10DBF0008D01C3F8582193F88B21C3F8541104F018
:10DC0000070142EA012200F03F014901C3F85C210B
:10DC100041EAD40193F88E21C3F8601193F88F1173
:10DC2000920093F8904142EA901201F0010042EA1A
:10DC30008022C3F8642193F8910104F00F02D2010D
:10DC400042EA510200F07F01090141EA1411C3F8D0
:10DC50006C11C3F8682193F8922193F89341520014
:10DC600004F0030142EAD01242EA412293F89401FF
:10DC7000C3F8702193F8952100F01F018901D200AB
:10DC800042EA501241EA9401C3F87411C3F87821B2
:10DC9000012030BDAC18E4786040082410F0800FFB
:10DCA0004FEA400018BF80F0D500013CC0B2F5D16A
:10DCB000013245E7A0F128035842584130BD00BF6A
:10DCC00034160020B117002070B5304E0546337869
:10DCD0002F4C3BB1D4F8C03183429EBF0023337038
:10DCE00084F8C4312B4B1B6813F001021CD094F84C
:10DCF000C52194F8C63193420CD00123002184F849
:10DD0000C431254B84F8C6211970D4F8C8312B448E
:10DD1000C4F8C03194F8E43173BBD4F8F4018542FF
:10DD200034BF0020012070BD13F4005308D0134607
:10DD30001A4A32F8131009BB01330C2BF9D1E9E769
:10DD400084F8E431D4F8F0319847C307E2D50123D1
:10DD500000F00200002814BF1A46002284F8E431C3
:10DD60000D4B5A700CBF012300233370D4F8C83117
:10DD70002B44C4F8C031CDE7012070BD012300223F
:10DD800084F8C431044B1A70F0E700BF2D2B00203B
:10DD9000341600208C2100201000002000180020E4
:10DDA00000207047002070470023032BCCBF0122C6
:10DDB00000220CBF05211E2100F8132000EB4302B6
:10DDC0000133122B5170F0D1704710B500234FF47E
:10DDD0007A744FF4FA61C452C2180433102B518084
:10DDE000F9D110BD024B03EB4101B1F8CC017047F2
:10DDF00034160020024B03EB4101B1F8CC0170470F
:10DE000034160020044B93F8F80118B100220120C9
:10DE100083F8F821704700BF34160020024B03EB53
:10DE20004101B1F8FA01704734160020024B03EBB0
:10DE30008101B1F82002704734160020034610B566
:10DE400000F16004064A0C3303CA43F80C0C106856
:10DE500043F8081C43F8040CA342F3D110BD00BFE3
:10DE6000E4B3010840F2DC530380322343800123F2
:10DE7000042283730023C2731A4630B5084C838191
:10DE800019198D792D0741BF0D7981180D71013256
:10DE9000D02B03D0072A03F11003F1DD30BD00BF02
:10DEA000A0C6010870B50546FCF76EFA324CD4F8EE
:10DEB0005832C4F85802C31AB3F5FA5F82BF002380
:10DEC00084F85C3284F85D3294F85C3233B9A12D69
:10DED0001ED1012284F85D221B22227094F85D225B
:10DEE0002AB1E218EDB20133557084F85C3294F82F
:10DEF0005C522378AB420AD194F85E32052B0ED0E7
:10DF0000062B0FD0002384F85D3284F85C3270BD9C
:10DF1000A22DE3D1012284F85D222322DDE7002037
:10DF2000FFF710FCA3781E2BECD100200246013D28
:10DF3000C3B2AB4207DB25446B789A42E2D103209F
:10DF4000FFF700FCDEE7082123445B78DBB282EABE
:10DF5000030616F0010F4FEA530301F1FF310CBF26
:10DF6000DBB283F08C0311F0FF01C2F34702EED164
:10DF700001301A46DCE700BF3416002010B5044615
:10DF8000FCF702FA41F288310D4BD3F86022C3F856
:10DF90006002821A8A4284BF002283F8642293F8C6
:10DFA0006422142A03EB02010CBF0122013281F822
:10DFB000494014BF83F8642283F8482010BD00BF95
:10DFC0003416002010B50446FCF7DEF9254BD3F8D3
:10DFD0006822C3F86802821AB2F57A6F84BF002201
:10DFE00083F86C2293F86C224AB9A82C38D183F8B4
:10DFF0007E20A3F88020991881F8824006E0022A4A
:10E0000002D183F87F40F6E7242AF4D993F87F10F1
:10E0100001320231D2B249008A4283F86C2216DA08
:10E02000082241F22101B3F88000E4B280EA042022
:10E0300010F4004F02F1FF324FEA400018BF484091
:10E0400012F0FF0280B2F3D1A3F8800010BD0131BD
:10E050008A4201BF002283F86C22012283F87E20CD
:10E0600010BD00BF34160020F8B5434C94F874027C
:10E07000002859D0002384F8743294F8753294F84B
:10E08000765205EB0325FCF77FF93C4BADB2B0FBB4
:10E09000F3F0D4F88832002B47D1A4F88C52C4F89E
:10E0A00088020322D4F8903294F88F521E7894F8A4
:10E0B0008E0294F89472511E631893F875322B41B6
:10E0C00003F00F03B34212D20B2B10D808B18342D6
:10E0D0000DD0214491F875E2A11891F875120EEA5D
:10E0E000070E04EB830301EB0E21C3F8A8100232E4
:10E0F000112AE0D194F89532ABB194F8963293B1ED
:10E1000094F877321B060ED5FCF73EF9D4F870323E
:10E110001B4964301BB15A68121A002A28DB194ABD
:10E12000D36004320A600120F8BD9842B9D0C31A06
:10E13000012BB2D194F88E22002AAED0B4F88C32E2
:10E1400094F8A71092002244EB1A49B16FF0130122
:10E15000DB0293FBF1F303F50063C2F8A8309CE700
:10E160006FF013019B0293FBF1F303F58063F4E777
:10E1700003F108019B68CDE73416002020A10700B9
:10E18000A41800201000002010B50446FCF7FCF88D
:10E1900041F288310E4BD3F89822C3F89802821AC4
:10E1A0008A4284BF002283F89C2293F89C220F2A83
:10E1B0000DD8511CC9B21A441029E4B282F8754234
:10E1C00014BF0022012283F89C1283F8742210BD30
:10E1D0003416002010B50446FCF7D6F840F6AC51D2
:10E1E000104BD3F8A022821A8A42C4BF002283F8BF
:10E1F000A42293F8A4228AB90F2C11D1C3F8A0024B
:10E20000511CC9B21A44192982F8214114BF0022B5
:10E21000012283F8A41283F8202101E0182AEFD903
:10E2200010BD00BF3416002010B50446FCF7ACF852
:10E23000154BD3F8A82202F57A72904284BF0022CF
:10E2400083F8AC2293F8AC221AB9C3F8A8020521CE
:10E2500004E0022AFBD993F87E110231914211DDCC
:10E26000501CC0B21A44814282F87D41D4BF0122C1
:10E27000002283F87C21D8BF002283F8AC02D8BFEB
:10E2800083F8AC2210BD00BF3416002010B5044640
:10E29000FCF77AF8284AD2F8B032C31AB3F5FA7FFD
:10E2A000134628D9002283F8B42283F8B52293F8C4
:10E2B000B422C3F8B00292B9E1B2042901D02029F6
:10E2C00021D183F8B71283F8B8120221002083F815
:10E2D000B9124FF6FF7183F8B602A3F8BA12991873
:10E2E00081F8BC4293F8B81201398A4220D1012248
:10E2F00083F8DC2210BD92F8B5120029D7D001397D
:10E3000082F8B51210BD93F8B71271B9552C0CD123
:10E3100001211F2083F8B61283F8B74283F8B802B0
:10E32000A3F8BA2283F8B912D9E78C42D7D010BD2E
:10E33000013283F8B422FAE73416002010B5074CF6
:10E3400094F8962242B104F2DD21D4F8F402FCF7ED
:10E35000EEF8002384F8963210BD00BF341600207A
:10E36000F8B52A4E96F8DC3234460BB90020F8BDD9
:10E37000002596F8B63286F8DC52012B96F8B812D2
:10E3800032D1314491F8BB3291F8BA22B6F8BA02D0
:10E3900002EB032296F8B93292B203F11C05EDB2FA
:10E3A000E61896F8BD7296F8BC12023301EB07210D
:10E3B000DBB20144AB4288B2F2D18242D6D1002214
:10E3C00094F8B952124905EB4203DBB2234493F8A7
:10E3D000BD0293F8BC3203EB002341F82230013236
:10E3E0000E2AF0D10120F8BD06F52F7001F047FE8E
:10E3F0000028BBD096F8B732202BE0D006F52F705E
:10E4000001F058FE86F8B502B0E700BF34160020D0
:10E41000541800202DE9F04105460F460446094EE8
:10E4200006F10808217809B9BDE8F08105480CF02B
:10E4300025FA20B140453EBF801B631B3B5401348D
:10E44000F0E700BFF0B3010810B500212C2204460C
:10E450000CF0DFF90123637223752923A37540F2C1
:10E46000DC53238340F21A43638340F26C73A3832B
:10E470000223A377132384F8203040F246536384A9
:10E4800040F27533A38440F64303E3840623214618
:10E4900084F828300148BDE81040BBE7A5CC01084E
:10E4A000124B03EB400393F8F8222AB1022A12D050
:10E4B0000F4B33F810007047022809D90328F7D111
:10E4C0000C4B1B6813F4805F0B4B02D1988C704788
:10E4D000094B188B704793F8F90200EB800000EBB2
:10E4E000800000F2EE2080B2704700BF341600209A
:10E4F000542B00208C2100205422002008B5FBF76B
:10E5000043FF0222064B83F82023C3F81C03054B6C
:10E510001A68054B9A60012283F8212008BD00BFCC
:10E520003416002098220020982B002008B5FBF715
:10E530002BFF0222074B00F5B71083F82023064A71
:10E5400000F55870C3F81C03936803F2DC53936022
:10E5500008BD00BF34160020982B002070B50024A1
:10E56000114D2146702205F2223085F821430CF02E
:10E5700050F9214605F29234A4F17000631893F922
:10E5800002207AB11E680A180E509E889B790731C6
:10E59000937195F82133702903F10103968085F872
:10E5A0002133EBD170BD00BF341600200C230B4A81
:10E5B00003FB002393F80F341146FF2B07D092F88A
:10E5C000E8219A4203D9064A32F9130070470C2316
:10E5D00003FB0010B0F90C04704700BF3416002094
:10E5E000542B002038B5134A134B04461B7810688F
:10E5F000124D5843124B186008F0F4FD114908F011
:10E6000049FEC5F86404204605F004F9204605F0EB
:10E6100031F8208D08F0EAFD0B4908F03BFEC5F803
:10E620006804608D08F0E2FD074908F033FEC5F884
:10E630006C0438BD043700207420002034160020FC
:10E6400068210020BD3786356F12833A7FB5094BAC
:10E65000094A0493094B0A4903930A4B0A48029357
:10E660000A4B01930A4B00930A4BFCF7C5FE07B017
:10E670005DF804FBE9CC0108AECC01080EC8010826
:10E68000B3CC010805C80108BECC0108F9C70108D0
:10E69000EECC01080120002038B50A4B0D4603EBF3
:10E6A000C00494F8C020084853F82210FCF73EFF3D
:10E6B00094F8C6302BB1691C0448BDE83840FCF71B
:10E6C00035BF38BD08B4010859D90108EDC90108A2
:10E6D0002DE9F04F0025AA46A9465F4EDFF87CB130
:10E6E0008BB05E4B5E491A680023934225DB0135EF
:10E6F0000F2D06F13406F4D15A4BDB78D3B14FF429
:10E700007A73DBF84410DBF84820B1FBF3F35209CD
:10E71000DBF84C105448FCF76FFE0A229AFBF2F328
:10E7200099FBF2F102FB13A002FB119200904F48FB
:10E73000FCF762FE0BB0BDE8F08F51F82300864273
:10E7400022D00133D1E73B46079A01214848FCF724
:10E75000EDFE444639E038B108F048FD0146454831
:10E7600008F04CFE08F072FF04463A46294642483B
:10E77000FCF7DCFE4FF0000827E0069830E0214669
:10E780003E48FCF739FE58E07368012D0793F36AA1
:10E7900037680693336BF0690893B36A0993DAD14B
:10E7A00038B108F023FD0146324808F027FE08F092
:10E7B0004DFF334B80461B78012B90FBF3F4C2D9FD
:10E7C0003A4601212C48FCF7B1FE069B002BD4D021
:10E7D00041F288314FF47A7003FB0411B1FBF0F081
:10E7E000099B5B091DBF41F288324FF47A7103FB2C
:10E7F00004221A4618BFB2FBF1F21A49052DC97856
:10E800001CBF814492440029B9D04FF47A71089F0B
:10E81000B7FBF1F104910A2192FBF1F701FB1722FA
:10E82000039290FBF1F201FB120100920191029719
:10E83000069A21461348FCF7DFFD012D7FF457AF00
:10E840000F4B1B78012B7FF652AF424607990E48BB
:10E85000FCF7D2FD4BE700BFFC000020D81B0020D6
:10E86000DC1B0020FC1F00204ACD01086ACD0108F6
:10E8700003CD010800247449F4CC010846CD0108F9
:10E880007420002016CD01083ACD0108374B2DE940
:10E89000F34119684FF47A733548B1FBF3F1FCF793
:10E8A000ABFD344B34491A78344B098803EB8203AF
:10E8B000334AD3F8603112783248FCF79DFD324B71
:10E8C000324F1968324B3348B1FBF3F1FCF72EFE9F
:10E8D00007F026FDB7F850502F4A30493048FCF772
:10E8E0008BFDADB22F4A304B2946304DD31A3048FC
:10E8F000B7F85220FCF780FD2E6D002E33D0304645
:10E9000008F074FC01462B4808F078FD08F09EFEE4
:10E910008046D5F8EC0038B108F068FC014625487F
:10E9200008F06CFD08F092FE0446E86938B108F082
:10E930005DFC01461F4808F061FD08F087FEB7F84E
:10E940005410434664290190A8BF642100943246C4
:10E950001948FCF751FD194B1948198802B0BDE858
:10E96000F041FCF749BDB046D3E700BF9822002034
:10E9700098CD0108812B00201E22002008B4010838
:10E9800032220020B2CD010820000020D81B002038
:10E9900040420F00D8CD01080050002000080000C0
:10E9A000E8CD01080000020800F80108FC00002082
:10E9B0000CCE01080024744946CE0108BC2B00206F
:10E9C0008CCE01082DE9F04F0746304C87B02378F4
:10E9D0002F4A608852F82380FAF76EFE2D4BD0F84C
:10E9E00004A093F8563082689BB1D3469246012624
:10E9F00007F040030593A379721E002B08BF012383
:10EA0000934208DC244B08349C42E0D107B0BDE8B7
:10EA1000F08F9B46EBE7A38813441AF803501BF8CA
:10EA20000330EA1AD2F1000949EB020993B90096C2
:10EA300043461A4A49463846FCF7A6FFC5B9059B26
:10EA400033B900964346154A49463846FCF7B2FFAB
:10EA50000136D0E703F00F021B0940330292019305
:10EA6000009643460E4A49463846FCF78DFFE5E7D7
:10EA700005F00F032D09403502930195009643469A
:10EA8000074A49463846FCF795FFE1E7C8B4010854
:10EA900008B40108D81B002068B50108A7CE0108FA
:10EAA000BBCE01082DE9F04F89B0074607F02EFED6
:10EAB000044628B94120FFF785FF09B0BDE8F08F73
:10EAC0000246914938460BF0E7FE904D0646002875
:10EAD00049D18F4807F03AFC8E4CDFF86C82DFF8A2
:10EAE0006C9204F58C77A2882168B2FA82F201F167
:10EAF0004041A379A1F58431890A413155F8233089
:10EB0000C2F11F024046FCF711FDE17911B1484600
:10EB1000FCF70CFD083407F003FCA742E3D107F033
:10EB2000FFFB7D4807F012FC7C4CDFF82482DFF805
:10EB30002492DFF824A2237E01363246012140468A
:10EB400055F82370FCF7F2FC627E39463AB1504624
:10EB5000FCF752FC072E04F11C04ECD1ADE748464B
:10EB6000FCF74AFCF6E7384607AA6D4909F054FA63
:10EB700005F1C00782460026B84617F8363022460F
:10EB800055F8231050464FEAC6090BF085FE30B108
:10EB90000136142EF1D1634807F0D8FB8DE707AAA0
:10EBA0005F4909F039FA044609F0DAF94D4495F85D
:10EBB000C6200746EAB9002828DCC844B8F8020095
:10EBC000FAF77AFDFBB20193019AB8F8043027787E
:10EBD0001344029343680393002F00F0928052493C
:10EBE00020460BF01EFED8B9039B029A98544F485A
:10EBF000D2E7002805DD1346BB4209DA002A08BF28
:10EC0000012201214A48FCF704FC56E70123F3E7FF
:10EC100007AA4349002009F0FFF9013F0446CCE769
:10EC2000A7F14105EDB2072D04D9A7F16105EDB2B9
:10EC3000072D66D8601C09F093F9C3B20F2B8246EA
:10EC40005FD86C1C40EA0414E4B22046FBF79CFC3D
:10EC5000002856D0002C49D04FF00008230940333B
:10EC60000493DFF8F89004F00F03059300272FE0DA
:10EC7000B9F80200FAF720FDB9F8043042683B44C5
:10EC8000D15CA14223D1464504D101998F421ED0C7
:10EC90000021D154059A04992648FCF747FC5FFAF5
:10ECA00087FB5FFA88F3594618460093FFF7F4FC98
:10ECB000464509D12048FCF739FC00985946FFF732
:10ECC000EBFC1E48FCF732FC1D4807F03FFB013708
:10ECD00099F80630002B08BF01239F42C8DB08F1DA
:10ECE0000108B8F1140F09F10809BFD15FFA8AF2DF
:10ECF00005F141011348FCF77FFB039B029A9C54EA
:10ED0000DBE6FCF757FBD8E6D1CE010808B40108D2
:10ED1000D6CE0108301C0020E4CE010824000020DB
:10ED200021CC010802CF0108B6CE01080ACF0108A4
:10ED30003BCA010810CF010834CF010837CF0108C2
:10ED400076C9010841CF0108D9CE0108EDC90108F3
:10ED5000E9CE010858D90108FBCE0108C8B4010862
:10ED60002DE9F04F0E468DB0C449044603F09AFADF
:10ED70000546002840F02682C149204603F092FA59
:10ED80000546002840F02082BE49204603F08AFA5A
:10ED90000546002840F01A822046BB4903F082FA5B
:10EDA0000028054612BF0824254601240EB144F070
:10EDB0001004B64EB64FBE42C0F00A820123B54ED3
:10EDC00086F8563001F0D8FFFBF7B9F8B24928466B
:10EDD00003F068FA029608B144F0200414F0090F19
:10EDE00000F0D7810020FFF731FC04F01803182B46
:10EDF00004D1AA4807F07BFA07F092FAA84B204604
:10EE00001A78A84F002AA84A06BF012113460021FC
:10EE1000A64AFCF7CFFD2046FFF7D4FDA44B3D7872
:10EE20001B78A44AEE1A75427541A34E294606EB9B
:10EE30008303D3F870312046FCF7A6FD3B782946C2
:10EE400006EB8306D6F870319A4A2046FCF7B2FDED
:10EE5000029B0021D3F870014FF0010508F0AEFBD2
:10EE600000B9054605F00101944A2046FCF7A2FDD1
:10EE7000934A204602F18001924DFDF7E9FD924A46
:10EE800092492046FDF706FA95F902100026B1FADC
:10EE900081F18F4A49092046FCF78CFD2A468D49AD
:10EEA0002046FDF72DF88C4BDFF834A21F688B4B02
:10EEB000DFF870B2D3F800905AF82650002D40F0D9
:10EEC0008E81DFF864A269EA070B854B53F8258031
:10EED000B8F1000F40F0A381029B4546D3F8707251
:10EEE000D3F87C32DFF844927B40DB43DFF840A26A
:10EEF00003932846FCF726F9039B7A4A03424FF016
:10EF00000C0314BF4FF001084FF0000803FB05236A
:10EF1000D3F808B017EA000614BF4A4652465B46CB
:10EF200041462046FCF730FD0135002E14BF524605
:10EF30004A465B4641462046FCF73CFD132DD8D19E
:10EF400001260023684D694FDFF8E8E15A5DD95D7D
:10EF50000CA8104400F8201C13F80E000DF1300C22
:10EF600084440CF8101C16B1101A46424641013375
:10EF7000082BEBD1002508AB5D4A314620468DF8C1
:10EF80001850FCF701FD04AB594A31462046FCF706
:10EF900011FD584A58492046FCF7FAFD574A58498E
:10EFA0002046FDF7C5FB574A57492046FDF72CFB85
:10EFB000524A53492046FDF76FFA544A204602F15F
:10EFC0005001FCF7D7FE524A204602F15A01FCF7E5
:10EFD00003FD504A50492046FDF7A4FC0127DFF805
:10EFE00058A1DFF858B16B0003931AF815201BF8ED
:10EFF00015309A4240F0348117F80A6017F80B1068
:10F00000711A4E424E41022ADFF8AC8040F02A814C
:10F010004FF019091BF80720434409FB02F293F84B
:10F02000583302F2EE22019200933C4A2B463146BD
:10F030002046FCF7A9FC17F80A30384A09FB03F907
:10F0400009F2EE2301936B0013F80A30314698441D
:10F0500098F85833204600932B46FCF7ABFC01355B
:10F06000122D07F10207BED121460020FCF70BFC50
:10F0700014F0080F2A4D00F00D8161E064CF010803
:10F08000D7E501086BCF010871CF010878EB0108C3
:10F0900038EF0108D81B002075CF01087ECF01088A
:10F0A000EB210020912100204DCF01088ECF0108D7
:10F0B0008821002096CF010808B401089FCF0108DD
:10F0C000481D0020C6190020381A0020C41A00204C
:10F0D000AECF0108241B002094210020C82000206E
:10F0E000E8B5010864B60108B0220020F0B30108B9
:10F0F000D2CF0108163700205C370020AC29002051
:10F10000D02B00202C2A0020502C0020601E002034
:10F11000001F0020A41B0020941B002021C901080F
:10F12000FC210020BBCF0108C7CF01084FCF010849
:10F1300059CF010854220020B41B00202C190020B4
:10F14000214600202E7803F099F82146012003F093
:10F1500095F82146022003F091F8304601F0D8FAE4
:10F16000544802F015FD214600206D7803F072F836
:10F170002146012003F06EF82146022003F06AF8D0
:10F18000284606F02FFF4B4802F0E2FC4A4807F001
:10F19000AEF8A20704D5494B2146187803F06EF863
:10F1A000630704D5454B2146587803F053F8444C87
:10F1B000444B9C4277D30023029A82F856300DB01C
:10F1C000BDE8F08F0124F1E50224EFE50424EDE52C
:10F1D00072887168B06808F0EBFE1436EBE52B78A6
:10F1E000DBB14FF0010869EA070308FA06F813EAF1
:10F1F000080F14BF012100212B465A462046FCF778
:10F20000C3FB67EA090313EA080F5A462B4614BFEB
:10F21000012100212046FCF7CDFB01364CE698F891
:10F220000030DBB10126AE4019EA060F0AD067EACA
:10F23000090333425246434614BF012100212046B0
:10F24000FCF7A2FB374209D01BEA060F43465246A1
:10F2500014BF012100212046FCF7ACFB013534E648
:10F260000026D0E6434493F8583331460093164ABB
:10F270002B462046FCF788FB144B6A009B5C31460A
:10F28000984498F85833104A009320462B46FCF7D0
:10F2900091FBE4E62146287802F0F0FF21466878E9
:10F2A00002F0D8FF75E76288A168606808F080FE08
:10F2B00014347DE7EDC7010889CF0108FC21002047
:10F2C00078EB010838EF010831C90108B41B0020B0
:10F2D000904B73B5186808F0D1FF8F4C0546206835
:10F2E00008F0CCFF0646402005F094F9002866D1CE
:10F2F000206961794C2800F23183DFE810F04D007D
:10F30000530063006A006E007200780087008C0072
:10F31000910096009B00A000A500B100BB00C000BA
:10F32000CB00D000D500DA00E200EA00F200FA00DB
:10F33000020177017F01870194019D01A601AF01C0
:10F34000B801C101CA01D301DC01E201EB01F20104
:10F35000F801FE0104020A02110218021F0225022E
:10F360002B02320239023F0245024B025102560281
:10F370005B02600265026A02700276028302880202
:10F380008D02920297029C02A2020D031203170340
:10F390001C03210326032A03604A6149614805F0E2
:10F3A0008EFE09E0604B614A0193614B6149009315
:10F3B0006148624B05F083FE23690133236100201D
:10F3C00002B070BD5E4B5F4A5F49604805F077FE52
:10F3D000F2E75F4A52495F48E1E75F4A50495F48B8
:10F3E000DDE75F4B5F49B3F900205F48D7E705F0E1
:10F3F000A3FE5E4A5A491288B1F90010424392FBBB
:10F40000F1F20346D2B25A495A48DFE7574B554901
:10F410001A885948C3E7594B52491A8A5848BEE7D7
:10F42000564B50495A8A5748B9E74FF07E525649D1
:10F430005648B4E7B3B2AAB255495648C6E7B4F83D
:10F44000402055495548AAE7554B1B68DB0404D5B5
:10F4500094F8742050495348A1E70F232361ABE788
:10F46000514952488B784A7809780091504905F003
:10F4700026FEA1E74F4B48491A884F488FE74A4B71
:10F480009B79012B98D1B4F97830B4F97A204049AE
:10F490004A489BE74A4B33491A684A487FE74A4B38
:10F4A00030499A7849487AE794F87C202D494848B1
:10F4B00075E70C2303FB0141464891F87E2029495A
:10F4C0006DE70C2303FB0141434891F88020254957
:10F4D00065E70C2303FB0141404891F87F20214957
:10F4E0005DE70C2303FB01413D4891F887201D494E
:10F4F00055E70C2303FB01413A4891F88120194953
:10F500004DE70C2303FB0141374891F88220154950
:10F5100045E700BFD0370020F81F0020D5D30108F1
:10F5200059D90108E1D30108AECC0108B3CC0108D8
:10F530000EC80108EFD30108FDD30108EECC010885
:10F5400005C80108F9C701089FCC01080FD40108BC
:10F55000E80000201DD401081020002030D401084C
:10F5600094370020EEC901083BD40108D0330020B5
:10F5700046D401084CD4010857D40108B8370020FC
:10F580005FD401086BD40108A2CE010877D401082A
:10F590004ED5010882D401088ECC01088ED4010812
:10F5A000B437002095D40108862B0020A9D4010887
:10F5B000A0D40108CE370020B9D40108C1D4010875
:10F5C00004370020CFD401086C340020D8D40108BF
:10F5D000E8D40108FAD4010802D501080AD50108C7
:10F5E00016D5010822D501082AD501080C2303FBF2
:10F5F0000141964891F886209549D0E60C2303FBFB
:10F6000001419448B1F888209149C8E60C2303FBD6
:10F61000014191F8843091F8832091F885108E484B
:10F6200000918E4923E7D4F8A4108D484B780A78CE
:10F630008978009189491AE7D4F8A41089480B7990
:10F64000CA7849790091854911E7D4F8A410864811
:10F65000CB798A79097A0091804908E7D4F8A41017
:10F6600082488B7A4A7AC97A00917C49FFE6D4F8BD
:10F67000A4107F484B7B0A7B897B00917749F6E693
:10F68000D4F8A4107B480B7CCA7B497C0091734959
:10F69000EDE6D4F8A4107848CB7C8A7C097D0091F3
:10F6A0006E49E4E6D4F8A41074488B7D4A7DC97D88
:10F6B00000916A49DBE6D4F8A43065491A7E7048A7
:10F6C0006DE6D4F8A4106F480B7FCA7E497F009185
:10F6D0006249CCE6D4F8A4305D4993F826206A4804
:10F6E0005DE6D4F8A4305A491A8C684857E6D4F835
:10F6F000A4305749DA8B664851E6D4F8A43054490F
:10F700005A8C64484BE6D4F8A43051499A8C62482C
:10F7100045E6D4F8A4304E4993F827205F483EE6EA
:10F72000D4F8A4304A4993F82C205D4837E6D4F841
:10F73000A430474993F82D205A4830E6D4F8A43035
:10F7400043495A8E58482AE6D4F8A43040499A8E44
:10F75000564824E6D4F8A4303D4993F8362054485E
:10F760001DE6D4F8A4303A4993F83720514816E6FC
:10F77000D4F8A43036491A8F4F4810E6D4F8A43094
:10F7800033495A8F4D480AE6D4F8A43030491A8DCF
:10F790004B4804E6D4F8A4302D495A8D4948FEE57B
:10F7A00094F8A8202A494848F9E594F8A92028495E
:10F7B0004648F4E5464B2649DA784648EFE5444B9F
:10F7C00023491A794448EAE5414B21495A7943488B
:10F7D000E5E53F4A4249D38942485289F6E53C4A29
:10F7E0003F49138A40489289F0E5B4F8AE0007F02B
:10F7F000FDFC3E4907F04EFD07F028FF1449024684
:10F800003B48CCE594F8B12011493A48C7E53A4B5A
:10F810000F495A793948C2E594F8C1200C49384853
:10F82000BDE594F8CA200A493648B8E5364B084980
:10F830009A7F3648B3E5344B054993F82020344885
:10F84000ADE5314B02495A8C3248A8E533D5010861
:10F85000EEC901083CD501086BCF01084BD5010862
:10F8600054D501085CD5010865D501086CD501089F
:10F8700073D501087AD5010882D501088AD5010817
:10F8800093D501088CD501089AD50108ACD501089B
:10F89000B9D50108C4D50108D3D50108E6D50108BA
:10F8A000F3D5010801D6010812D6010829D60108AE
:10F8B0003BD6010855D601086BD6010879D6010858
:10F8C00083D6010890D60108B3E20108A1D6010849
:10F8D0006C340020AED60108B7D60108C9D601089D
:10F8E0004ED50108D9D60108E7D601080000C84264
:10F8F000F9D6010804D70108D22C002011D701083D
:10F900001FD701082CD701085422002042D7010834
:10F9100053D701086DD70108114B12491A7A1248C2
:10F920003DE5124B0F491A79114838E50F4B0D4947
:10F930009A78104833E50D4B0A491A880E482EE58F
:10F940000A4B0849DA890D4829E5A27905490C488E
:10F9500025E5D4F8D02003490A4820E501202FE509
:10F9600054220020EEC9010887D70108B8370020CB
:10F9700099D70108AAD70108BDD70108CCD701083B
:10F98000DDD70108E8D701082DE9F74FA3EB020BFB
:10F9900016460E9B0D9A002914BF062504259B1AB6
:10F9A00001934E4B04465A6989460132984628D144
:10F9B0001A69954240F28F80DFF838A15AF8220088
:10F9C00006F0A4FE0B3004F025FE074618B1012016
:10F9D00003B0BDE8F08FD8F8101041485AF8212044
:10F9E000032994BF2146494605F094FB3D4988F818
:10F9F000D4700A68101AD8F8142008600132C8F8C8
:10FA00001420DFF8E090D8F814400C9B9C421BDBDC
:10FA100013D1012004F0FEFD78B932490A200A68AA
:10FA2000013A0A6004F0C4FED8F810200132C8F888
:10FA300010204FF0FF32C8F81420D8F8100085428B
:10FA400094BF00200120C3E70D9B53B1019B04FB31
:10FA500003F20D9B995C01228A40234909680A42FE
:10FA600028D004FB0BF4D8F81020371942BB3059CA
:10FA700006F04CFE00F1050A504604F0CBFD0028CC
:10FA8000A5D1D9F8000098F8D420A0EB0A00C9F855
:10FA90000000C2B12C2004F08BFED8F81020B2B9BF
:10FAA000305904F01BFE97F904104B1C02D00F488C
:10FAB00005F030FBD8F814200132C8F81420A2E772
:10FAC0004FF0030AD8E7012288F8D420E5E717446D
:10FAD00039790748ECE700207AE700BFF81F0020DB
:10FAE000F1D70108CC330020B437002000D801083A
:10FAF000EEC90108C0B701082DE9F84F374B0025C2
:10FB00001C68374F264604F1300846F8040B07F10D
:10FB10000C0B07F1180AA7F1AC09E85907F096FD9C
:10FB200046F8040B55F80B0007F090FDB06055F84F
:10FB30000A0007F08BFD2B4B7061EB18586808F03A
:10FB40009DFB09EB05039B6B043528F8020B0C2D7C
:10FB5000A8F80430E1D10025234F04F1280657F816
:10FB6000250007F073FD0135042D26F8020BF6D1B0
:10FB700000261E4D04F14407B5F8FC2005F58279F6
:10FB8000A287B5F8FE20E287B5F80021A4F840204E
:10FB9000B5F80221A4F84220154A92F800804645A3
:10FBA00014DB144B5B88A4F86430D5F82831A4F832
:10FBB0006630D5F85431A3660F4B1B88A4F86C301F
:10FBC000B5F86631A4F85E30BDE8F88F59F8260024
:10FBD00007F03CFD013627F8020BE0E7A8370020CC
:10FBE000D02000200437002034220020F81F0020FD
:10FBF000D43700201E2200207C2B002010B50B4C97
:10FC000021780B290BD801238B4040F603011940C2
:10FC10000BD113F4C06F02D0FF2005F0C3FA044BE0
:10FC20001A68044B5A610B23237010BDA6370020BD
:10FC300098220020F81F00205E2810B5084C07D13C
:10FC400023685D2098473E202368BDE81040184790
:10FC50005D282368F9D1984723683D20F5E700BF68
:10FC60000C2200202DE9F0410E46054607464FF6CE
:10FC7000FF7443189F4211D1DFF83880BD4212D182
:10FC8000E1B2D8F80400FAF74FFCD8F80400210AD2
:10FC9000FAF74AFCB01CC0B2BDE8F08117F8012B9E
:10FCA000A41AA4B2E6E715F8011BD8F80400FAF785
:10FCB0003BFCE3E70C22002007B58DF80610090A8B
:10FCC0008DF807100421062360F05F008DF8050011
:10FCD0000DEB01008DF80430FFF7C4FF03B05DF8B1
:10FCE00004FBA0F17D03012B70B504460D460B4EBD
:10FCF00011D87D21B068FAF717FC84F02001B068B4
:10FD0000FAF712FC35B12888204400EB102000F0EF
:10FD1000FF00288070BD0146F1E700BF0C220020E3
:10FD2000024B0146D868FAF7FFBB00BF0C22002047
:10FD3000084BDA68D10709D4DA68520708D4DB68BF
:10FD400013F0100F14BF03200420704701207047E8
:10FD500002207047002002400B88F0B54E88B1F8B1
:10FD600004E00F89CC88002B3CD1038C23F00103E5
:10FD70001B041B0C0384018B824B89B221F0F3011D
:10FD8000058C4EEA010141EA07119842ADB289B2F1
:10FD900012D003F5006398420ED0B0F1804F0BD023
:10FDA000A3F59833984207D003F58063984203D0B7
:10FDB00003F58063984212D125F0020546EA050357
:10FDC00043F0010301830384038B23F00C031B0422
:10FDD0001B0C0383038B9BB21C430483F0BD25F0F3
:10FDE0000A05EBE7042B44D1038C4FEA0E2E23F0D7
:10FDF00010031B041B0C0384038B4EEA073723F408
:10FE000040731B051B0D1F435E4B018C984289B24A
:10FE1000BFB212D003F5006398420ED0B0F1804F0C
:10FE20000BD0A3F59833984207D003F5806398422E
:10FE300003D003F58063984214D121F0200141F0F2
:10FE4000100343EA06139BB207830384038B23F456
:10FE500040631B041B0C0383038B9BB243EA042403
:10FE6000A4B2BAE721F0A00146EA010343F010036F
:10FE7000EAE7082B038C3FD123F480731B041B0C8F
:10FE80000384818B3F4B89B221F0F301028C4EEA4F
:10FE9000010141EA0711984292B289B212D003F5EA
:10FEA000006398420ED0B0F1804F0BD0A3F5983389
:10FEB000984207D003F58063984203D003F580632E
:10FEC000984213D122F4007343F4807343EA06236B
:10FED0009BB281830384838B23F00C031B041B0CD4
:10FEE0008383838B9BB21C438483F0BD22F4206305
:10FEF000334343F48073ECE740F6FF4223F480532E
:10FF00001B041B0C0384818B038C0A40390341EAD8
:10FF10000E2111431B4A9BB290421FFA81FE12D060
:10FF200002F5006290420ED0B0F1804F0BD0A2F5E6
:10FF30009832904207D002F58062904203D002F5D9
:10FF40008062904215D123F4005343F4805343EA76
:10FF500006339BB2A0F81CE00384838B23F4406338
:10FF60001B041B0C8383838B9BB243EA0424A4B23F
:10FF7000BAE723F400735B045B0C334343F4805310
:10FF8000E8E700BF002C01402DE9F041CB780E8856
:10FF9000DA0648BF8A7803F00F0548BF154316F00C
:10FFA000FF0F1AD000214FF0010E4FF00F0C026826
:10FFB0000EFA01F737EA06040BD18C000CFA04F8AC
:10FFC00022EA080205FA04F4282B42EA040225D1A9
:10FFD000476101310829EBD10260FF2E1CD90021B5
:10FFE0004FF0010E4FF00F0C426801F108040EFAB9
:10FFF00004F434EA06070BD18F000CFA07F822EA62
:020000040801F1
:10000000080205FA07F7282B42EA07020AD14461E1
:1000100001310829E9D14260BDE8F081482B08BFD1
:100020000761D6E7482B08BF0461F1E70F4B1A6858
:1000300042F001021A6059680D4A0A405A601A6873
:1000400022F0847222F480321A601A6822F480222C
:100050001A605A6822F4FE025A604FF41F029A6036
:100060004FF00062034B9A60704700BF00100240DF
:100070000000FFF800ED00E080F3088870470246BA
:100080004FF6FF7330B58C1E151AAC420BD80144E5
:1000900011F8012CB2EB132F0AD1005DDBB2C31AA9
:1000A0005842584130BD12F8015B5B1B9BB2EBE735
:1000B000002030BD13B52E4B4278197C02F00F049E
:1000C00009B904B11C74197C8C4203D3611AC8B2FB
:1000D00002283BD9002049E0902A11D106238DF84F
:1000E0000430244B64F06F045B5C04218DF806300F
:1000F00002238DF805408DF807300DEB010033E049
:10010000A02AE7D11B4A525C022A1AD0032A09D03E
:10011000012ADFD10A21184BB3F95030594301F5B8
:10012000C87109E00A215A8A514393F825201AB16F
:1001300093F8263091FBF3F189B22046FFF7BCFD1E
:1001400014E0586B07F0A8FA81B2F6E702F0F0026B
:10015000802AC1D10423022164F07F048DF8043089
:100160008DF805400DEB0300FFF77CFD02B010BDDC
:100170000C220020E8B7010880340020024B93F8DD
:100180003810D86BFAF7D0B90C22002038B50446E5
:10019000054D0146E86BFAF7C7F995F838305C4031
:1001A00085F8384038BD00BF0C22002010B5044649
:1001B000C0B2FFF7EBFF200ABDE81040E6E738B514
:1001C00000230546084C2421E06B84F83830FAF708
:1001D000ABF9E06B5421FAF7A7F92946E06BBDE8CB
:1001E0003840FAF7A1B900BF0C2200207FB50024E7
:1001F0000B0A04AD8DF808008DF80A10000A8DF87E
:100200000B3025F80A4D0B0C090E8DF809008DF8FE
:100210000D10102029468DF80C30FFF762FD02AE5C
:10022000305D29460134FFF75CFD062CF8D19DF8BE
:1002300006000021C043C0B2FFF753FD04B070BDFB
:1002400073B50D4C0646206C0D46FAF725FD637F0D
:10025000A27F003318BF01230AB143F008030193C2
:1002600096F9000000954FF4964300220821FAF712
:1002700041FD206402B070BD0C22002010B5054C79
:10028000206CFAF74EF900B910BD206CFAF746F968
:10029000F6E700BF0C22002008B5094B5A6C927893
:1002A0001E3A012A07D9186C01210430FFF7C8FF54
:1002B000BDE80840E2E70121186CFAF729F9F7E7F1
:1002C0000C2200200028114AB8BF404290FBF2F3F4
:1002D00030B50F4C04FB03053C2068430D4D90FBEB
:1002E000F2F2ED7F75B903EB830303EB830302EBBB
:1002F00083030B804FF47A7304FB020292FBF3F248
:100300004A8030BDC3EB0313F1E700BF809698002D
:10031000806967FF0C22002010B50446C0B2FFF7C9
:100320008BFCC4F30720BDE8104085E4014B5E2040
:100330001B6818470C22002070B50546044C5E204F
:100340002368984723682846BDE87040184700BFD7
:100350000C22002003885A0602D513F4057F0BD126
:1003600003F48253B3F5825F08D1054B93F8500034
:10037000C31F584258417047012070470020704702
:100380000C2200202DE9F3418A4C676F67B3384691
:10039000FFF7E0FF884E804638B12368B34223D090
:1003A000A36F0BB3E36026601EE094F87C0003F0BB
:1003B000D9F8236805469A1B53425341834213D010
:1003C000002874D0637F97F90200B3FA83F35B09C6
:1003D000019302234246009304214FF41653FAF787
:1003E00089FCE0600028DED194F87D0003F0BAF8C3
:1003F00094F87E30054683421AD000285FD0636CA3
:10040000B3B1A27F93F90200002A0CBF0022082298
:1004100003230192009300224FF496430821FAF738
:1004200069FC206420B1FFF737FF012384F87E3098
:1004300094F87F0003F096F894F8803005468342E4
:1004400022D0002842D0D4F88420EAB1A37F92F9C8
:100450000200002B14BF08230023627F2021002A02
:1004600008BF43F0010301930323002200934FF4DC
:100470006143FAF73FFCA06030B1012384F8883073
:1004800084F88030D4F88C30D4F890503DB32846AE
:10049000FFF760FF18B394F89430002B43D1A36F9B
:1004A000002B40D0E363012384F894303BE0E06804
:1004B000002899D0FAF7F0FBE560256094E7206CFE
:1004C000FAF7EAFB256484F87E50B1E7A068FAF7F2
:1004D000E3FBA56084F8885084F88050D4E794F852
:1004E000950003F03FF894F89430064683421AD002
:1004F00000284FD0BDB1AB79304A002B08BF022392
:1005000002EB8303627F95F90200003218BF0122DB
:10051000019202225B68009210210022FAF7EAFBA6
:10052000E0630028BFD194F8960003F01BF894F81C
:100530009730054683422AD098B34FF47A72204B05
:10054000C3F8B422D4F898300BB31A8802F482525C
:10055000B2F5825F1BD093F90200637F0022002B6B
:1005600014BF09230823019303234FF48051009300
:100570004FF4E133FAF7BEFBC4F89C0038B1002316
:1005800001226060237484F8972084F8A03002B0C0
:10059000BDE8F081E06BFAF77FFBE66384F89460D6
:1005A000C1E7D4F89C00FAF777FBC4F89C5084F8B4
:1005B0009750ECE70C22002021FD0008E8B7010865
:1005C000FC00002038B50546064C206800B938BD4F
:1005D0004368EB1A002BFADB8368236003689847B3
:1005E000F3E700BFA418002000231A4630B5084CDA
:1005F000037219198D79AD0742BF0979815401320F
:10060000D02B03D0072A03F11003F2DD30BD00BF69
:10061000A0C60108002210B5064C04EB02118B792C
:1006200013F0010302D00B79037010BD01320E2AC2
:10063000F3D1F9E7A0C60108142201234270152264
:1006400003708371C271037121228370112342717F
:10065000C37070472C23037002234370704708B5A2
:100660000B4B1820197800231D460A4C8B4207DBE0
:1006700040F2DC50F9F7D0FE074A084BDA60FEE79B
:1006800000FB03F2125902B115800133EEE700BFFF
:10069000D43700204C2800200400FA0500ED00E0CB
:1006A00080B501210220F9F7F7FF144B1B7803F006
:1006B0000503052B12D1124B0024186806F0C6FF63
:1006C000104B114F1D7806B2AC4210DB0F4B1B785C
:1006D0000BB103F087F93220F9F7A9FE00210120C0
:1006E000F9F7DAFF00210846F9F7D6FFFEE73046B2
:1006F00006F07CFD47F824000134E5E7C50A002038
:1007000094290020D4370020FC200020281200204B
:10071000022828BF0220064B064A18704E2303FB0E
:100720000023054A0130C0B21360FAF7C9BD00BF0B
:10073000FC1F0020922F00209C2000202DE9F04F6C
:100740008BB0FDF7F3FE0326DFF840914A4FA7EB8D
:1007500009071822002104A80AF05BF8474B484A11
:10076000CDF8109005975A6002F188325A60012244
:100770008DF824203422DA60424B02221B8869461D
:1007800004A8ADF80030F8F759FF022269464FF689
:10079000FF70F9F76EFB4FF0000B80463A4CDFF824
:1007A000F0A0544536D300250AAC24F8245D02227B
:1007B000214604A8F8F742FF022221464046F9F7F5
:1007C00058FB40BAC0430222ADF8080002A904A8B1
:1007D000F8F734FF079860B106ABC0F10402294670
:1007E00018440AF016F8069904A8F8F7B9FE079518
:1007F00008909DF82430089A23B120490B6943F0F2
:1008000080030B61013E2DD0002AA2D1F9F747FBEE
:1008100050B32CE0658802A9C5F30B05AB1DADF8FC
:100820000830238804A8C3F30B02ADF80A201B0B81
:1008300006228DF80C308DF80DB0F8F7FFFE062279
:1008400002A94046F9F715FB804661682A4604A8CC
:10085000F8F7F4FE616840462A46F9F70AFB1434BB
:1008600080469EE7002AD1D00520F9F76CFFFDF7FE
:1008700045FE0BB0BDE8F08F0000020800200240EA
:10088000230167452CB8010878EB010800F801083E
:1008900038EF0108F8B53D4B5A899989914228BF34
:1008A0000022198A28BF5A81DA89914228BF002282
:1008B000D97828BFDA8139B1072905D00122344817
:1008C0009A7002700022DA71D8799A78002830D0B4
:1008D000102AB8BF10229A702E4A92F857200A2A7E
:1008E0002BD00C2A0CBF2C4C2C4C29B1072903D03F
:1008F0000A2A14BF2A4C2B4C00B12B4C2B4DAA7842
:10090000022A97BF2A49284E01EB82014E682979B5
:10091000A9B1013A032A37D831464FF07E5006F08C
:100920006DFD07F0ABFC2B88984228BF1846288045
:10093000F8BD032AB8BF0322CDE71E4CD5E798784F
:1009400006F054FC214606F0A5FC0746104D2C7815
:10095000204606F04BFC394606F09CFC014630462A
:1009600006F054FE80B13946304606F047FD06F0E9
:100970006DFE1028A8BF10200128B8BF0120C3B207
:100980009C4298BF04462C70F8BD00BF6C34002018
:1009900074200020803400200AD7A3396F12033955
:1009A0006F12833A0F506E3A6F120338B837002037
:1009B0002CB801085304E9382DE9F047FDF7B6FDDE
:1009C000194C1A4FDFF86C80BC4235D2184D00E04C
:1009D00015462E88002E00F07381AA19424580F03A
:1009E0006F81052E40F26C8123886988C3F30B0365
:1009F0009942EDD16B799B07EAD16168204695F861
:100A00000490F8F734FE2388B9EB133F0AD16388CA
:100A1000B21FC3F30B039A42A8BF1A46A91D606810
:100A200007F0C6FA1434CFE778EB010838EF010875
:100A300002F8010800000208A64A1178A1F1170384
:100A4000022B12D9A44BC80013F8314024B11C1852
:100A500064680CB91724147003445B782BB19F4B66
:100A600013F831300BB9182313709D4C6378022BA7
:100A700084BF002363702378022B84BF002323707C
:100A8000984B9A78042A40F010819A8AB2F57A7FBE
:100A900002D24FF47A729A82934D944A2B681A408C
:100AA00012B943F001032B602B68D80702D5904898
:100AB000F8F714FE2B68590402D58E48F8F70EFE9D
:100AC0002B681A0702D58C48F8F708FE2B689B04A0
:100AD0000FD58A48F8F702FE4FF40040F8F7FEFD04
:100AE000874B40209A79012A04BF00229A71F8F7B7
:100AF000F5FD844E00273368DFF864825A8C998CA8
:100B00003D46914224BF00225A84FFF7C3FEC246ED
:100B10004FF0FF0937F80820530803F077339008A7
:100B200000F03330D31A1B1AD00800F011301B1A12
:100B300003EB231303F00F3393FBF9F012F00101E1
:100B4000C0EB002018BF0135A3EB000318BFEDB2C6
:100B5000012B0DDD022B40F0B88011B112F42F7F74
:100B600006D10AEB0700FFF7F5FB002800F0AD8087
:100B70000837202FCED1013D022D00F2A680802023
:100B8000F8F7ACFD4FF40070F8F7A8FD4FF4003013
:100B9000F8F7A4FD4FF48020F8F7A0FD4FF4001003
:100BA000F8F79CFD4FF00070F8F798FD4FF080606B
:100BB000F8F794FD4FF00060F8F790FD4FF000500B
:100BC000F8F78CFD504B1B78012B05D84F4BDA788A
:100BD000022A04BF0122DA706378022B05D80C21A7
:100BE0004B4A01FB03234B4A13602378022B9FBF20
:100BF0004E21494A01FB0323336005F037FC3022C4
:100C00000021464809F005FE3068FDF7EBFC0020A6
:100C100005F0A2FB424A434B1179642280F00100A7
:100C20004A4318703468404BC8321C603F4B5A60CE
:100C300000229A60DA601A615A619A61DA6183F877
:100C4000202083F821203A4B3A4A136033F8062CCF
:100C5000394B1A80394B5B6B0BB1FCF777F9384D88
:100C6000384B28881E8806F0C1FA374906F012FB77
:100C7000364C6060688806F0B9FA334906F00AFB22
:100C80006B79334A23722B7920606372314B304683
:100C90001A6006F0ABFA01462F4806F0AFFBBDE83C
:100CA000F0472E4B1860FDF729BC002A7FF4F4AE04
:100CB0001A88B2F5F07F84BF4FF4F0721A80EBE629
:100CC00061682046F8F7D3FCACE62548F9F7D4FE76
:100CD00055E700BF8821002054B0010870AF01081B
:100CE000FC1F0020B8370020C82000200960000247
:100CF00008600002092000020160000209400002B1
:100D0000862B00209C200020C40A0020A620002062
:100D1000762000203C3C0020922F00202814002048
:100D2000982E0020000000205C140020982B00204A
:100D3000AC2000200C3C0020701500202420002056
:100D4000F4220020BC10002017B7D138542E002008
:100D50003661023D802E0020C0C9FB48C010002033
:100D60001637002008B5FFF7E9FCFFF725FEBDE8C0
:100D700008400120FAF7A4BA38B50D4C0D4DAC422D
:100D80000FD3F9F7DCF800220B4B0C481A705A709D
:100D90000B4B0C4A0C491A60BDE83840086003F060
:100DA000B7BA61682046F8F762FC1434E7E700BF81
:100DB00078EB010838EF0108FC1F0020922F00207B
:100DC0003C3C0020762000209C20002070B50C299F
:100DD00048D8DFE801F00747474748474747844777
:100DE0004747BE00038C158823F001031B041B0C2E
:100DF0000384038C8488018B23F0020321F07301A8
:100E00000904090C2943568815891B0435431B0C1A
:100E10002B43674DA4B2A8429BB20FD005F50065E5
:100E2000A8420BD005F54065A84207D005F58065BE
:100E3000A84203D005F58065A8420ED1558923F05C
:100E400008032B43958823F004032B43D689958907
:100E500024F4407435432C43A4B2D28884800183A7
:100E60008286038470BD038C148823F010031B0456
:100E70001B0C0384038C8588018B23F0200321F451
:100E8000E6410904090C41EA0421568814891B042F
:100E900034431B0C43EA0413454CADB2A04289B263
:100EA0009BB203D004F50064A04213D1548923F00F
:100EB000800343EA04134FF6BF741C409388D6891D
:100EC00044EA0313948925F44065344345EA8405D4
:100ED0009BB2ADB2D288858001830287C1E7038CC3
:100EE000148823F480731B041B0C0384038C8588F3
:100EF000818B23F4007321F073010904090C214351
:100F0000568814891B0434431B0C43EA0423284CE1
:100F1000ADB2A0429BB203D004F50064A04213D14D
:100F2000548923F4006343EA04234FF6FF341C4042
:100F30009388D68944EA0323948925F440553443A1
:100F400045EA04159BB2ADB2D28885808183828741
:100F500087E7038C158823F480531B041B0C038440
:100F6000038C8488818B23F4005321F4E641090427
:100F7000090C41EA0521568815891B0435431B0CD1
:100F800043EA05330A4DA4B2A84289B29BB203D00A
:100F900005F50065A84205D1958924F4804444EA0A
:100FA0008514A4B2D28884808183A0F8402058E7B9
:100FB000002C014030B598B10A4B00221C461D7927
:100FC000854207D19D79294202D004EB021030BD41
:100FD0000029FAD001320E2A03F11003EFD10020CC
:100FE00030BD00BFA0C6010801490248F9F7C0B8EA
:100FF000243B00200008004001490248F9F7B8B836
:10100000FC3A00200004004002494FF08040F9F70C
:10101000AFB800BFD43A002001490248F9F7A8B898
:10102000AC3A0020002C0140FFF7F6BF426A806A0C
:10103000131A5842584170474171704743799B07D2
:101040000AD5436A8269D154436A01690133B3FB0B
:10105000F1F201FB123343627047437913F002034C
:1010600008D00369426A806A013B101A1840C0B276
:10107000181A704718467047437913F001031FBFD1
:10108000C369026AC0689B1A1ABF00F1FF3018409A
:101090001846704710B54379014613F001030ED08E
:1010A000FFF7EAFF60B10B6A4A69CC68D05C013394
:1010B000B3FBF4F204FB1233C0B20B6210BD18464E
:1010C00010BD90F8433230B53BB9012490F841127D
:1010D00090F84232DAB2914200D830BDB0F84A52AC
:1010E00004FA03F22A43A0F84A220133F2E7836BA1
:1010F00019685A79012393400A8C9BB292B222EA72
:1011000003020A840A8C92B213430B84704738B5E9
:10111000A0F517746379A579DB0744D594F84032BC
:101120001BB3A06B0268938DC3F34E03938494F8B2
:101130005132012B07D094F8453223B1B4F84C3228
:101140000133A4F84C32E94301F0010103F0CFFC74
:10115000012384F84332002384F8413284F8423278
:1011600084F84032A4F84A3238BD94F8433220461D
:10117000012B04BF94F8413284F84232FFF7A1FFFB
:1011800094F843324BB90123E94384F843321940C0
:10119000A06BBDE8384003F0AABC002305F00101B4
:1011A00084F84332F4E738BD10B583790446DB0791
:1011B000006B4CBF2A214A21F9F70CFA012384F86D
:1011C000443284F840320023204684F84132BDE89E
:1011D00010408CE7084B10B41A681346B3FBF1F4C7
:1011E000B4F5803F03D3012BFAD95B08F6E7A1B22F
:1011F00010BCF9F721B800BF200000208160806B8F
:10120000E8E78379406BDB0744BFB1FA81F1490914
:1012100009B1F9F706BAF9F7FFB910B5A0F51574D9
:1012200063799A0714D594F84522002A59D1A36A04
:10123000616A994221D194F844324BB9A3791B07D2
:1012400006D5606B0621F9F7C5F92046FFF7ACFF1C
:101250006379D90740F1998094F84032002B40F02F
:10126000948094F841320133DBB2092B84F8413287
:101270004DD12046BDE8104023E7591CA069A1626A
:10128000C35C2069DBB25B0043F40073A4F848320E
:101290000A2381424FF0010184F8463294F8443227
:1012A00028BFA26284F84512002BD1D0A379180779
:1012B000CED5A06B02684079138C81409BB223EAA3
:1012C00001031384138C206B9BB213840621F9F75E
:1012D00081F90023122184F84432606BF9F77AF91E
:1012E000B6E794F946327BB1B4F8481220464B0871
:1012F000A4F8483201F00101FFF783FF94F8463269
:10130000013B84F84632A3E784F84532A0E70A2B74
:101310003BD194F843322BB9B4F84A3243F001037D
:10132000A4F84A32B4F84A02820501D4C3071AD499
:10133000B4F84E320133A4F84E320122002384F86F
:10134000402294F8432284F84132012A1DD1A17928
:10135000A06B84F8433201F0010103F0C8FB204682
:10136000BDE81040C3E6E36AC0F347000BB19847FD
:10137000E3E7E3696269D054E369E1680133B3FBF1
:10138000F1F201FB1233E361D7E710BD08B50A4A59
:101390001378D9070FD523F001031370074B9B78FF
:1013A0000BB1FEF72BFC0020F9F74AF9BDE8084025
:1013B0000420F9F7EDBE08BD2C2B0020D03300200F
:1013C0002DE9F041624E3378DD0705D5BDE8F041E7
:1013D00001210020F9F760B95E4D2B881C060BD562
:1013E0005D4B1A685D4B19794FF47A734B43934206
:1013F00002D8802005F07AF9594A5A4C1378904661
:101400006BB9594A20781778002870D137B104F0A9
:10141000DDFF002872D0082005F070F927701B202E
:1014200004F0D4FF00286DD0102005F067F904F017
:10143000E1FF00286AD0202005F060F94B4B1B78B3
:10144000180767D4232004F0C1FF002862D1402090
:1014500005F054F9464B4FF480601B88642B5DD92E
:1014600005F04CF9434B1B68590701D5628842B916
:10147000A2880AB19A0704D43F4BB3F8B430002BCA
:101480004FD04FF4006005F039F9242004F064FFD8
:1014900058B1242004F09AFF002847D033785B0726
:1014A00044D44FF4807005F021F998F8003083B9E6
:1014B0002B88002B3FD0314A127812B123F42063DD
:1014C000CBB3002004F082FFA8B34FF4007005F006
:1014D00015F92B8803B10223A371F8F755FFA36810
:1014E000C01A002831DBBDE8F041F9F791BB002FAD
:1014F00094D0184604F06AFF00288FD1082005F028
:10150000F5F88BE7102005F0F1F890E7202005F0C2
:10151000EDF893E7402005F0E9F89BE705F0E6F8E1
:10152000A0E74FF4006005F0E1F8AEE74FF48070FB
:1015300005F0E4F8B9E7002004F048FF0028C8D11E
:101540004FF4007005F0D2F8C3E7BDE8F08100BFAA
:101550002C2B0020BC2B002098220020FC1F0020F8
:1015600000000020042300202D2B0020491500201E
:101570002C1C00208421002080340020C220002068
:1015800070B5324D2B783BB1314C237823B93148BB
:10159000FBF740FC01232370FFF712FF2E4B1A8844
:1015A0002ABB2E4E3478E3074FD444F003032420A3
:1015B000337004F0D1FE10B144F0070434700A22F5
:1015C000274B4FF47A70B3F9043093FBF2F3254ABA
:1015D0001380254B254A1968AB7800FB0313D360B1
:1015E000002305201361BDE87040F9F7D1BD184B09
:1015F0001B781BB11E4BB3F8B43033BB92FAA2F385
:10160000002AB3FA83F308BF4FF0FF33174A0133C0
:1016100011698B4219D01361DBB29B00402BA8BF2C
:101620004023002214260A20052512495418565436
:1016300004326070A5709A4202EB010404F8010CB8
:10164000F4D3FF230E208B54CDE770BDC2200020C1
:101650004011002034350020BC2B00202C2B002012
:101660006C2E00208C1000209822002004230020E3
:1016700080340020B41F00202DE9F04F4FF418747F
:1016800087B099469DF84030804E019300F10A03DF
:101690003344009293F8E02403914443002105462B
:1016A000104693F8D4A40292FFF784FC0021059021
:1016B0005046FFF77FFC029A80461046F8F764FF19
:1016C00004905046F8F760FF019B06F1140713F0F1
:1016D0000803029307EB040B049A059B00F09C801F
:1016E000B8F1000F03D1002007B0BDE8F08F98F8E3
:1016F00007305B07F7D43319C3F84C8098645864FB
:1017000005F10B03DBB210B10B22C37182714FF4F0
:1017100018784FF0000A4FF4807208FB05685C4BA4
:10172000C8F82020C8F81430009BC8F82420C8F856
:101730001C309DF80430009988F81A30039BD8F8C3
:101740004C00C8F8403004F140033B44C8F828304E
:1017500004F5A0733B44C8F82C3088F81990C8F8F9
:1017600034A0C8F830A0C8F83CA0C8F838A088F861
:101770006452A8F860A2A8F862A288F858A288F873
:1017800059A2FFF727FD019BD8F84C0003F0010197
:1017900003F0ADF93F4A04F51773C8F870223E4ACA
:1017A00004F5157419F0020F3B44C8F86822274469
:1017B000C8F86CA25FD0D8F8500000285BD0D8F8E9
:1017C0004C10026809688A4255D00122009988F8B5
:1017D00065220193FFF7FEFC3A465146D8F85000C7
:1017E000F8F77EFD019B52461946D8F84C00F8F7F1
:1017F00077FD029B5BB94FF4187303FB056512215B
:10180000A86CF8F7E7FE01215846FFF7FAFC5846A6
:10181000FFF7CAFC584667E719F0010E10D0002BFD
:101820003FF461AFD97949073FF55DAF3119CB641A
:1018300005F10B034A64DBB212B10C21D371917133
:1018400019F0020F3FF463AFBAF1000F3FF44BAF52
:101850004FF418730D4A03FB05239864BEF1000F83
:1018600006D1B8F1000F3FF43EAFC3F84C8047E714
:10187000C3F8508044E74FF41870002200FB056065
:10188000194680F865223A46C06CB0E70423002070
:101890003CB801080F1101081B1201081FB50123F4
:1018A000ADF808300023ADF80C30ADF80A30094B24
:1018B000ADF8041093F8F83401A9012B08BF0323F5
:1018C000ADF8062008BFADF80C30FEF745FA05B0BC
:1018D0005DF804FB042300202DE9F84F0024804626
:1018E00025464FF00D0ADFF85090DFF850B00AFBA4
:1018F000049637684146384609F01CF878B13946F5
:101900005846F9F713FE00213046F9F7B1FF04F00D
:1019100007FD3046F9F70AFF04F002FD01350134F6
:10192000BA2CE4D125B9BDE8F84F024804F00EBD49
:10193000BDE8F88FF9CB010864B8010817CA01089F
:101940002DE9F74F804604F0E1FE054628B1012855
:1019500020D198F800302A2B1CD1774804F0F6FCEF
:1019600000244FF00D09DFF8D881744F09FB04867D
:1019700038463168F9F7DAFD291C18BF01213046D5
:101980000134F9F775FF04F0CBFCBA2CEED103B0AB
:10199000BDE8F08F3D21404608F070FF002800F0C0
:1019A000C680064616F8013C721E202B48D0A6EBD6
:1019B00008060130044623780130202BFAD0002796
:1019C0000D23DFF87CA1F6B203FB07A5D5F8009044
:1019D0000193484604F09AFE494602468346404633
:1019E00008F05AFF019B8146002840F09680B345DD
:1019F00040F093802B7903F03003102B22D0202B62
:101A000051D08BBB204606F0ABFAB5F9053001B2D8
:101A10008B4229DCB5F907308B4225DB2846F9F7E4
:101A2000DCFC0D23464A474803FB07273968F9F7D2
:101A30007DFD0021284603B0BDE8F04FF9F718BF3F
:101A40001646AFE706468146834695F805803C4B2F
:101A500003EBC80898F878A9564502D2B9F1000FEF
:101A60000BD0BBF1000FDCD1374804F06FFC2846E7
:101A700003B0BDE8F04FF9F759BED8F874392146E4
:101A800053F8260008F0CDFE00280CBF4FF00109E6
:101A90004FF0000905D131B22846F9F79EFC4FF00E
:101AA000010B0136D8E70D268346254B95F80580B6
:101AB00006FB0736C845D4DD23461C462178013392
:101AC0002029FAD02C21204608F0D8FE824618B9E9
:101AD00008F1FF334B4513D1337903F00303022B95
:101AE00011D0032B0FD02846F9F76AFC8346204615
:101AF00006F036FA0BF809004FF0010B0AF1010469
:101B000009F10109D6E72846F9F75AFC8346204631
:101B100006F026FA2BF81900EEE70137BA2F7FF40A
:101B200053AF0A4803B0BDE8F04F04F00FBC404685
:101B300003B0BDE8F04FCFE67DD8010817CA010811
:101B400064B8010890D801089BD80108F9CB0108B6
:101B500038B504460B4D2046F9F7EEFB30B10A4B81
:101B60000A485978BDE83840F9F746BC204606F0E7
:101B7000F7F9022804D8C0B204F034FA2C46EAE798
:101B800038BD00BFEDC70108FC1F0020A9D801081F
:101B900070B504460A4E0B4D2046F9F7CDFB30B127
:101BA000074B09481978BDE87040F9F725BC204675
:101BB00006F0D6F9022802D830702C46ECE770BD4A
:101BC000FC1F0020EDC70108ADD801082DE9F7433F
:101BD0000546F9F7B1FB044620B1F9F7EBFB03B07A
:101BE000BDE8F083284601AA2F4906F015FA2646DB
:101BF00025462E4FDFF8CC80DFF8CC9070B9022C50
